:020000040800F2
:1000000000200010E13103084932030801D600083E
:10001000493203084932030849320308000000004E
:10002000000000000000000000000000493203084A
:10003000493203080000000049320308892A0008F9
:100040004932030849320308493203084932030898
:100050004932030849320308693C0008953D00080D
:10006000593D00081D3D0008E13C0008D19B0008F7
:10007000C19B0008B19B0008A19B0008919B000850
:100080007D9B0008699B0008493203084932030838
:10009000493203084932030849320308A53C0008E5
:1000A000B1180008BD1B0008E5170008391D00083D
:1000B000011B0008451A00087D1900084932030891
:1000C0004932030849320308493203084932030818
:1000D00049320308C12B0008452B0008C92A000833
:1000E0002D3C00084932030849320308493203080D
:1000F00049320308493203084932030849320308E8
:100100000000000000000000000000004932030869
:10011000493203084932030879EC010865EC01080B
:10012000559B0008419B00082D9B0008199B000867
:10013000059B000849320308000000000000000091
:10014000493203084932030849320308000000001D
:10015000000000000000000000000000000000009F
:100160000000000000000000493203084932030883
:1001700049320308000000000000000000000000F9
:080180000000000049320308F1
:10018800436A8269D154436A0169C26B01338B4265
:1001980028BF002343623AB370B4EFF311835022AF
:1001A80082F31288C66B3268D20704D5DBB283F3B8
:1001B800118870BC7047716869B9D0E909429442E6
:1001C80018D085691544F56018D9A21A726084623E
:1001D800002280F85820326842F00102DBB2326017
:1001E80083F3118870BC7047426D136843F0800335
:1001F80013607047012280F85820D7E70469A21AD3
:1002080072608162E4E700BF034610B4846BD9686A
:10021800406954B19A6C8C1A013A005D5DF8044B40
:1002280008BF0A46C0B29A6470471A6A805C0132F5
:100238008A4228BF2246C0B21A625DF8044B704752
:10024800C36B13B190F858007047D0E90903181A26
:10025800B0FA80F040097047D0E909120369914269
:1002680038BFC9188A1AC16B013B19B149680A44D9
:100278009A4201D2981A704700207047836B43B1A5
:10028800826C5B689A4291BF981AC0689B1AC01822
:100298007047D0E907239A422FBFD01AC068801848
:1002A800C01A70470A4B30B503F1140493F90020C3
:1002B8005D78072AC8BF143A811804330D7313F800
:1002C800025C855413F8012C0A769C42EED130BDAD
:1002D8007036030803682DE9F0415D6A1DB12B46AD
:1002E800BDE8F0411847002A174611DD04460E46BE
:1002F8000F4400E023689B68204698470028F9D0FF
:10030800236816F8011B1B6820469847BE42F1D1A6
:10031800BDE8F08103681B69184700BF002323224A
:10032800027043708370C370704700BF437A5A1CD1
:100338000344D2B242729972037A93420AD84AB1FC
:1003480010B5044604F10A01D0E9003098470023AB
:10035800637210BD7047CB0702D4024B024ADA60C1
:10036800704700BF00ED00E00400FA0520B10078F6
:10037800B0FA80F04009704701207047037903F014
:100388001803082B0AD002D82BB100207047102B75
:1003980016D0182BF9D1B0F80B007047114BB0F8F4
:1003A8000B0093F90030591C06BF0F4B1B78DBB2CA
:1003B800C3EB0312C3EB820300EB430080B2704728
:1003C800084BB0F80B0093F901305A1C06BF064BD6
:1003D8005B78DBB203EB430203EB820300EB4300E1
:1003E80080B2704700000020E4140020F0B50679C0
:1003F80006F06003402B09D144794FF0FF35002304
:10040800012006F00706A3420BD1F0BD602B08BF00
:1004180045794FF001040CBF04FA05F54FF0FF359C
:10042800EDE7042E0CD8DFE806F0030D18242E00A3
:1004380030B1C85CD75C784028420CBF012000204E
:100448000133E0E70028FBD0C856D756A0EB070CCD
:10045800DCF1000040EB0C00F2E70028F0D031F8A6
:10046800130032F81370784028420CBF0120002096
:10047800E6E70028E4D031F9130032F91370C71BFE
:1004880078427841DCE70028DAD051F8230052F8A6
:100498002370784028420CBF01200020D0E745E7B0
:1004A80090ED057A90ED004AD0ED066AD0ED014A4C
:1004B800D0ED047A90ED035AD0ED025AA4EE007AFA
:1004C800B0EE406AB0EE470AB0EE667AA4EE867ADD
:1004D80067EEC07AA5EE407AE5EE867A80ED057A79
:1004E800C0ED067A704700BFD0ED057A90ED013A6D
:1004F800D0ED003AD0ED064A90ED024A90ED077A29
:1005080090ED035A90ED086AD0ED045AC0ED067AD2
:10051800F0EE406A27EE830AC0ED056AA3EEA60A4C
:1005280080ED087AA4EE240AA5EE470AA5EEC60ACD
:1005380080ED070A704700BFD0ED007A90ED017A90
:1005480030EE670AE7EE007AB0EE670AC0ED007A8F
:10055800704700BF704700BF0378202B024600F1A8
:100568000100F9D0092BF7D02D2B00F0A4802B2BFC
:1005780003BF5378B7EE000A0246B7EE000AA3F1AC
:100588003001C8B209289FED577A10D8F2EE046AF4
:1005980007EE901AF8EEE77A12F8013FE7EE267AAE
:1005A800A3F13001C8B20928B0EE677AF0D92E2B32
:1005B80063D003F0DF03452B02D020EE070A704713
:1005C80010B451782D294FD02B2979D0A1F13003BF
:1005D800092B02F101027AD80024002303EB8303DC
:1005E80001EB430312F8011FA1F130000928A3F120
:1005F8003003F3D9B3F59A7F1A4628BF4FF49A729D
:10060800072B6CD9DFED386A1346F7EE007A083B02
:10061800072B67EEA67AFAD802F00702DAB1F2EEF3
:10062800046A012A67EEA67A15D0022A67EEA67A2E
:1006380011D0032A67EEA67A0DD0042A67EEA67AAF
:1006480009D0052A67EEA67A05D067EEA67A062AAB
:1006580018BF67EEA67A002C3BD087EE277A5DF8A4
:10066800044B20EE070A70479178A1F13003092B5B
:1006780002F1020230D80124AFE75378A3F1300128
:10068800C8B2092802F1010293D8F2EE046AF0EE2A
:10069800665A07EE901AF8EEE77A12F8013F87EEED
:1006A800A66AA3F13001C8B2092866EEA56A37EE3A
:1006B800067AEED97DE75378BFEE000A02465EE778
:1006C8009178A1F13003092B02F1020284D9F7EEE7
:1006D800007A27EE277AC2E7F7EE007ABDE7F7EE51
:1006E800007A9BE70000000020BCBE4C0028F0B454
:1006F80003DA2D230B7040420131092804464FF0DC
:10070800010307DD03EB83035B00B0FBF3F2092A67
:10071800F8D883B10F48A0FB0326B4FBF3F2092AEB
:1007280002F1570C02F1300709DD03FB1244F3080C
:1007380001F801CBEFD100230B70F0BC704703FB2D
:100748001244F30801F8017BE5D100230B70F0BCDB
:10075800704700BFCDCCCCCC884270B44FF00104B8
:1007680042D301FB04F4B0FBF4F58D42F9D2ECB1AD
:1007780042BB092D04FB150005F1570605F13002AF
:100788000EDDB4FBF1F403F8016B7CB1B0FBF4F5BA
:10079800092D04FB150005F1570605F13002F0DCC0
:1007A800B4FBF1F403F8012B002CEFD100221A70EE
:1007B80070BC704703F8016BB4FBF1F4002CF5D062
:1007C800B0FBF4F5092D04FB150005F1370605F11A
:1007D8003002EFDCB4FBF1F403F8012B002CEFD16D
:1007E80000221A7070BC70470546002AEAD1C0E79B
:1007F80003685A1C02601970704700BF2DE9F04762
:10080800089C2578002B804689460CBF4FF0200AAB
:100818004FF0300A661C25B3002A26DD334601E076
:10082800024698B113F8011B501E0029F8D1971EF3
:1008380060B13D46013D51464046C8476B1C002B00
:10084800F8DC257827EAE770013045B1041B294612
:100858004046C847301916F8015B002DF7D1BDE8AE
:10086800F087002A03DC2846F9E70020EEE7571E48
:10087800DFE700BF034600F11001FF221A705A702B
:1008880002339942FAD1027042708270C2700271CA
:1008980042717047FF2310B42E212D242F2244715A
:1008A8008171C271C370037103724372437383739E
:1008B8005DF8044B704700BF10B400223D240123AB
:1008C80004218471C17102704271437003715DF833
:1008D800044B7047084B09498B4203D309E0143392
:1008E8008B4206D21A88C2F30B029042F7D11846FF
:1008F800704700231846704770B9030820BE0308E4
:1009080070B50546B0F80900FFF7E4FF064B1E78FE
:1009180004462846FFF732FD16B1A368184470BD97
:1009280063681844FBE700BFB80E002038B50546D9
:100938000C46FFF7E5FF2A7902F0070302F0600290
:10094800602A28D1022B0ED0042B18D03BB96A7923
:1009580001239340DBB2027814B11343037038BD0E
:1009680022EA0303FAE76A79012393409BB20288DB
:1009780014B113430380F2E722EA0303FAE76A7922
:10098800012303FA02F2036814B113430360E6E794
:1009980023EA0203FAE7042BE1D8DFE803F00303B4
:1009A800050507000470DAE70480D8E70460D6E795
:1009B800002306214FF47A720170C0E90123037302
:1009C800704700BF2C22022302704370704700BF9B
:1009D80008307047704700BF81617047012380F875
:1009E8005030704790F8213033B1012B03D14FF4C8
:1009F80000630383704770474FF480630383704735
:100A0800704770474378007840EA032010FB01F0F4
:100A18004FF4807190FBF1F000F30F0000B27047C3
:100A28002DE9F04FDFF8DCC1754CDCF80450228862
:100A3800B4F90AA0C2EB25135200C2EBE502B4F9DF
:100A480002505B436A43B4F904501B135D43AD1372
:100A580005EBE225B5F5FA324FEAE57B85B04BF1B7
:100A6800FF33CDE90023DDE900325343009AA56145
:100A7800A2FB0289CDE90201B4F908200199009886
:100A880009EB43095143D31700FB0311A2FB0023D1
:100A98000B444FEAEA7B0AFB09F11F0308FB0B131F
:100AA800AAFB080119444FEA102A4AEA016A160308
:100AB8004FEA212B47EA12571AEB0602E6884BEB5E
:100AC800070312F1000A43F5004BAAFB060106FBD7
:100AD8000B114A10CB1752EA030100F08E80B4F9CB
:100AE8001060009806FB09F1F71708FB0711A6FB31
:100AF80008673944B4F90E808B4601994FEAE879C2
:100B080008FB01F100FB0911A8FB00898944DCF806
:100B180008104FEA4947C1F5801C47EAD837B24662
:100B28004FEA4846B4F90C801AEB060A66464BEBC6
:100B3800070BF7174FEAC806019600260096F90733
:100B4800DDE900674FEACC7016EB0A0647EB0B07A6
:100B580041EA5C01801B61EB070140F6354C894690
:100B6800A0FB0C010CFB091132F06AF9B4F916204C
:100B7800B4F914A04E13470B47EAC14702FB06FC21
:100B8800D31707FB03CCA2FB07236344564307FB99
:100B98000366A2FB07233344560E46EAC3163218EF
:100BA8004FEA636747EB010380460AFB01F14FEA0E
:100BB800EA7B08FB0B17AAFB08013944C60C46EA76
:100BC800413612EB06084FEAE147B4F9122043EB2D
:100BD80007094FEA182141EA096113010B44029AF7
:100BE8000AB11B0A1360039B23B105EB8505803509
:100BF8002D121D6005B0BDE8F08F0023EFE700BFA0
:100C0800246D0020B80E002070472DE9F041334BC9
:100C1800334E9A897489B6F91450B6F90480B6F936
:100C28000E70B6F920C01B69121B34895443E213B5
:100C3800B6F912401544E40294FBF5F4B6F90250F3
:100C48001444A4F57A6E0EFB0EF20EFB05F50EFBAE
:100C580008FEB6F90C80F4611213574302FB08F240
:100C6800121402EB6E32ED1205EBE7270232B6F9E9
:100C78000050B6F806E0921002F5004207EB85072F
:100C88000EFB02F207FA0CF74FEAD23E02374CF29B
:100C98005032A3EBA70742FA0CF37B4355BF5B0026
:100CA800B3FBFEF3B3FBFEF35B0078B11A1202FB51
:100CB80002F540F6DE326A430A4D12145D4302EB38
:100CC800254202F6CF6203EB2213036021B10A2307
:100CD8005C43083424110C60BDE8F081B80E002094
:100CE800EC6C002043E3FFFF6D4B2DE9F04F5C698E
:100CF8006C4BB3F80AE0B3F804809A894FEA0E2ADD
:100D0800B4EB0A044FEA1E6B4FF0000587B065EBA1
:100D18000B05CDE900450746009C1889019EA0FBFC
:100D2800044500FB0655E00940EA45604FEA0844DF
:100D38008C46E9114FEA184510EB0408D888009C46
:100D480041EB0509CDE90489A0FB0445B3F802800D
:100D580000FB0655200A40EA05604FEAC83429120C
:100D68004FEA584510EB040841EB05090099A2FB2E
:100D7800010102FB06114FEAD05A4AEA412A1AF544
:100D8800FA634FEAE15B4BF10004B3F5FA6FCDE982
:100D9800023474F10003424E64DA0524AAFB04010C
:100DA80004FB0B1100FB0BF40AFB0144DDE90423EF
:100DB800A0FB0A0121444D104FEA3004121B4FEAF0
:100DC800900463EB050344EA8174B8EB0408CDE9A9
:100DD8000423DDE9023434484FEAA10569EB05092B
:100DE8004FF0FF31834274EB010326DA40F6AC5032
:100DF8001AEB00024FF000014BEB010302FB03F179
:100E0800A2FB022303EB4103D400DD00101B45EADB
:100E1800527563EB0501DDE9044524184D41CDE920
:100E280004450B24A2FB040104FB031149104FEAFB
:100E38003000B8EB000869EB0109DDE900325343E3
:100E4800009ADDE90201A2FB02AB0BEB430B4FEA70
:100E5800DA7242EA4B02801A4FEAEB7361EB030144
:100E6800CDE9020197B1B169A1FB082301FB093360
:100E7800540D5D1544EAC324DDE90423A21A65EB89
:100E880003031D46D30B43EA45433B60BCF1000F07
:100E980002D0029BCCF8003007B0BDE8F08F00BF4D
:100EA800B80E0020106D002024FAFFFF13B50C4681
:100EB8006A4603210C3016F025FDA0B19DF80020EC
:100EC8009DF8013043EA022323809DF802209DF813
:100ED800033043EA0223A3809DF804209DF80530DF
:100EE80043EA0223638002B010BD07B5F7216A46C2
:100EF80016F008FD9DF801309DF800100B4A1B0103
:100F080043EA01339DF8021043EA111393609DF8F8
:100F180004309DF803101B0143EA01339DF80510C6
:100F280043EA1113536003B05DF804FBB80E0020C8
:100F380070B4D0E90041057B02690223AB406360CD
:100F48000B684FF6FE7003400B60EFF311835021DE
:100F580081F31288D66B3168C9071CD4706870B9E0
:100F6800D2E909418C4213D095690D44F56017D830
:100F78001469611A71609062002182F85810326811
:100F880042F00102DBB2326083F3118870BC704713
:100F9800012182F85810DBB283F3118870BC7047C6
:100FA800611A71609462E7E770B40468037B226891
:100FB800022101FA03F31A4216D0026911481249B4
:100FC800642505FB02020D785068016875B915693A
:100FD800528928684FF6FE7630402860C868D243A8
:100FE80092B20240CA60636070BC704700690268D0
:100FF8004FF6FE752A400260CA684FF6FF6002404D
:10100800CA60F0E7D43C0020D03C002038B5074C3B
:10101800074DAC4203D3074B00221A7038BD6288D3
:10102800D4E9010132F0A9FA1434F2E770B90308DF
:1010380020BE0308B80E002038B5074C074DAC4257
:1010480003D3074B01221A7038BD6288D4E9011016
:1010580032F093FA1434F2E770B9030820BE03089B
:10106800B80E002010B42721262401220023047082
:1010780041708270C3705DF8044B704770B5448846
:101088000546C4F30B0422460846002132F099FABB
:101098002969094A9142034602D3084A914204D376
:1010A80041B11846BDE8704008472246BDE8704087
:1010B80032F063BA70BD00BF20BE030830BF03081A
:1010C80010B50368017B1A6802238B40134204465B
:1010D8000FD00F4AD3690133202BD3610AD11822CC
:1010E80000210C4832F06DFA217B226802238B40E4
:1010F800536010BD222BF7D10023D361064A137029
:101108004268136823F001031B041B0C1360EBE710
:10111800B80E0020681400205B14002030B40223AD
:1011280014210122152522240372417000234FF651
:10113800FF714571C47002700271827043818381AE
:10114800C3810182817430BC704700BF30B504464A
:10115800406D21710368A26823F00103036087B022
:101168006379009213F0040F4FEA03324FEA032326
:1011780014BF4FF48055002503F4806302F4005235
:101188000195CDE90223002511F0010305952ED123
:10119800049308238D07694648BF04931AF09EFC00
:1011A8002079636D617900F00202002A15BF4FF4BF
:1011B80040324FF480324FF40034002410F0010F15
:1011C800586808BF2246CC074CBF024320EA0202F7
:1011D8005A609A6809074CBF42F0080222F00802D8
:1011E8009A601A6842F001021A6007B030BD042301
:1011F80004930C23CEE700BF30B50446406DA160D0
:10120800036823F0010303606379257987B013F03D
:10121800040F4FEA03324FEA032303F4806302F416
:101228000052CDE90223009114BF4FF480510021F0
:10123800EB0748BF042301914FF00001CDE90411E9
:1012480054BF08230493694648BF0C23AD0748BF21
:1012580004931AF043FC2079636D617900F002026F
:10126800002A15BF4FF440324FF480324FF4003457
:10127800002410F0010F586808BF2246CC074CBF65
:10128800024320EA02025A609A6809074CBF42F0FA
:10129800080222F008029A601A6842F001021A60F5
:1012A80007B030BD08B5202132F0A2F90346184630
:1012B80023B10278202A03F10103F8D008BD00BF4A
:1012C80001211BF02FB970B50D461446FFF7EAFF50
:1012D8000646A0B1FFF7F4FF40F634039842A8BFD2
:1012E8001846B0F5617FB8BF4FF461701923A0F5B7
:1012F800617090FBF3F02870237801332370304637
:10130800FFF7D0FF0646A0B1FFF7DAFF40F6340337
:101318009842A8BF1846B0F5617FB8BF4FF4617016
:101328001923A0F5617090FBF3F0687023780133FE
:101338002370304670BD7FB5002500F10C060C46C1
:101348000D804D808D800DF107020621304616F084
:1013580073FA10B9002004B070BD9DF807305B0720
:10136800F8D502AA2946304616F0CCFA0028F1D062
:101378009DF809209DF8083043EA022323809DF850
:101388000B209DF80A3043EA022363809DF80D2064
:101398009DF80C3043EA0223A380DCE738B52C2201
:1013A800002132F00EF9034640F2DC51642040F28D
:1013B8001A4240F2022418745982132019219A8281
:1013C80040F2753240F26C751C8398760E24022028
:1013D8001977DA830A210122DD8283F82A0040F690
:1013E800430583F82B1083F822409A7383F825204D
:1013F80083F829201D8419460248BDE8384030F09A
:1014080085BD00BF387E0308014B18600CF026B973
:10141800C038002070B5244924480A784B78CD7B21
:101428002349244EC2EB0214C2EB840203EB4304AB
:10143800002D03EB8403204D204C01EB430300EB0C
:10144800420214BF2821202133602260296028F03D
:101458007DFC302200211A4832F0B3F8206824F0CD
:10146800CBFB28F0E5FB174A17491079174A184BA8
:101478001160C822642111FB00210022C3E9011276
:10148800C3E90322C3E90522DA6183F8202083F83F
:10149800212030F019F80F4BBDE8704093F8221066
:1014A800188C27F01BBA00BFE41400201015002088
:1014B800B01600208C1E0020D00700200015002048
:1014C800A462002008590020681C0020EC100020AD
:1014D8007C170020B80E00200C290ED8DFE801F098
:1014E8001B0D0D0D140D0D0D0E0D0D0D0700C3690F
:1014F80023F4006343EA0222C2617047C36923F000
:1015080008031A43C2617047836923F4006343EAFE
:10151800022282617047836923F008031A438261BB
:10152800704700BFF0B40C292BD8DFE801F0752A0A
:101538002A2A502A2A2A2C2A2A2A0700046AB2F8B8
:101548000CC0978816686B4D24F480540462036AB3
:101558004468C16923F4005343EA0C3321F4E6419B
:10156800A84243EA073341EA062100F0BC8005F5AA
:101578000065A84200F0B78092684460C1610264C7
:101588000362F0BC7047046AB2F80CC0978816680A
:10159800584D24F480740462036A4468C16923F4D2
:1015A800007343EA0C2321F07301A84243EA07239E
:1015B80041EA060100F0848005F50065A8427FD065
:1015C80092684460C161F0BCC26303627047046AF8
:1015D800B2F80CC097881668464D24F010040462CF
:1015E800036A4468816923F0200321F0807143EA8B
:1015F8000C1321F4E641A84243EA071341EA062105
:101608004BD005F50065A84247D0926844608161D7
:10161800F0BC826303627047046A9389B2F804C01D
:101628001768344E24F001040462046A456881692D
:1016380021F4803124F0020443EA0C0321F0730101
:10164800B04243EA040341EA07010ED02A4CA04203
:101658000BD004F54064A04207D004F58064A04292
:1016680003D004F58064A04210D1D489168A578A21
:10167800B2F806C023F00803234325F4407523F08D
:10168800040346EA07044CEA0303254392684560CD
:101698008161F0BC426303627047D589178AD68896
:1016A80023F0800343EA051324F44064558A23F0A9
:1016B800400344EA870443EA061344EA8504A4E79E
:1016C800D589178AD68823F4006343EA052324F4CE
:1016D8004054558A23F4806344EA071443EA0623F6
:1016E80044EA05146CE7158A24F4804444EA851416
:1016F80042E700BF002C0140003401402DE9F047CB
:101708004FF48C7200212948294D2A4E2A4FDFF8C0
:10171800B880DFF8B890DFF8B8A031F052FF274A58
:101728002748DFF8B0C0DFF8B0E002F5CC7119E067
:10173800B3F1804F23D0B34226D0BB4226D06345B5
:1017480026D0734526D0434526D04B4527D0534550
:1017580028D01C4CA34208BF4FF4802407D018326D
:101768008A420AD013688342E2D14FF40064AB691D
:10177800183223438A42AB61F4D1BDE8F0870123D4
:10178800EC692343EB61EAE70223F9E70423F7E76F
:101798001023F5E72023F3E74FF40054E7E74FF46D
:1017A8008034E4E74FF40034E1E700BFD82E00208E
:1017B80000100240000400400008004020630308B5
:1017C800002C014000480140003401400040014025
:1017D8000044014000100040001400402DE9F84387
:1017E8002F4D2A69EB6812EA030826D02D4E4FF0D8
:1017F8000047B8FA88F327FA03F2D2431B3B2A6161
:1018080008EA0208042B15D8DFE803F0372D23195E
:101818000300D6F81431002B39D1EB6A1FFA83F98B
:10182800D6F8104134B12368204649469847646881
:10183800002CF8D1B8F1000FDBD1BDE8F883D6F859
:10184800F000696B036889B29847B8F1000FD0D1EE
:10185800F3E7D6F8F400A96B036889B29847B8F1A2
:10186800000FC6D1E9E7D6F8F800E96B036889B23A
:101878009847B8F1000FBCD1DFE7D6F8FC00296C17
:10188800036889B29847B8F1000FB2D1D5E703F1E0
:10189800FF3900231FFA89F9C6F81431C0E700BFE1
:1018A80000480140D82E00202DE9F8432F4D2A6921
:1018B800EB6812EA030826D02D4E4FF00047B8FA1D
:1018C80088F327FA03F2D2431B3B2A6108EA02088D
:1018D800042B15D8DFE803F0372D23190300D6F8B9
:1018E800C430002B39D1EB6A1FFA83F9D6F8C0400F
:1018F80034B123682046494698476468002CF8D1DB
:10190800B8F1000FDBD1BDE8F883D6F8A000696B09
:10191800036889B29847B8F1000FD0D1F3E7D6F839
:10192800A400A96B036889B29847B8F1000FC6D123
:10193800E9E7D6F8A800E96B036889B29847B8F1D7
:10194800000FBCD1DFE7D6F8AC00296C036889B278
:101958009847B8F1000FB2D1D5E703F1FF3900235A
:101968001FFA89F9C6F8C430C0E700BF004001403B
:10197800D82E00202DE9F8432E4D2A69EB6812EA8B
:10198800030826D02C4E4FF00047B8FA88F327FA00
:1019980003F2D2431B3B2A6108EA0208042B15D83C
:1019A800DFE803F0352B22190300D6F89C30002B12
:1019B80037D1EB6A1FFA83F9D6F8984034B1236817
:1019C8002046494698476468002CF8D1B8F1000FC2
:1019D800DBD1BDE8F883B06F696B036889B29847BB
:1019E800B8F1000FD1D1F4E7F06FA96B036889B2A1
:1019F8009847B8F1000FC8D1EBE7D6F88000E96B3B
:101A0800036889B29847B8F1000FBED1E1E7D6F86C
:101A18008400296C036889B29847B8F1000FB4D1E3
:101A2800D7E703F1FF3900231FFA89F9C6F89C307C
:101A3800C2E700BF00080040D82E00202DE9F84377
:101A48002B4D2A69EB6812EA030824D0294E4FF07F
:101A58000047B8FA88F327FA03F2D2431B3B2A61FE
:101A680008EA0208042B13D8DFE803F0322920170C
:101A78000300736F002B34D1EB6A1FFA83F9346FBC
:101A880034B123682046494698476468002CF8D149
:101A9800B8F1000FDDD1BDE8F883306D696B0368DC
:101AA80089B29847B8F1000FD3D1F4E7706DA96BEC
:101AB800036889B29847B8F1000FCAD1EBE7B06D57
:101AC800E96B036889B29847B8F1000FC1D1E2E722
:101AD800F06D296C036889B29847B8F1000FB8D146
:101AE800D9E703F1FF3900231FFA89F97367C6E7BD
:101AF80000040040D82E00202DE9F8434FF080451F
:101B08002A69EB6812EA030824D0294E4FF00047EF
:101B1800B8FA88F327FA03F2D2431B3B2A6108EA92
:101B28000208042B13D8DFE803F03229201703003A
:101B3800F36C002B34D1EB6A1FFA83F9B46C34B11F
:101B480023682046494698476468002CF8D1B8F1C4
:101B5800000FDDD1BDE8F883B06A696B036889B20C
:101B68009847B8F1000FD3D1F4E7F06AA96B03687E
:101B780089B29847B8F1000FCAD1EBE7306BE96B2F
:101B8800036889B29847B8F1000FC1D1E2E7706BDA
:101B9800296C036889B29847B8F1000FB8D1D9E722
:101BA80003F1FF3900231FFA89F9F364C6E700BF80
:101BB800D82E00202DE9F8435A4D2A69EB6812EA1D
:101BC800030825D0584E4FF00047B8FA88F327FA93
:101BD80003F2D2431B3B2A6108EA0208042B14D8FB
:101BE800DFE803F04A41382F0300736A002B40F006
:101BF8009280EB6A1FFA83F9346A34B1236820466D
:101C0800494698476468002CF8D1B8F1000FDCD138
:101C1800464D2A69EB6812EA03084AD0424E4FF053
:101C28000047B8FA88F327FA03F2D2431B3B2A612C
:101C380008EA0208042B39D8DFE803F05B51473D76
:101C480027003068696B036889B29847B8F1000FBC
:101C5800BBD1DDE77068A96B036889B29847B8F112
:101C6800000FB2D1D4E7B068E96B036889B298472E
:101C7800B8F1000FA9D1CBE7F068296C036889B2E5
:101C88009847B8F1000FA0D1C2E7D6F8EC30002B86
:101C980039D1EB6A1FFA83F9D6F8E84034B12368E2
:101CA8002046494698476468002CF8D1B8F1000FDF
:101CB800B7D1BDE8F883D6F8C800696B036889B264
:101CC8009847B8F1000FACD1F3E7D6F8CC00A96B70
:101CD800036889B29847B8F1000FA2D1E9E7D6F8AE
:101CE800D000E96B036889B29847B8F1000F98D122
:101CF800DFE7D6F8D400296C036889B29847B8F1B1
:101D0800000F8ED1D5E703F1FF3900231FFA89F9B7
:101D1800C6F8EC30C0E703F1FF3900231FFA89F950
:101D2800736269E7002C0140D82E0020004401406E
:101D38002DE9F8432B4D2A69EB6812EA030824D0F1
:101D4800294E4FF00047B8FA88F327FA03F2D24336
:101D58001B3B2A6108EA0208042B13D8DFE803F0CA
:101D6800322920170300736A002B34D1EB6A1FFA5B
:101D780083F9346A34B12368204649469847646831
:101D8800002CF8D1B8F1000FDDD1BDE8F883306838
:101D9800696B036889B29847B8F1000FD3D1F4E7AB
:101DA8007068A96B036889B29847B8F1000FCAD167
:101DB800EBE7B068E96B036889B29847B8F1000FA0
:101DC800C1D1E2E7F068296C036889B29847B8F195
:101DD800000FB8D1D9E703F1FF3900231FFA89F9B9
:101DE8007362C6E7002C0140D82E0020F0B50668C3
:101DF8004D4CB30AA34200F094800AD94B4CA3423D
:101E080000F089800134A34266D0023CA34267D027
:101E1800F0BD4A3CA34200F081800134A34205D0C2
:101E2800B3F5801FF4D14827012501E09827032541
:101E380090F805C002232CFA03F084468340A800DA
:101E4800002955D0D6F80CE044190CEB440C9BB291
:101E5800374C43EA0E030CF1040E44F82C1044F8F6
:101E68002E20F360E319EFF31181502282F31288D8
:101E7800421904EBC202D2F810C0BCF1000F03D023
:101E880044F807C013690433421904EBC2025769C6
:101E980017B11F6053690433421904EBC2029769F2
:101EA80017B11F6093690433421904EBC202D76962
:101EB80017B11F60D36904330022C9B21A6081F3D5
:101EC8001188284404EBC004236A63B9F3684FF609
:101ED800FE721340F360F0BD4FF488770625A7E73C
:101EE800C0270425A4E7F36843F00103F360F0BDBD
:101EF800D6F80CE00E4CDB439BB203EA0E0300EB72
:101F0800050E0CEB4E0CF3600CF1040344F82C1096
:101F180044F82320A6E7E827052589E77027022546
:101F280086E72027002583E74B00100051001000AA
:101F3800D82E002030B50368594D1888594CB4FB89
:101F4800F2F20139013AAB4294B283B089B282B25B
:101F58000DD0554883420AD0B3F1804F07D0A0F581
:101F68009830834203D000F58060834202D122F08A
:101F7800700292B24D48834269D000F58060834276
:101F880041D022F4407200F58C3092B283421A801C
:101F9800D9621C8564D100221A8601225A611A88E6
:101FA8003F4942F001028B421A8069D0B3F1804F59
:101FB80068D03F4A934267D002F58062934265D069
:101FC80002F50062934263D002F58062934261D0C9
:101FD80002F5903293425FD002F5406293425DD0A1
:101FE80002F58062934217D002F58062934208BFDF
:101FF800092212D002A84FF0012340F8043D18F03E
:10200800FDFA03B030BD01201A80D9621C855861E1
:102018001A8802431A80C9E70822264B03EBC20339
:1020280001A85C7E8DF80440012300228DF805305C
:102038008DF807308DF8062018F0E0FA1B2CE0D157
:102048001D4B019301A818F0D9FA03B030BD012047
:102058001A80D9621C8558611A8802431A80A8E739
:10206800114A934297D002F54062934293D002F509
:10207800806293428FD002F5806293428BD08CE7C6
:102088000022CAE70122C8E70222C6E70322C4E702
:102098000422C2E70522C0E70622BEE70722BCE702
:1020A800002C014000A24A04003401400010004006
:1020B8000004004070360308190100011F4B9842C4
:1020C8002CD0B0F1804F2BD0A3F59433984229D06F
:1020D80003F58063984227D003F50063984225D022
:1020E80003F58063984223D003F59033984221D0BA
:1020F80003F5406398421FD003F58063984207D0E8
:1021080003F58063984208BF092202D00020704777
:1021180008220B4B03EBC203187E70470022F8E736
:102128000122F6E70222F4E70322F2E70422F0E7AD
:102138000522EEE70622ECE70722EAE7002C014039
:102148007036030870B4104E002332461D4603242F
:1021580003E00133112B0CD0947930EA040402F126
:102168001802F6D1A94207D001330135112BEDB27F
:10217800F2D1002070BC704703EB430306EBC303A6
:1021880070BC1879704700BF2063030810B50021A0
:1021980004460120FFF7D6FF207010BD10B40C4C88
:1021A80010212246002303E00133112B0BD01179B3
:1021B800884202F11802F7D103EB430304EBC30092
:1021C8005DF8044B704700205DF8044B704700BF72
:1021D800206303082DE9F04F013085B0C3B20393A3
:1021E800994C9A4FDFF874A2994D9A4E0A2302939C
:1021F80015F082F94FF4FA73DFF86CE201934FF0AF
:102208001008DAF80430C3F30803002B40F0D98033
:10221800EFF31183002B40F0D4802068AA6823686C
:102228009842FAD133689A42F7D8D7F800C04FF4E9
:102238007A7101FB0CF39B1AB3FBFCF301FB003032
:102248004FF47A7C4FF00109DAF80430C3F308033D
:10225800002B40F09880EFF31183002B40F093801F
:102268002368A96822689342FAD132689142F7D864
:102278003A680CFB02FBABEB0101B1FBF2F10CFB82
:1022880003131B1AB3F57A7FDED3019B013B01933D
:10229800B7D1039814F084FF4FF47A73DFF8C8E1DC
:1022A80001934FF01008DAF80430C3F30803002B49
:1022B80040F0A880EFF31183002B40F0A380206842
:1022C800AA6823689842FAD133689A42F7D8D7F8AF
:1022D80000C04FF47A7101FB0CF39B1AB3FBFCF3BB
:1022E80001FB00304FF47A7C4FF00109DAF8043032
:1022F800C3F308034BBBEFF3118333BB2368A9680F
:1023080022689342FAD132689142F7D83A680CFBB6
:1023180002FBABEB0101B1FBF2F10CFB03131B1A3F
:10232800B3F57A7FE2D3019B013B0193BBD1029BBA
:10233800013B02937FF45CAF4749484B4848494A00
:102348000860DA6005B0BDE8F08FEFF3118188F31B
:102358001288D5F808B02B68DB0344BFCEF800908C
:10236800D5F808B02368DEF80020C9B281F31188D7
:10237800396813440CFB01F2A2EB0B02B2FBF1F239
:102388000CFB0323CBE7EFF3118188F31288D5F810
:1023980008B02B68DB0344BFCEF80090D5F808B02E
:1023A8002368DEF80020C9B281F311883968134424
:1023B8000CFB01F2A2EB0B02B2FBF1F20CFB0323C4
:1023C8005FE7EFF3118388F31288D5F808C02A680D
:1023D800D20304D50122CEF80020D5F808C0206821
:1023E800DEF80090DBB283F3118839684FF47A7213
:1023F800484402FB01F3A3EB0C03B3FBF1F302FB2C
:1024080000301DE7EFF3118388F31288D5F808C070
:102418002A68D20304D50122CEF80020D5F808C0D6
:102428002068DEF80090DBB283F3118839684FF436
:102438007A72484402FB01F3A3EB0C03B3FBF1F3FC
:1024480002FB00304EE700BFC42D0020C82D00203D
:1024580010E000E0CC2D0020FC9F002000ED00E003
:10246800EFBEADDE0400FA05C02D00202DE9F04FC7
:1024780085B0CDE902109B4DDFF878A2029B013BA5
:102488000293013300F02A8115F036F8964C974FE5
:10249800DFF864E2964E4FF4FA7301934FF0100898
:1024A800DEF80430C3F30803002B40F0F680EFF3A6
:1024B8001183002B40F0F1802068AA6823689842B5
:1024C800FAD133689A42F7D8D7F800C04FF47A7136
:1024D80001FB0CF39B1AB3FBFCF301FB00304FF438
:1024E8007A7C4FF00109DEF80430C3F30803002BAF
:1024F80040F0B580EFF31183002B40F0B0802368E3
:10250800A96822689342FAD132689142F7D83A68AA
:102518000CFB02FBABEB0101B1FBF2F10CFB03136B
:102528001B1AB3F57A7FDED3019B013B0193B7D128
:10253800039B6F4E581CC0B214F032FEDFF8B8E1AE
:102548004FF47A730193DEF80430C3F308034FF0B5
:102558001008002B44D1EFF31183002B40D12068E1
:10256800AA6823689842FAD133689A42F7D8D7F80C
:1025780000C04FF47A7101FB0CF39B1AB3FBFCF318
:1025880001FB00304FF47A7C4FF00109DEF804308B
:10259800C3F30803002B44D1EFF31183002B40D180
:1025A8002368A96822689342FAD132689142F7D821
:1025B8003A680CFB02FBABEB0101B1FBF2F10CFB3F
:1025C80003131B1AB3F57A7FE0D3019B013B0193F8
:1025D8003FF454AFDEF80430C3F30803002BBAD03D
:1025E800EFF3118388F31288D5F808C02A68D2035C
:1025F80004D50122CAF80020D5F808C02068DAF806
:102608000090DBB283F3118839684FF47A7248443A
:1026180002FB01F3A3EB0C03B3FBF1F302FB003065
:10262800B0E7EFF3118188F31288D5F808B02B686A
:10263800DB0344BFCAF80090D5F808B02368DAF87D
:102648000020C9B281F31188396813440CFB01F2E8
:10265800A2EB0B02B2FBF1F20CFB0323B1E7EFF3A1
:10266800118188F31288D5F808B02B68DB0344BFC2
:10267800CAF80090D5F808B02368DAF80020C9B283
:1026880081F31188396813440CFB01F2A2EB0B02A9
:10269800B2FBF1F20CFB032342E7EFF3118388F35B
:1026A8001288D5F808C02A68D20304D50122CAF8CE
:1026B8000020D5F808C02068DAF80090DBB283F370
:1026C800118839684FF47A72484402FB01F3A3EB8E
:1026D8000C03B3FBF1F302FB003000E705B0BDE8E3
:1026E800F08F00BF10E000E0C42D0020C82D0020AE
:1026F800CC2D0020C02D002000ED00E0224B5B68AF
:10270800C3F3080330B4D3B9EFF31183BBB91F4A3D
:102718001F4D20481368846811688B42FAD12968D4
:102728008C42F7D81C4A11684FF47A7202FB01F008
:10273800001B30BCB0FBF1F002FB03007047EFF365
:102748001182102383F3128803F1E023D2B29C682C
:10275800196811F4803F11491EBF012008609C6868
:102768000A4B18680B6882F311880B4A11684FF4FA
:102778007A72034402FB01F0001B30BCB0FBF1F09D
:1027880002FB0300704700BF00ED00E0C42D0020ED
:10279800CC2D002010E000E0C82D0020C02D002026
:1027A8002DE9F84F8046274C274DDFF8A490274E97
:1027B800FFF7A4FFDFF89CE0DFF89CC04FF0100A99
:1027C8004FF47A77DCF80430C3F30803CBB9EFF39E
:1027D8001183B3B92368A96822689342FAD1326891
:1027E8009142F7D8DEF8002007FB02FBABEB0101B2
:1027F800B1FBF2F107FB03131B1A4345E2D3BDE813
:10280800F88FEFF311818AF31288D5F808B02B6896
:10281800DB0304D50123C9F80030D5F808B02368D4
:10282800D9F80020C9B281F31188DEF800101344EA
:1028380007FB01F2A2EB0B02B2FBF1F207FB032349
:10284800DAE700BFC42D002010E000E0CC2D002006
:10285800C02D0020C82D002000ED00E0F8B5304E56
:10286800304D32782B789A424FD12F4B93F800C0D5
:10287800BCF1000F48D02D4A2D4B1078002140F2B2
:102888000D3E11E05C681F896760276847F0010703
:102898002760A2F848E0D468013144F480748C457C
:1028A800D46003F59A730FDD1A680028EAD15062E4
:1028B800B3F83041D76801313C438C45D46003F507
:1028C8009A7323F8040CEFDC31782B7899421BD0EB
:1028D80003EB83029200174FB858BE18A0B9327A9A
:1028E80092B9727A82B9013303F00303D8B28142F4
:1028F800287009D003EB83039C003B191A72FFF779
:10290800FDFE736803443B51F8BD1BF0A1FE00288F
:10291800FAD0054B93F800C0BCF1000FABD1D3E758
:10292800E04B0020E14B0020F43F0020D03C002089
:10293800F83F0020E44B00202DE9F04FDFF834C1C8
:10294800494CDFF834E1DFF83481484E8246484884
:102958001AF1FF3AC0F08680DCF80430C3F30803AC
:10296800002B5ED1EFF31183002B5AD10568A268C2
:1029780003689D42FAD133689A42F7D8DEF80070AE
:102988004FF47A7101FB07F39B1AB3FBF7F301FBD2
:102998000535DCF80430C3F308034FF010094FF491
:1029A8007A77F3B9EFF31183DBB90368A16802689A
:1029B8009342FAD132689142F7D8DEF8002007FB3B
:1029C80002FBABEB0101B1FBF2F107FB03135B1B4D
:1029D800B3F57A7FBCD2DCF80430C3F30803002BCC
:1029E800E0D0EFF3118189F31288D4F808B0236896
:1029F800DB0304D50123C8F80030D4F808B0036815
:102A0800D8F80020C9B281F31188DEF80010134409
:102A180007FB01F2A2EB0B02B2FBF1F207FB032367
:102A2800D5E7EFF31183102282F31288A168226898
:102A3800D20303D50122C8F80020A168D0F800907D
:102A4800D8F80050DBB283F31188DEF800704FF439
:102A58007A724D4402FB07F35B1AB3FBF7F302FBF0
:102A6800053596E7BDE8F08F10E000E0CC2D00209A
:102A7800C42D002000ED00E0C82D0020C02D00204E
:102A880030B4EFF31183102282F312880848094901
:102A98000268094D094C013202608A682A600022E6
:102AA8002260DBB20A6883F3118830BC704700BF2C
:102AB800C42D002010E000E0CC2D0020C02D002007
:102AC8001D4B70B59C68636DA26BDD69CAB1E36B81
:102AD80033B12B0700D470BD636D08221A6270BD34
:102AE8002A06F6D5D4E909028242616D11D0501C3C
:102AF800A669A062B25C26690A85B042E9D3A362DE
:102B0800E7E7A906E3D5E26A42B1988C216B9047C2
:102B1800DDE70B6823F080030B60DAE7E1699B8C43
:102B28006069DBB24E1CE6614354E169E36899428F
:102B380028BFE261CBE700BF2C5800201D4B70B5C1
:102B48005C68636DA26BDD69CAB1E36B33B12B07B7
:102B580000D470BD636D08221A6270BD2A06F6D5CE
:102B6800D4E909028242616D11D0501CA669A062A5
:102B7800B25C26690A85B042E9D3A362E7E7A906F1
:102B8800E3D5E26A42B1988C216B9047DDE70B6888
:102B980023F080030B60DAE7E1699B8C6069DBB2A4
:102BA8004E1CE6614354E169E368994228BFE2613B
:102BB800CBE700BF2C5800201D4B70B51C68636D17
:102BC800A26BDD69CAB1E36B33B12B0700D470BDCA
:102BD800636D08221A6270BD2A06F6D5D4E9090287
:102BE8008242616D11D0501CA669A062B25C266950
:102BF8000A85B042E9D3A362E7E7A906E3D5E26A0A
:102C080042B1988C216B9047DDE70B6823F0800375
:102C18000B60DAE7E1699B8C6069DBB24E1CE66108
:102C28004354E169E368994228BFE261CBE700BFFA
:102C38002C580020002A12DD70B504460D468E1867
:102C4800236820469B6898470028F9D0236815F820
:102C5800011B1B6820469847B542F1D170BD7047EB
:102C68000368DB6A03B11847704700BF03689B6AB3
:102C780003B11847704700BF03682DE9F0415D6A4A
:102C88001DB12B46BDE8F0411847002A174611DD53
:102C980004460E460F4400E023689B682046984788
:102CA8000028F9D0236816F8011B1B6820469847AE
:102CB800BE42F1D1BDE8F08103685B69184700BFE7
:102CC8000368DB68184700BF03689B68184700BFA4
:102CD80003685B68184700BF03681B68184700BF94
:102CE800014B1868F8E700BF28120020054B53F87D
:102CF800203033B11A689B88918A0B4218BF1B0495
:102D080093617047902D002003682DE9F04F03F17F
:102D18003845A94EAD0A0124755D05F01F066D09F9
:102D2800022D04FA06F400F08D81032D00F0858150
:102D3800012D00F03B818088B0FA80F4C4F11F04B3
:102D4800A4B2E50803EB850504F007042E6AA40085
:102D58000F27A74026EA07062E622E6A01F003070E
:102D680002FA04F47A1E3443012AC1F3810EC1F336
:102D780000182C62C1F3411140F22281C60700F10C
:102D88000881850700F1F680440700F1E480020716
:102D980000F1D280C60600F1C080850600F1AE8041
:102DA800440600F19C80020600F18A80C60578D4AA
:102DB800850567D4440556D4020545D4C60434D4E1
:102DC800850423D4440412D4020401D4BDE8F08F4E
:102DD8001A6822F040421A601A6842EA87771F6030
:102DE800DA6822F0404242EA8171D960EEE71A6857
:102DF80022F040521A601A6842EA07721A60DA68CA
:102E080022F0405242EA0172DA60DDE71A6822F0E5
:102E180040621A601A6842EA87621A60DA6822F029
:102E2800406242EA8162DA60CCE71A6822F04072B6
:102E38001A601A6842EA07621A60DA6822F0407279
:102E480042EA0162DA60BBE71A6822F440021A60BB
:102E58001A6842EA87521A60DA6822F4400242EAA3
:102E68008152DA60AAE71A6822F440121A601A68D6
:102E780042EA07521A60DA6822F4401242EA015222
:102E8800DA6099E71A6822F440221A601A6842EA5E
:102E980087421A60DA6822F4402242EA8142DA6004
:102EA80088E71A6822F440321A601A6842EA074230
:102EB8001A60DA6822F4403242EA0142DA6077E7BF
:102EC8001A6822F440421A601A6842EA87321A6085
:102ED800DA6822F4404242EA8132DA6066E71A6828
:102EE80022F440521A601A6842EA07321A60DA6815
:102EF80022F4405242EA0132DA6054E71A6822F4B6
:102F080040621A601A6842EA87221A60DA6822F474
:102F1800406242EA8122DA6042E71A6822F440728B
:102F28001A601A6842EA07221A60DA6822F44072C4
:102F380042EA0122DA6030E71A6822F0C0021A6019
:102F48001A6842EA87121A60DA6822F0C00242EA76
:102F58008112DA601EE71A6822F030021A601A68D5
:102F680042EA07121A60DA6822F0300242EA0112D5
:102F7800DA600CE71A6822F00C021A601A6842EA52
:102F880087021A60DA6822F00C0242EA8102DA60EB
:102F9800FAE61A6822F003021A601A683A431A60BD
:102FA800DA6822F003020A43DA60EAE6034D6E6942
:102FB80034436C61BFE600BFD862030800100240CA
:102FC80000224FF0010C4FF003090CFA02F636EA22
:102FD80000042ED15400D3F808A009FA04F5ED43F3
:102FE80005EA0A0AC3F808A0D3F808B00EFA04FAEA
:102FF8004AEA0B0AC3F808A0B3F804A02AEA0606AE
:103008009E80B3F804A008FA02F646EA0A06B6B2A9
:103018009E801E682E401E60D3F800A007FA04F6B2
:1030280046EA0A061E60DE6801FA04F435402C43BD
:10303800DC600132102AC8D1C8E6054DEE69344378
:10304800EC6178E6024DAE693443AC6173E600BFCB
:1030580000100240036803F138422DE9F04F920A4C
:10306800A74DAA5C02F01F0552090124022A04FA9E
:1030780005F400F09F81032A00F09781012A00F0EF
:10308800518101F003077A1E012AC1F3810EC1F3B1
:1030980000188488C1F3411140F24981E60700F124
:1030A8003181A50700F11A81600700F10581220727
:1030B80000F1F080E60600F1DB80A50600F1C6808D
:1030C800600600F1B180220600F19C80E60500F15F
:1030D8008780A50572D460055FD422054CD4E60428
:1030E80039D4A50426D4600413D4220401D4BDE83D
:1030F800F08F1A6822F040421A601A6842EA87770D
:103108001F60DA6822F0404242EA8171D960BDE866
:10311800F08F1A6822F040521A601A6842EA077261
:103128001A60DA6822F0405242EA0172DA60220438
:10313800DDD5DEE71A6822F040621A601A6842EAB2
:1031480087621A60DA6822F0406242EA81626004AB
:10315800DA60CAD5DDE71A6822F040721A601A6888
:1031680042EA07621A60DA6822F0407242EA0162B3
:10317800A504DA60B7D5DDE71A6822F440021A60C0
:103188001A6842EA87521A60DA6822F4400242EA70
:103198008152E604DA60A4D5DDE71A6822F4401209
:1031A8001A601A6842EA07521A60DA6822F4401272
:1031B80042EA0152DA60220591D5DDE71A6822F465
:1031C80040221A601A6842EA87421A60DA6822F4D2
:1031D800402242EA81426005DA607FF57EAFDCE793
:1031E8001A6822F440321A601A6842EA07421A60E2
:1031F800DA6822F4403242EA0142A505DA607FF536
:103208006AAFDBE71A6822F440421A601A6842EA99
:1032180087321A60DA6822F4404242EA8132E605CF
:10322800DA607FF556AFDBE71A6822F440521A607D
:103238001A6842EA07321A60DA6822F4405242EA0F
:103248000132DA6022067FF541AFDBE71A6822F423
:1032580040621A601A6842EA87221A60DA6822F421
:10326800406242EA81226006DA607FF52CAFDBE734
:103278001A6822F440721A601A6842EA07221A6031
:10328800DA6822F4407242EA0122A506DA607FF584
:1032980017AFDBE71A6822F0C0021A601A6842EA20
:1032A80087121A60DA6822F0C00242EA8112E60642
:1032B800DA607FF502AFDBE71A6822F030021A60A5
:1032C8001A6842EA07121A60DA6822F0300242EA03
:1032D8000112DA6022077FF5EDAEDBE71A6822F00B
:1032E8000C021A601A6842EA87021A60DA6822F049
:1032F8000C0242EA81026007DA607FF5D8AEDBE7AC
:10330800D86203081A6822F003021A601A683A435E
:103318001A60DA6822F003020A43A507DA607FF52B
:10332800C3AEDBE7264A55692C435461A9E600225F
:103338004FF0010C4FF003090CFA02F636EA0400CC
:103348002ED15000D3F808A009FA00F5ED430AEA97
:10335800050AC3F808A0D3F808B00EFA00FA4AEA3A
:103368000B0AC3F808A0B3F804A02AEA06069E8050
:10337800B3F804A008FA02F646EA0A06B6B29E8036
:103388001E682E401E60D3F800A007FA00F646EA31
:103398000A061E60DE6801FA00F035402843D8604E
:1033A8000132102AC8D1BDE8F08F054AD5692C43EF
:1033B800D46166E6024A95692C43946161E600BFD0
:1033C8000010024010B50409013C052C17D80E4B1B
:1033D80033F8142000F00F0042FA00F313F0010351
:1033E8000FD0012303FA00F0013810402FF078FDC8
:1033F800064A074B125D104403EBC00010BD0020C5
:1034080010BD184610BD00BF0C63030818630308FD
:10341800C03000202DE9F04F4A484B4B4B4C4FF041
:1034280090414FF0010A4FF002094FF004084FF0A5
:10343800080E4FF0100C20274026802530F8022B6C
:1034480012F0010F03D01960A3F804A0083312F09A
:10345800020F03D01960A3F80490083312F0040F88
:1034680003D01960A3F80480083312F0080F03D0C2
:103478001960A3F804E0083312F0100F03D01960A4
:10348800A3F804C0083312F0200F02D019609F80FF
:10349800083312F0400F02D019609E80083312F0F2
:1034A800800F02D019609D80083312F4807F05D008
:1034B8004FF4807B1960A3F804B0083312F4007F3E
:1034C80005D04FF4007B1960A3F804B0083312F458
:1034D800806F05D04FF4806B1960A3F804B00833EF
:1034E80012F4006F05D04FF4006B1960A3F804B014
:1034F800083312F4805F05D04FF4805B1960A3F89D
:1035080004B0083312F4005F05D04FF4005B196073
:10351800A3F804B0083312F4804F05D04FF4804B61
:103528001960A3F804B00833D20B04D04FF400425A
:1035380019609A80083301F58061A1427FF47EAF5B
:10354800BDE8F08F0C630308C03000200018004865
:1035580000B9704703682DE9F04F03F138449C4ED9
:10356800A40A0125345D04F01F066409022C05FA3B
:1035780006F500F07481032C00F06C81012C00F03A
:1035880022818088B0FA80F4C4F11F04A4B2E5084F
:1035980003EB850504F007042E6AA4000F27A74053
:1035A80026EA07062E622E6A01F00307A2407C1E57
:1035B8003243012CC1F3810EC1F300182A62C1F312
:1035C800411140F20981C6070BD51A6822F003029F
:1035D8001A601A683A431A60DA6822F003020A434A
:1035E800DA6085070DD51A6822F00C021A601A688D
:1035F80042EA87021A60DA6822F00C0242EA810283
:10360800DA6044070DD51A6822F030021A601A6889
:1036180042EA07121A60DA6822F0300242EA01121E
:10362800DA6002070DD51A6822F0C0021A601A681B
:1036380042EA87121A60DA6822F0C00242EA81126E
:10364800DA60C6060DD51A6822F440721A601A6844
:1036580042EA07221A60DA6822F4407242EA01223A
:10366800DA6085060DD51A6822F440621A601A6875
:1036780042EA87221A60DA6822F4406242EA81222A
:10368800DA6044060DD51A6822F440521A601A68A6
:1036980042EA07321A60DA6822F4405242EA0132FA
:1036A800DA6002060DD51A6822F440421A601A68D8
:1036B80042EA87321A60DA6822F4404242EA8132EA
:1036C800DA60C6050DD51A6822F440321A601A6805
:1036D80042EA07421A60DA6822F4403242EA0142BA
:1036E800DA6085050DD51A6822F440221A601A6836
:1036F80042EA87421A60DA6822F4402242EA8142AA
:10370800DA6044050DD51A6822F440121A601A6866
:1037180042EA07521A60DA6822F4401242EA015279
:10372800DA6002050DD51A6822F440021A601A6898
:1037380042EA87521A60DA6822F4400242EA815269
:10374800DA60C6040DD51A6822F040721A601A6849
:1037580042EA07621A60DA6822F0407242EA0162BD
:10376800DA6085040DD51A6822F040621A601A687A
:1037780042EA87621A60DA6822F0406242EA8162AD
:10378800DA6044040DD51A6822F040521A601A68AB
:1037980042EA07721A60DA6822F0405242EA01727D
:1037A800DA6002040DD51A6822F040421A601A68DD
:1037B80042EA87771F60DA6822F0404242EA817164
:1037C800D960BDE8F08F034C666935436561D8E67A
:1037D800D86203080010024000224FF0010C4FF09D
:1037E80003090CFA02F636EA00042ED15400D3F885
:1037F80008A009FA04F5ED4305EA0A0AC3F808A087
:10380800D3F808B00EFA04FA4AEA0B0AC3F808A07B
:10381800B3F804A02AEA06069E80B3F804A008FAC2
:1038280002F646EA0A06B6B29E801E682E401E6060
:10383800D3F800A007FA04F646EA0A061E60DE6816
:1038480001FA04F435402C43DC600132102AC8D157
:10385800BDE8F08F044CE6693543E56191E6024C1A
:10386800A6693543A5618CE60010024000B970478F
:10387800036803F138422DE9F04F920AB24DAA5C71
:1038880002F01F0552090124022A04FA05F400F087
:103898005F81032A00F05381012A00F00D8101F0B5
:1038A80003077A1E012AC1F3810EC1F30018848828
:1038B800C1F3411140F20581E6070BD51A6822F0E1
:1038C80003021A601A683A431A60DA6822F003029F
:1038D8000A43DA60A5070DD51A6822F00C021A60AF
:1038E8001A6842EA87021A60DA6822F00C0242EA91
:1038F8008102DA6060070DD51A6822F030021A607A
:103908001A6842EA07121A60DA6822F0300242EABC
:103918000112DA6022070DD51A6822F0C0021A6077
:103928001A6842EA87121A60DA6822F0C00242EA8C
:103938008112DA60E6060DD51A6822F440721A6020
:103948001A6842EA07221A60DA6822F4407242EAE8
:103958000122DA60A5060DD51A6822F440621A60C1
:103968001A6842EA87221A60DA6822F4406242EA58
:103978008122DA6060060DD51A6822F440521A6076
:103988001A6842EA07321A60DA6822F4405242EAB8
:103998000132DA6022060DD51A6822F440421A6014
:1039A8001A6842EA87321A60DA6822F4404242EA28
:1039B8008132DA60E6050DD51A6822F440321A60C1
:1039C8001A6842EA07421A60DA6822F4403242EA88
:1039D8000142DA60A5050DD51A6822F440221A6062
:1039E8001A6842EA87421A60DA6822F4402242EAF8
:1039F8008142DA6060050DD51A6822F440121A6017
:103A08001A6842EA07521A60DA6822F4401242EA57
:103A18000152DA6022050DD51A6822F440021A60B4
:103A28001A6842EA87521A60DA6822F4400242EAC7
:103A38008152DA60E6040DD51A6822F040721A60E5
:103A48001A6842EA07621A60DA6822F0407242EAAB
:103A58000162DA60A5040DD51A6822F040621A6086
:103A68001A6842EA87621A60DA6822F0406242EA1B
:103A78008162DA6060040DD51A6822F040521A603B
:103A88001A6842EA07721A60DA6822F0405242EA7B
:103A98000172DA6022040DD51A6822F040421A60D9
:103AA8001A6842EA87771F60DA6822F0404242EAE1
:103AB8008171D960BDE8F08F244A55692C4354615F
:103AC800EDE600224FF0010C4FF003090CFA02F664
:103AD80036EA04002ED15000D3F808A009FA00F500
:103AE800ED430AEA050AC3F808A0D3F808B00EFAAD
:103AF80000FA4AEA0B0AC3F808A0B3F804A02AEAB5
:103B080006069E80B3F804A008FA02F646EA0A06FA
:103B1800B6B29E801E682E401E60D3F800A007FA39
:103B280000F646EA0A061E60DE6801FA00F0354033
:103B38002843D8600132102AC8D1BDE8F08F034A63
:103B4800D5692C43D461AAE6D86203080010024064
:103B5800024A95692C439461A1E600BF0010024017
:103B680010B1036882881A85704700BF10B10368D6
:103B780082889A61704700BF18B1838811B10268C2
:103B8800936170471B04FAE70E4B1B8801463BB94B
:103B98000D4B0E4A1B7810680BB981F00101EBE759
:103BA8000B4B5A691AB11A6810B9106058747047EB
:103BB80008480949008891FBF0F101201160587408
:103BC800704700BF9C2D00209E2D0020A02D0020B6
:103BD800A42D0020BC2D002020A1070010B40A4B02
:103BE8000A4A1C7801238340234052F8200029B94F
:103BF800B3FA83F149095DF8044BBDE7191C18BFF6
:103C080001215DF8044BB7E78C2D0020902D002092
:103C180030B102688388128A1A4214BF012000203A
:103C2800704700BF2DE9F0410B4E346873691C40A2
:103C38000FD0DFF828800127B4FA84F3C3F11F03FB
:103C480007FA03F558F8230003689847AC437561F1
:103C5800F2D1BDE8F08100BF00040140483C0020DB
:103C68002DE9F0410B4E346873691C400FD0DFF822
:103C780028800127B4FA84F3C3F11F0307FA03F578
:103C880058F8230003689847AC437561F2D1BDE842
:103C9800F08100BF00040140483C00202DE9F041BC
:103CA8000B4E346873691C400FD0DFF82880012759
:103CB800B4FA84F3C3F11F0307FA03F558F8230095
:103CC80003689847AC437561F2D1BDE8F08100BF45
:103CD80000040140483C00202DE9F0410B4E3468B7
:103CE80073691C400FD0DFF828800127B4FA84F3E9
:103CF800C3F11F0307FA03F558F823000368984730
:103D0800AC437561F2D1BDE8F08100BF0004014009
:103D1800483C00202DE9F0410B4E346873691C4083
:103D28000FD0DFF828800127B4FA84F3C3F11F030A
:103D380007FA03F558F8230003689847AC43756100
:103D4800F2D1BDE8F08100BF00040140483C0020EA
:103D58002DE9F0410B4E346873691C400FD0DFF831
:103D680028800127B4FA84F3C3F11F0307FA03F587
:103D780058F8230003689847AC437561F2D1BDE851
:103D8800F08100BF00040140483C00202DE9F041CB
:103D98000B4E346873691C400FD0DFF82880012768
:103DA800B4FA84F3C3F11F0307FA03F558F82300A4
:103DB80003689847AC437561F2D1BDE8F08100BF54
:103DC80000040140483C00200B490C4A0C4808B547
:103DD8008B6943F001038B61136843F480531360CC
:103DE800002140222FF0EDFB064B4FF0FF321A6006
:103DF800C3F8032008BD00BF0010024000000140C6
:103E0800483C0020883C002003685B6A184700BFD4
:103E180003681B6A184700BF70B44E1C0568C2725D
:103E28008672AC69A44670BC604700BF2DE9F041BA
:103E3800044618460D4616461F462EF045FD2844F2
:103E4800A0722068E672294645693B4632462046FC
:103E5800AC46BDE8F0416047036810B504461B68EE
:103E68009847236820469B689847E37B0133E373B0
:103E780010BD00BF10B5036804469B689847FF2330
:103E88000122A373627310BD70B5054600780E4613
:103E9800FFF798FA044618B1382301368371C671C2
:103EA80020466978FFF7E2FCAB78204613B1BDE8FD
:103EB80070405BE6BDE8704052E600BF064B984292
:103EC80002D04FF0FF307047044A538B01339BB246
:103ED8005383508B80B27047003800405C2D00201F
:103EE800F8B584894FF6FF764FF47A742BB311B383
:103EF8000F78013101E0B44217D00589013CAD07C4
:103F0800A4B2F8D507734FF47A7402E0BCB2B44295
:103F18000BD00589ED0704F1FF37F7D5057BEDB226
:103F28000AB115700132013BE0E7FFF7C7FF003027
:103F380018BF0120F8BDFF27DFE70120F8BD00BF4B
:103F480030B5437F83B004461BB90120637703B0C3
:103F580030BD0523ADF80430056800BFA868FFF739
:103F6800FFFD6A4601A902236868FFF7B9FFA86840
:103F7800FFF7FCFD00BF9DF8013003F0010383F05B
:103F88000100637703B030BDF8B5074C05460F460E
:103F9800266803E023689B1BBB4204D82846FFF72A
:103FA800CFFF0028F6D0F8BDC42D0020F0B5077F5C
:103FB80083B004464FF0030C0020009016461D46BF
:103FC8008DF804008DF800C06FB30B0E8DF801302A
:103FD8000DF10203080C0A0A997018700621204690
:103FE8005A70FFF7D1FFE0B1236800BF9868FFF768
:103FF800B7FD237F2268002B14BF052304236946DD
:1040080050680022FFF76CFF236832460021586889
:104018002B46FFF765FF23689868FFF7A7FD00BFE9
:10402800284603B0F0BD0DF10103D3E7F8B50378D6
:10403800012B49D0022B4DD1836801F07F0113B1C8
:104048001C689B88238504464068154640F2E9337E
:10405800828902E0002B00F0A0800289013B12F067
:10406800020F9BB2F6D0017340F2E93302E0002B55
:1040780000F093800289013B12F0010F9BB2F6D049
:10408800037B606840F2E933828902E0002B00F08C
:1040980081800189013B11F0020F9BB2F6D00573B4
:1040A80040F2E93301E0002B74D00289013B12F0A1
:1040B800010F9BB2F7D0037BA368002B68D01A6866
:1040C8009B8893610120F8BD90F904305C1C01D0F5
:1040D800022B01DD0020F8BD434C03EB830304EB06
:1040E80083035B68002B6DD04579404E6D004FF41B
:1040F8002040EDB270629C69270400F1FF303DD486
:104108005C683B4F45F080703C4040F49030204361
:104118004FF420445860746201E0671C54D09869D9
:1041280010F0020004F1FF34F7D04FF420409962F8
:104138007062014601E04F1C19D0986910F08000A8
:1041480001F1FF31F7D05968294845F00075014061
:1041580045F480350D434FF420415D6071629869E4
:1041680010F0020001F1FF311AD14C1CF7D1214A9D
:104178007162138801339BB21380F8BD441CBAD115
:104188001C4A7062138801339BB213800020F8BD6B
:104198000120F8BDFFF792FE8EE7FFF78FFE70E76C
:1041A8004FF420419A6271620A4602E012F1FF322E
:1041B80011D3996911F02001F8D020217262D961D8
:1041C8000120F8BD1846F8BD0A4A74621388013305
:1041D8009BB21380F8BD074C7262238801339BB2EF
:1041E80008462380F8BD00BF5C580020B80E0020A8
:1041F800009800FC240F00202DE9F04F87B090F8BC
:1042080061300290002B40F0F380029B724C734E99
:10421800DFF8D481724DDFF8D491724F103318460D
:1042280080226B210393FFF701FF64230193FEF7BC
:1042380065FA4FF0010A4FF0100E4FF47A7CD8F867
:104248000430C3F30803002B40F0A580EFF311837B
:10425800002B40F0A0802368A96822689342FAD115
:104268003A689142F7D832680CFB02FBABEB0101CC
:10427800B1FBF2F10CFB03131B1AB3F57A7FDED303
:10428800019B013B0193D2D1DDF80C90564F544D60
:10429800DFF8588103226B214846FFF7C7FE029BCF
:1042A800484693F86020DFF83C911921FFF7BEFEDD
:1042B8000F230193FEF722FA4FF0010A4FF0100E78
:1042C8004FF47A7C7B68C3F30803002B45D1EFF3E6
:1042D8001183002B41D12368A96822689342FAD13F
:1042E800D9F800209142F6D832680CFB02FBABEB00
:1042F8000101B1FBF2F10CFB03131B1AB3F57A7F32
:10430800E0D3019B013B0193D4D1029A92F85B3030
:10431800032B5ED892F85E20A2F10102B2FA82F273
:104328005209039C1A212046FFF780FE18221B2100
:104338002046FFF77BFE18221C212046FFF776FE59
:10434800022237212046FFF771FE2046012238213C
:10435800FFF76CFE07B0BDE8F08FEFF311818EF325
:104368001288D5F808B02B68DB0344BFC8F800A052
:10437800D5F808B02368D8F80020C9B281F31188AD
:10438800316813440CFB01F2A2EB0B02B2FBF1F211
:104398000CFB0323B1E7EFF311818EF31288D5F8F4
:1043A80008B02B68DA0344BFC9F800A0D5F808B0F4
:1043B8002368D9F80020C9B281F311883168134401
:1043C8000CFB01F2A2EB0B02B2FBF1F20CFB032394
:1043D80052E7019AA5E700BFC42D0020C82D002090
:1043E80010E000E0CC2D002000ED00E0C02D002002
:1043F8001D09013D052D03F00F0300F26981A94A4B
:1044080032F8150040FA03F2D40740F161814FF009
:10441800010909FA03F3013B18402EF061FDA24B94
:10442800A24A5B5D184412EBC00500F0518152F8B6
:104438003030AA88198A12EA01007FF4E6AEB2FA8F
:1044480082F1029CE871C1F11F0199482026AE71E2
:10445800E060481C3FF4D9AE03F13840800A954F1C
:10446800954E3F5CDFF85CC2765C07F01F087F0959
:1044780004F10C0E022F09FA08F44CF821E000F0C0
:104488003B81032F00F031814F4500F02681D7078B
:1044980009D51C6824F003041C601C681C60DC68D7
:1044A80024F00304DC60940709D51C6824F00C048C
:1044B8001C601C681C60DC6824F00C04DC60570776
:1044C80009D51C6824F030041C601C681C60DC687A
:1044D80024F03004DC60140709D51C6824F0C004FB
:1044E8001C601C681C60DC6824F0C004DC60D70613
:1044F80009D51C6824F440741C601C681C60DC68C6
:1045080024F44074DC60940609D51C6824F44064E3
:104518001C601C681C60DC6824F44064DC6057067E
:1045280009D51C6824F440541C601C681C60DC68B5
:1045380024F44054DC60140609D51C6824F4404473
:104548001C601C681C60DC6824F44044DC60D705EF
:1045580009D51C6824F440341C601C681C60DC68A5
:1045680024F44034DC60940509D51C6824F4402404
:104578001C601C681C60DC6824F44024DC6057055F
:1045880009D51C6824F440141C601C681C60DC6895
:1045980024F44014DC60140509D51C6824F4400494
:1045A8001C601C681C60DC6824F44004DC60D704D0
:1045B80009D51C6824F040741C601C681C60DC6809
:1045C80024F04074DC60940409D51C6824F040642D
:1045D8001C601C681C60DC6824F04064DC605704C4
:1045E80009D51C6824F040541C601C681C60DC68F9
:1045F80024F04054DC60140409D51A6822F04042C3
:104608001A601A681A60DA6822F04042DA60CAB2A0
:1046180002F0FC0303F1804303F5803302F0030248
:1046280094004FF00F0E9A68DFF89CC0234F0EFAE3
:1046380004FE22EA0E029A60C2B29868DFF88CE0A3
:10464800A2400124024304FA01F09A60CCF8000069
:104658003B68C24313403B60DEF800301340CEF89D
:1046680000303B6803433B605CF80C3C144F13403C
:104678004CF80C3CDEF808301A40CEF808205CF8FC
:104688000C3C03434CF80C3CBB5DF02B3CD8481C5D
:104698003FF4BBAD012303FA01F1084A136819433B
:1046A8001160B2E50C63030818630308C0300020EA
:1046B800E5090008D8620308C06503080004014042
:1046C800883C0020483C00201404014004040140B8
:1046D800029A194BD3600121DFE7DFF860C0DCF8EC
:1046E80014703C43CCF81440D1E6144FD7F81CC0E2
:1046F80044EA0C04FC61CAE6DFF840C0DCF8187034
:104708003C43CCF81840C2E60D4B8DF817409B5D32
:104718008DF81430F0230322BB5505A800238DF82B
:1047280015208DF8163015F069FFA988B1FA81F1C6
:10473800C1F11F01ABE700BFE50900080010024006
:10474800DC65030810B500F10C0401220B2120469A
:10475800FFF76CFC20B11D2209212046FFF766FCFB
:1047680000F0010010BD38B500F10C0504467022B8
:1047780000212846FFF75AFC202201212846FFF78E
:1047880055FC002202212846FFF750FC6420FEF762
:10479800D3F8607EC8B1FEF715FE0546FFF738FA74
:1047A80098B11DB12223AB710023EB712146084B50
:1047B80041F8083FF0220023284615F055FF284607
:1047C80013F018F9284613F015F9012038BD00BF79
:1047D8000B0A0008F0B500F10C0585B004460F4639
:1047E8000DF107020221284613F026F818B9002611
:1047F800304605B0F0BD9DF80730DB07F7D502AAB3
:104808000321284613F07EF80DF1070209212846F6
:1048180013F012F806460028E9D011220A2128468A
:10482800FFF704FC9DF8073013F00C0FDFD1B4F943
:104838001A1002A8FCF7E6F840423880B4F91C10B8
:104848000DF10A00FCF7DEF840427880B4F91E103A
:1048580003A8FCF7D7F84042B880C9E73122F42111
:10486800FFF7E4BB044B93F820209201343202F0A6
:10487800FC02F421FFF7DABBEC6C00202E22F421B5
:10488800FFF7D4BB01224821FFF7D0BB01225821F2
:10489800FFF7CCBB427A4AB110B5044604F10A01CD
:1048A800D0E9003098470023637210BD704700BFFD
:1048B800A8B10D4B012210B402FA01F103F17504FD
:1048C80002E00333A3420BD013F8012C8242F8D143
:1048D8001A780A42F5D001205DF8044B70477047FA
:1048E80000205DF8044B7047D536030830B40A4DF4
:1048F800002305F1640401E0272B0AD003EB4302EF
:104908000133A15C8142F7D12A4430BC92F8660099
:104918007047002030BC704770360308024B0146D0
:104928001868FBF703BD00BF1C11002038B5064D01
:10493800441E14F8011F286811B9BDE83840A9E7DA
:10494800FBF7F4FCF5E700BF1C11002010B5044686
:104958000B48FFF7EBFF0B4B1868FFF79BFF0A4B61
:10496800186807F08BFC23F043F9084B084A24B178
:10497800084909480860DA6010BDDA60FCE700BF42
:104988008C7403081C1100202011002000ED00E0A9
:104998000400FA05FC9F0020EFBEADDE38B5094DD6
:1049A8002868FFF777FF084B00241C70074B1C6032
:1049B800074B1C7023F0AAFA2046FFF7C7FF2C60AC
:1049C80038BD00BF1C110020281100202411002030
:1049D800711B00200120B9E70048A7E7FC7903080C
:1049E80038B5064D002455F834000134FFF79EFF12
:1049F800FFF7F2FF292CF6D138BD00BF7451030828
:104A080008B5FFF793FFBDE80840E5E7024A1368D9
:104A180023EA000010607047C03800206B4B1B6809
:104A2800B3F5FA7F10B500F2BC80694BDA885C896F
:104A38009889D989B2F57A6F84BF4FF47A62DA809F
:104A48001A89B2F57A6F84BF4FF47A621A81B4F585
:104A58007A6F84BF4FF47A645C81B0F57A6F88BF4F
:104A680000201A8A88BF9881B1F57A6F84BF4FF405
:104A78007A61D981B2F57A6F84BF00221A828442A2
:104A88009CBF00205881914298BF0022998B98BF03
:104A9800DA81DA8B914284BF00229A839A784D4951
:104AA800012A91F8581031D00A2934D00C2975D12F
:104AB8009FED497A494CA278062A97BF4849DFED0D
:104AC800496A01EB8201D1ED376A217961B3013A74
:104AD800032A6BD9444B45499A78022A04BF00221D
:104AE8009A704B78052B45D803EB4300404A03EBFB
:104AF800800302EB43030A783E48022A036041D947
:104B080000230B703C4B3D4A1A6010BD3C485A705C
:104B18000A29027040D19FED3B7A012ACAD10A299D
:104B280050D19FED397AC5E75B78354907EE903A61
:104B38000A78F8EEE77A67EE877A07EE102AB8EE79
:104B4800C77A27EE277AF4EEC76AF1EE10FAC1DDCC
:104B580086EEA77AFDEEC77A17EE903A102BA8BF1B
:104B68001023012BB8BF0123DBB29A4238BF1A4683
:104B78000A70AFE700224A700A781E481C4B03608F
:104B8800022ABDD81D4BC2EB0211C2EB810203EB16
:104B98004202194B1A6010BD0C2913D09FED1B7AE5
:104BA800BBE74FF00050FFF731FF3EE7B7EE000AD2
:104BB80080EE260A2EF086FC2388984228BF1846E5
:104BC800208087E79FED127A74E700BF203200202B
:104BD800F8310020303200200AD7A339503B00209A
:104BE800703603086F12033868170020E414002099
:104BF800B01600208C1E0020001500201015002083
:104C08007C6A00205304E9380F506E3A6F1203395A
:104C18006F12833A2DE9F041BF490B78A3F11702CF
:104C2800022A0FD9BD4A12F83300002840F09481B7
:104C3800D800024452782AB1B94A12F83330002B0E
:104C480000F0EE810024B74EB74F2546315B4B0884
:104C580003F077334FEA910C0CF0333CCB1ACA08B7
:104C6800A3EB0C0302F011329B1A03EB231303F09E
:104C78000F33A7FB03C2D209C2EB02229A1A11F022
:104C880001031CBF0135EDB2012A06EB040004F153
:104C980008040BDD022A40F03B8113B111F42F7F89
:104CA80004D110F0D5F9002800F03281282CCDD19C
:104CB800013D022D00F22C819C4F8020FFF7A6FEBB
:104CC80000263B4607F5B17E4FF47A6C4FF0640836
:104CD8005A88B2F57A6FB3F84C2088BFA3F802C09F
:104CE800B2F57A6F9A8888BFA3F84CC0B2F57A6F8C
:104CF800DA8888BFA3F804C09988B2F57A6F84BFB0
:104D08000022DE809142B3F86210B3F8642098BFA5
:104D18009E80914293F8732088BFA3F86260013A9D
:104D2800632A93F8742088BF83F873800132D2B263
:104D3800092A88BF83F8746003F16D0019460022C0
:104D48008C7A10F8015F0132A54228BF0670032A49
:104D580001F10601F4D176339E45B9D174498B78B7
:104D6800042B00F0028133B90B88B3F5F07F84BFC0
:104D78004FF4F0730B806F4CFFF750FE23686E4AB8
:104D88001A40002A00F02581DA0700F125815E0427
:104D980000F11A811D0700F1FB80980400F1F380EF
:104DA8001904664A14D50023D37382F82330137E7E
:104DB800C3B1537E032B00F01481012B21D0022BA9
:104DC80026D000233B83A7F88E30A7F8043118E1DA
:104DD800D17B002900F01B81002382F82330137E49
:104DE800002BE6D1BB817B82A7F88230A7F88830F8
:104DF800A7F8F830A7F8FE303B83A7F88E30A7F85D
:104E08000431002387F84F3087F8C53087F83B31E5
:104E18004B4BDA79022A08BF01224FF0070008BF7E
:104E2800DA7124F041FD002840F0B7804FF480602B
:104E380007F086FB002800F0BA80424E344604F1A1
:104E48007D057836617979B1207858B13E4B02E01A
:104E580006339D4208D013F8052C8A42F8D11A78F7
:104E6800002AF5D024F0CAFC0634A642EAD14FF451
:104E78000050FFF7CBFD4FF48040FFF7C7FD4FF41C
:104E88000030FFF7C3FD4FF40010FFF7BFFD2F4CB4
:104E98004FF00070FFF7BAFD4FF08060FFF7B6FDE6
:104EA800A388002B40F08880294A136813F07F4FAD
:104EB8001CBF00231360936823F4007323F00203DC
:104EC8000BB1002393601379013B042B84BF0123AA
:104ED8001371204BB3F86E2002F00F01022903D89A
:104EE800C2F30312012A03D94FF42062A3F86E20FB
:104EF800B3F8702002F00F01022903D8C2F303129D
:104F0800012A03D940F60122A3F87020BDE8F081F8
:104F1800044805F0A3F9CFE6706C0020B8640308D4
:104F28006C6F0308BC3B0020818080801015002036
:104F3800503B0020C038002009600002181F0020E4
:104F480008590020486E00204D6E0020445800206B
:104F58001061002088130020D80014186468002C01
:104F68007FF467AE17240C7063E64FF48050FFF7A8
:104F78004DFDCB8AB3F57A7F37BF4FF47A728B78C1
:104F88008B78CA82EFE62848FFF740FD236807E7D9
:104F98002648FFF73BFD2368FFE6072024F02EFC98
:104FA8004FF4806007F0CCFA00287FF446AF4FF04A
:104FB8000060FFF72BFD40E72078FDF7EFF80028A9
:104FC8007FF472AFA0806FE71948FFF71FFD2368D1
:104FD800E0E643F0010323601648FFF717FD236856
:104FE800D5E60023BB817B82A7F88230A7F88830FA
:104FF800A7F8F830A7F8FE303B83A7F88E30A7F85B
:105008000431537E023B022B3FF6FBAE00E742F22F
:1050180001010B423FF4CBAE002382F82330DEE6D9
:1050280018230B700EE600BF094000020160000261
:1050380009200002086000022DE9F84F2CF0F0FF6B
:105048002B4B2C4A934250D22B4F03F114069B460C
:105058004FF00108294C258862197DB1BA420DD25A
:10506800052D0BD936F8143C6188C3F30B0399421C
:105078000AD0144625886219002DEFD156F8101C65
:105088005846FBF7FBFF0FE0637913F0030AF0D1F2
:1050980056F8101C94F804905846FBF7EFFF36F8C2
:1050A800141CB9EB113F11D04FF00008114B0BF154
:1050B800140B9B4506F11406CCD3FFF7ABFDFCF7A8
:1050C800A9F92CF043FF4046BDE8F88F36F8123CAA
:1050D80056F8100CAA1FC3F30B039A4204F10601F9
:1050E800A8BF1A462EF049FAE0E74FF00108E4E7B6
:1050F80070B9030820BE03080000040802F0030882
:1051080008B508F0ABFAFFF797FF0120BDE80840A3
:1051180007F050BB2DE9F341056906460F467DBBF4
:10512800D0F80080C8F30A0323B30023D6F8008020
:10513800019313F035FB042819D1224C236943F05D
:1051480001032361BBB2A8F8003013F029FB04283F
:105158002ED108F102030193019B3F0C1F8013F02D
:105168001FFB2369042823F00103236125D06FF076
:10517800010505E013F014FB042805D04FF0FF35B6
:10518800284602B0BDE8F0810E4C236943F00203C3
:105198002361C4F81480236943F04003236113F0AA
:1051A800FFFA2369042823F002032361BDD0E5E751
:1051B800236923F001032361D9E73368043333609B
:1051C800DEE700BF00200240F8B504460D468E1801
:1051D8000027B54201D12069F8BDE368591CE16098
:1051E800234415F8012B1A720429F2D1A16820462C
:1051F800FFF790FFC4E90370EBE700BF30B4026823
:105208001146531C036011F8024B0160D31C5178FE
:1052180003609378151D05601B0443EA0123D078C9
:10522800234343EA006030BC704700BF0368591C41
:105238001A46016012F8021B0260587841EA002001
:10524800704700BF03685A1C02601878704700BF97
:1052580038B50446006815462EF08FF922682A44AE
:10526800226038BD036810B40A0A5C1C04601A7016
:1052780003685A1C026019705DF8044B704700BF40
:1052880003685A1C026010B4197003680A0A5C1C8F
:1052980004601A7003680A0C5C1C04601A700368C6
:1052A800090E5A1C026019705DF8044B704700BF64
:1052B80003685A1C026019700368090A5A1C0260C4
:1052C8001970704710EE103AC3F3160242F07E527E
:1052D80007EE102ADFED167ADFED164A9FED165A13
:1052E800DFED165A9FED166ADFED163ADFED166A06
:1052F8009FED164AE7EE274ADB1507EE903AA4EE33
:10530800875AF8EEE77AE5EE075A67EEA37AA5EE34
:10531800876AB5EEC00AE6EE077AF1EE10FAD4BF56
:10532800B0EE440AB0EE660A37EE800A704700BF56
:10533800DACDFE3CB9D593BE5CB8903FAA841DC0B7
:1053480022E061401872313F07F1B3C2000080FFCC
:10535800DFED1D3ADFED1D7A9FED1D7A9FED1D4AA9
:10536800DFED1D4A9FED1D5ADFED1D5A9FED1D6AA9
:10537800DFED1D6AE0EE237AF4EEC77AF1EE10FA5B
:1053880088BFF0EE477AF4EEC47AF1EE10FAB8BFAF
:10539800F0EE447AFDEEE77A17EE903AC3F3160280
:1053A80042F07E5207EE102AA7EE245A03F0FF437C
:1053B80000EE103AE5EE075AA5EE876AE6EE076AB0
:1053C80026EE800A704700BF3BAA384B00007E4E8D
:1053D8000000FF4E00000000ED185E3C81900FBBFE
:1053E800AF9D2A3EB2D19F3EE886023F07EE901A53
:1053F800F8EE677A9FED837A27EE800A20EE070A97
:10540800FDEEC07A17EE903A2033402B00F28180EF
:10541800DFED7D7AB4EEE70AF1EE10FA40F3E680AC
:10542800B0EE407A9FED796ADFED796A01E0B0EE7F
:10543800677AB4EEE67AF1EE10FA77EE467AF6DCA1
:105448009FED747AF4EEC77AF1EE10FA40F1D1804C
:105458009FED6E6ADFED706A01E0F0EE477AF4EED8
:10546800E67AF1EE10FA37EE867AF6D4DFED6B7A4B
:10547800B4EEE77AF1EE10FA40F3A780DFED627A36
:1054880037EEC77A27EE076ADFED655ADFED657AF2
:10549800DFED656A9FED655AE6EE257A67EE065AF6
:1054A800E6EE276AF7EE007AA5EEA67AF0EE675ADE
:1054B800E7EE055AE7EE457A87EEA55ADFED577A0B
:1054C80030EE277AFDEEC76A16EE903A2033402B6D
:1054D80024D99FED577AF6EE006AB7EE006AF7EE28
:1054E800004AC4EEA57A0023836143610362C36165
:1054F80080ED045A67EEA66A27EE866A27EE877A59
:10550800C0ED006AC0ED026A80ED016A80ED037AA1
:105518007047B7EE005AF0EE455ACFE7B4EEE70A07
:10552800F1EE10FA6BDD9FED396ADFED396A01E0C3
:10553800B0EE677AB4EEE67AF1EE10FA77EE467AD4
:10554800F6DC9FED347AF4EEC77AF1EE10FA53D513
:105558009FED2E6ADFED306A01E0F0EE477AF4EE57
:10556800E67AF1EE10FA37EE867AF6D4DFED2B7A8A
:10557800B4EEE77AF1EE10FA33DCDFED2E7AB4EE12
:10558800E77AF1EE10FA44BFDFED227A37EEC77AF8
:1055980027EE076ADFED224ADFED226ADFED227A85
:1055A800E6EE246A67EE064AE6EE267AB7EE006A69
:1055B800A4EEA77AF6EE006A36EE476AF8EE007AAD
:1055C80027EE277A66EE266A89E7DFED1A7AB4EEC7
:1055D800E77AF1EE10FA44BFDFED0E7A37EEC77ABC
:1055E80050E7DFED097A37EEC77AD1E7F0EE407A77
:1055F80026E7B0EE677A39E7B0EE677AB6E7F0EEFD
:10560800477A9EE727D4D236DB0F4940DB0FC940E3
:10561800E4CB1641DB0F49C0E4CB16C1DB0FC93F11
:1056280092E741B99730083C15A82ABEF304353FE4
:1056380000000000DB0FC9BFDFED2B7AB4EEE70AEC
:10564800F1EE10FA4ADDDFED296A9FED297A01E0D3
:10565800B0EE670AB4EEC70AF1EE10FA70EE667A99
:10566800F6DC9FED247AF4EEC77AF1EE10FA38D51D
:10567800DFED1E6A9FED207A01E0F0EE407AF4EE4D
:10568800C77AF1EE10FA37EEA60AF6D4DFED1B7AE8
:10569800B4EEE70AF1EE10FA14DDDFED137A37EE17
:1056A800C00A60EE006A9FED166A9FED167ADFED7C
:1056B800167AA6EE867A20EE266AE6EE877AA6EEB7
:1056C800270A7047DFED117AB4EEE70AF1EE10FA17
:1056D80044BFDFED087A37EEC00AE2E7F0EE407A21
:1056E800BFE7B0EE670AD1E7DB0F4940DB0FC940DF
:1056F800E4CB1641DB0F49C0E4CB16C1DB0FC93F31
:1057080092E741B99730083C15A82ABEDB0FC9BFFC
:1057180002B370B48E1803E0121B14D1B14215D035
:1057280010F8012BA2F14103192B11F8013BA3F149
:10573800410598BF2032192D03F12004ECD9D21A63
:1057480001D1002BEAD1104670BC704700221046E8
:1057580070BC70471046704770B5044608460D4641
:105768002DF0B2F8064602E014F8013F43B1324684
:1057780029462046FFF7CCFF0028F5D1204670BD0A
:105788001C46204670BD00BF4FF0FF32FFF7C0BF78
:10579800A0F16103192B98BF20387047A0F141038D
:1057A800192B98BF20307047202805D009380428C5
:1057B8008CBF0020012070470120704770B5044657
:1057C80008460E462DF080F831460546024620462A
:1057D800FFF79EFF68B9635D1846FFF7E5FF00B95C
:1057E80033B901352C44204601340378202BFAD0F4
:1057F80070BD0020FCE700BF613819288CBF00206D
:1058080001207047413819288CBF002001207047BB
:10581800303809288CBF002001207047A0F13003E0
:10582800092B07D920F02000413819288CBF002007
:105838000120704701207047F8B50646154608460E
:10584800B6FBF2F434B905FB14640C4B1B5D00F88D
:10585800013BF8BDB4FBF2F75FB905FB1747074BEF
:1058680005FB1464DA5D00F8012B1B5D00F8013BB1
:10587800F8BD3846FFF7E0FFEFE700BF447E0308B6
:10588800B5EEC00ADFED677A674AF1EE10FACCBFD1
:1058980030EE270A30EE670ADFED647A20EE270A39
:1058A8002DE9F047FDEEC07A88B017EE904A84EAF9
:1058B800E4760023A6EBE476CDE902330493A2FB59
:1058C80006325FEAD208054641D105AF5848394645
:1058D800554BA3FB0623DB0803EB8303A6EB43032B
:1058E800002CC35C0B704FF00002ACBF20232D23AB
:1058F8004A7038468DF808302CF0E6FF0128394602
:1059080039D0022842D0032805BF302302A802A8B4
:105918008DF809302DF05DFE02A82CF0D5FF033874
:10592800C4B2224602A928462DF089FE00232B5531
:1059380028462CF0C9FF2E22431C02A92A542144D0
:10594800E8182DF062FE284608B0BDE8F087394B0C
:10595800A3FB06235B0922D105AF35483946324AF5
:10596800A2FB0832D20802EB8202A8EB4202835C57
:1059780001F8013BACE7302302A88DF809308DF817
:105988000A308DF80B302DF024FEC5E7302302A82D
:105998008DF809308DF80A302DF01BFEBCE7264A39
:1059A800A2FB06125FEA92190ED105AF20483946CC
:1059B8001D4AA2FB03C2D20802EB8202A3EB4203F8
:1059C800C35C01F8013BCAE71C4AA2FB06125FEA66
:1059D800523A0ED105AF16483946134AA2FB09C2FE
:1059E800D20802EB8202A9EB4202825C01F8012B89
:1059F800DEE71348B6FBF0F058B905AF39460A2080
:105A0800BAFBF0F200FB12A20948825C01F8012BF4
:105A1800E3E705AF39460A220193FFF70DFF019B23
:105A28000146ECE76F12033ACDCCCCCC00007A44A7
:105A3800447E03081F85EB51D34D62105917B7D127
:105A4800A086010070B406688E4217D90139751E08
:105A5800002311F8014F0822634013F0800F4FEA2A
:105A6800430318BF83F0D503013ADBB2F5D18D4269
:105A7800EFD1721C0260337070BC7047721C002337
:105A88000260337070BC70470A44914215D010B45C
:105A98000139541E11F8012F0823504010F0800FCF
:105AA8004FEA400018BF80F0D500013BC0B2F5D1E5
:105AB800A142EFD15DF8044B704770474840082376
:105AC80010F0800F4FEA400018BF80F0D500013B6E
:105AD800C0B2F5D1704700BF0A44914215D030B426
:105AE8000139551E41F2210211F8014F082380EABD
:105AF800042004044CBF82EA40004000013B80B20D
:105B0800F7D18D42F0D130BC7047704770B5022292
:105B18001349144C144E4FF6FF70FFF7DDFF22882F
:105B28004AB1A518B54218D2052A16D92146FFF759
:105B3800D3FF2C46F3E721460222FFF7CDFF0222CE
:105B4800A118FFF7C9FF094BE41A094B1C8541F658
:105B58000F53C31A5842584170BD0020FCE700BFDC
:105B680000F0030802F0030800000408FAEF030835
:105B7800B80E00202DE9F043002489B006460D46F2
:105B88001F46A04605E025290CD030460134A84719
:105B9800039A531C039311780029F4D1204609B0C5
:105BA800BDE8F083931CCDE903385078302842D003
:105BB800A0F13003DBB2092B4FF0000945D96C285E
:105BC8002AD0642873D019D9732858D063D9752876
:105BD80040F0828007F1040C386805AB00220A21E6
:105BE8006746FAF7B9FD05AB049A009329464B4678
:105BF8003046FAF703FE039A0444CAE725283CD046
:105C080051D958286BD06328C2D139783046A84773
:105C180004370134039ABCE7039B5A1C03921B7890
:105C2800642B52D016D8252B27D064D9582B18D0DE
:105C3800632BEAD0ADE7D31C03939078A0F130032F
:105C4800DBB2092B4FF00109B9D804AA03A912F055
:105C5800BDFDB4E7732B12D051D9752B2DD0782BFD
:105C680097D1A3F15802B2FA82F23868520905AB0B
:105C780010210437FAF770FDB5E7252185E73B6861
:105C8800049A0093294600233046FAF7B7FD0437F3
:105C98000444039A7DE76E287FF47AAF039A3B6841
:105CA80004371C6075E700283FF478AF70E7386860
:105CB80005A9FAF71BFD043795E7386805AB0022FC
:105CC8000A21FAF749FD04378DE73B1D386805A915
:105CD8001F46FAF70BFD86E778287FF459AFA0F145
:105CE8005802B2FA82F23868520905AB1021FAF765
:105CF80033FD043777E7002B3FF450AF49E76E2BAD
:105D0800CDD046E710B5064C0B460246054920683B
:105D1800FFF730FF2068BDE81040FEF7BBBD00BFAD
:105D28001C110020A704000838B504460D46084891
:105D3800FEF7FCFD29462046FFF7E4FF0548FEF77D
:105D4800F5FD054B1B7813B1044B01221A7038BDC1
:105D580098740308A37403087812002079120020AD
:105D68000FB407B504A951F8040B0191FFF7DCFF44
:105D7800FEF732FE03B05DF804EB04B0704738B5A7
:105D88000F4D2B7863B10F4C23784BB10E48FFF7BA
:105D9800E7FF0E48FFF7E4FF00232B70237038BDA0
:105DA8000B4B93F82A203AB1D86AFBF72DFB002059
:105DB800BDE83840FEF7CABD07F050FCF7E700BF62
:105DC8007812002079120020A7740308DE740308F3
:105DD800B80E002038B5052215490446FFF798FC8F
:105DE80058B9144A13781BB901211170124A13705B
:105DF8001248BDE83840FEF703BE0322104920468A
:105E0800FFF786FC80B90B4C0B4D227842B12B78FA
:105E180033B10C48FFF7A4FF002323702B7038BD63
:105E28000948FEF7EDFDF7E70848BDE8384097E771
:105E3800257D03087812002079120020FC740308DD
:105E48008B7D0308A77403081275030826750308D9
:105E5800004885E7357503080FB407B504A951F85C
:105E6800040B0191FFF760FF03B05DF804EB04B089
:105E780070470FB407B504A951F8040B0191FFF757
:105E880041FFFEF7A9FD03B05DF804EB04B07047CD
:105E980010B5104C03461846FAF768FA58B10E4B7D
:105EA8000E4893F901104B1C0ABF0D4BC9B2597823
:105EB800BDE81040DDE71846FBF702FA052804D8CC
:105EC800C0B218F0DFFE2346E5E705210548BDE826
:105ED800104045E7FE7903080000002041750308DB
:105EE800E41400205075030810B5104C03461846FA
:105EF800FAF73CFA58B10E4B0E4893F900104B1CB8
:105F08000ABF0D4BC9B21978BDE81040B1E7184671
:105F1800FBF7D6F9022804D8C0B207F0EDFE2346F5
:105F2800E5E702210548BDE8104019E7FE790308B6
:105F38000000002045750308E41400205575030887
:105F480038B50D46FBF7BCF90C4B19788842044666
:105F580005D201460A48FFF78CFF204638BD2DB10F
:105F6800FF2803D10748FFF784FFF6E70139064801
:105F7800FFF7F6FE4FF0FF34EFE700BF7D12002079
:105F88007075030881750308947503082DE9F341BA
:105F98000346FAF7EBF9044620B1FFF759FF02B0C0
:105FA800BDE8F08101AA2B49DFF8A88018462DF03A
:105FB8003FFA2746054626467DB9022CEDD1A7F5BE
:105FC8007A73B3F57A7F20D94FF4FA634FF47A7273
:105FD80021492248FFF7C4FEE1E74CB1012C0FD05C
:105FE80001AA414600202DF023FA01340546E3E7D3
:105FF80001212846FFF7A4FF431C0646F0D1CEE74F
:106008002846FBF75DF90746EAE7B8B221F07CFDC0
:10601800FF2EBCEEC00A124B0BD1124AF8EE407AA2
:106028001278AA4212DC10EE101A0F48FFF721FF6F
:10603800B5E7F8EE407A03EB860310EE102A3146F6
:106048000A48C3ED007AFFF714FFA8E7E3EC017AEA
:106058000135E6E7457C0308C57D0308BA750308E2
:10606800645F00207D120020E0750308D3750308E3
:106078002DE9F3470346FAF779F9044610B1FFF71B
:10608800E7FE25E001AA2A49DFF8B480DFF8B490DA
:10609800DFF8B4A018462DF0CBF92646054627466A
:1060A80055B9244B3246A1B2186814F03DF878B9B6
:1060B8002148FFF755FE0BE06FB1012FDFD1B31E6A
:1060C800594259412846FFF73BFF421C044622D15A
:1060D80002B0BDE8F08728462CF0F6FB414606469C
:1060E80002462846FFF714FBA0B132464946284627
:1060F800FFF70EFBB8B1324651462846FFF708FBBA
:1061080098B132460D492846FFF702FB0028B6D160
:10611800032600E03E4601AA054900202DF088F933
:1061280001370546BCE70126F5E70226F3E700BF7D
:10613800457C030820110020FB750308F875030847
:10614800EF750308F2750308F57503082DE9F347A1
:106158000346FAF70BF9044618B92B4A9278042A31
:1061680004D8FFF775FE02B0BDE8F08701AA2749F9
:10617800DFF8AC80DFF8AC90DFF8ACA018462DF063
:1061880057F90127264640B9214B224A1B689B1A1A
:10619800214A18BF01231370E5E766B90121FFF70B
:1061A800CFFE431C0446DED001AA18490020013660
:1061B8002DF03EF9E7E7FBF783F82F2805461ED8B0
:1061C800D7B118F09DFA062D06D10520FCF7B4FBCF
:1061D8005046FEF715FC09E00120FCF7ADFB0F491E
:1061E8000123EAB20978E0B217F0A4FC2946484630
:1061F800FFF73FFE0027D7E70628F0D1E8E72F2171
:106208004046FFF7ADFDCFE7503B0020457C030833
:10621800C43C0020C1CE0108984900207D1200200E
:1062280039760308287603081976030807B5752117
:106238000DF10702144811F0FFFAF8B19DF80710A4
:106248001248FFF716FE0DF107021A210E4811F049
:10625800F3FAA8B19DF807100D48FFF70AFE0DF1F3
:1062680007021B21084811F0E7FA58B19DF80710FA
:106278000848FFF7FEFD03B05DF804FB0146DFE7C1
:106288000146E9E70146F3E7403200205976030862
:106298006C7603087F7603082DE9FF4107462CF04A
:1062A80013FB08283CD1002201AEB85CFFF770FA56
:1062B800B0540132082AF8D10024DFF870808DF834
:1062C8000C40385DFFF764FAC5B2305529464046A0
:1062D8002DF08EF928B10134294630192DF088F9AE
:1062E80020B1FFF7B5FD04B0BDE8F081082CE8D176
:1062F8000D4930462BF00AFE0B4C0C4800231A5D62
:1063080004A90A44195C02F80C1C0133082BF6D1C5
:10631800002301A906488DF80C30FFF7AAFDE2E733
:106328000028E9D0DDE700BF181F002068740308C3
:1063380092760308034B044A04491B6812680968EB
:10634800034896E5B4F7FF1FB0F7FF1FACF7FF1F30
:1063580099760308F7B50646FAF708F8054658B1DE
:10636800002401A9204613F0D5FD0134FFF7F2FF00
:10637800122CF6D103B0F0BD3046FAF7A1FFC4B233
:10638800112C61D8701CFAF78DFF334D0746D0B930
:10639800324B13F814108A1E514251412F4B13F8F7
:1063A8001420154495F8F820002948D003EB44033D
:1063B80019205B7840F2EE2100FB031321462848A0
:1063C800FFF757FDD6E705F1F806017830462DF0BE
:1063D8000FF958B1032C8CBF03230023801B2B44D7
:1063E80053FA80F090F8FC60032E02D1FFF730FDDD
:1063F800C0E73846FAF756FFF0B1022EF6D1FAF7A1
:106408005FFF40F6CA0280B29042144BA8BF104604
:1064180040F2EE22904203EB4403B8BF1046A0F2CC
:10642800EE20192290FBF2F05870B31E59425941E0
:106438000A4B03F81460B1E7022EF6D1D6E72146DD
:106448000848FFF716FD95E711232A46064907482D
:10645800FFF786FC8EE700BF70360308746F0020D4
:10646800AD760308BD760308CA760308BA75030833
:106478000FB407B504A951F8040B0191FFF742FCCA
:1064880003B05DF804EB04B070472DE9F843044607
:106498002CF01AFA024680B320461949FFF738F95A
:1064A800044650BBFEF798FA1648174D174E184F7A
:1064B800DFF86480FEF7A4FA2B7D072194FBF1F145
:1064C800C1EBC10206EB8303A21A0132013138463F
:1064D800D3F80491FFF7CCFF6A7D49464AB10D48CD
:1064E800FFF7C7FC01340C2C05F11C05E4D1BDE80D
:1064F800F8834046FFF7BDFCF4E7BDE8F843A7E49E
:10650800D2760308D7760308040000207036030803
:10651800DC760308EE7603086779030838B50B4B79
:1065280003EBC0040D4694F8F821094803EB8203F5
:10653800D3F80411FFF79CFF94F8FE3123B1691CCE
:106548000448BDE8384093E738BD00BF70360308FB
:1065580068790308CA7A03087FB50B4B04930B4B81
:1065680003930B4B02930B4B01930B4B00930B4A7A
:106578000B4B0C490C48FFF77BFF0C48062107B072
:106588005DF804EB75E400BF367703083B77030832
:10659800457703084E7703085A770308F57603080A
:1065A800EB140020007703080B77030860770308D3
:1065B8002DE9F04F93B00025DFF8A4B1DFF8C0A1B2
:1065C800DFF8C0910795A84608A9E8B218F0E4FCDE
:1065D8009DF82830002B6DD0022D40F09A809DED5B
:1065E800117AB5EE407AF1EE10FA00F08980DFED0D
:1065F800586AC6EE877AFDEEE77AF8EEE77AFDEE9E
:10660800E77A17EE906A99F80040089B012C79D92F
:1066180096FBF4F41A4602214E48FFF729FF0D9A1B
:10662800002A00F08B8041F2883002FB04004FF40E
:106638007A73B0FBF3F00F9B002B00F0818041F2DE
:10664800883103FB04114FF47A7CB1FBFCF1062D71
:1066580003D0079F0F44804407979BF803C0BCF101
:10666800000F6FD04FF47A7C0E9FB7FBFCFCCDF87F
:1066780010C04FF00A0C91FBFCFE0CFB1E11CDE97B
:1066880002E190FBFCF10CFB1100CDE90010214662
:106698003148FFF7EEFB022D08D199F80030012BA5
:1066A80004D9324609992D48FFF7E3FB0AEB851315
:1066B80000229A630135182D86D1294BDB78E3B186
:1066C800284B29481968294B1A684FF47A73B1FB8B
:1066D800F3F3274952090968FFF7CBFB0798079B93
:1066E8000A2293FBF2F302FB130798FBF2F10097DF
:1066F80002FB11821F48FFF7BCFB13B0BDE8F08F07
:10670800002680E7099A1C480221FFF7B1FE3446AB
:1067180085E7109C5CB107EE904ADFED0D6AF8EE54
:10672800677A86EEA77AFDEEC77A17EE904A089A3E
:1067380008482946FFF79CFE002670E710467AE7CE
:10674800194684E721460D48FFF793FBA3E700BFEE
:1067580000247449787703089A770308BE770308FA
:10676800E4140020D4510020CE770308CC51002037
:10677800D8510020EE77030887770308CA77030803
:10678800B40800207C6A0020F0B5482285B045494D
:106798004548FFF76DFEFEF71FF9444A444945484E
:1067A800FFF766FEFEF718F9434B444A4448D21AED
:1067B800444B198DFFF75DFB434B444819684FF470
:1067C8007A73B1FBF3F1FFF753FEFEF705F9404981
:1067D800D1F89C20002A55D007EE902ADFED3D6ABB
:1067E800B8EEE77AC6EE877AFDEEE77ACDED037A62
:1067F800394B1B885BB107EE903ADFED366AF8EE4D
:10680800677A86EEA77AFDEEC77A17EE903AC969DD
:1068180059B107EE901ADFED2F6AF8EEE77A86EEA7
:10682800A77AFDEEC77A17EE901A2C482C4E0088EE
:106838002C4F6428CDE900310146039B2A48A8BFA4
:106848006421FFF716FB294B29491A78294B098837
:10685800294803EB8203294AD3F8D0321278FFF78C
:1068680008FB274B27481988FFF703FB2648FEF744
:106878005DF8264B1C68012534B905B0BDE8F04029
:10688800FEF7AAB80392B3E794FAA4F3B3FA83F332
:1068980005FA03F256F82310384624EA0204FFF7F3
:1068A800E7FDE9E71C7803082178030800200010B9
:1068B800000800003478030800F00308000004080A
:1068C80058780308B80E0020C42D002082780308E9
:1068D800B4080020002474490A5200209A6300205A
:1068E80050540308677903089C780308131800209C
:1068F8000818002070360308E27803080E180020F4
:10690800240F00200979030818790308A81B002020
:106918002DE9F047214FDFF8A480DFF88490DFF8F5
:10692800A0A0054628462BF0CFFF064658B91C4BB9
:106938001C481A781C4B03EB8203BDE8F047D3F8D8
:10694800E012FFF796BA024639462846FEF7E0FEFF
:1069580078B91648164C174DFDF7E8FF54F8041F90
:1069680019B12846FFF784FDF8E7BDE8F047FEF7C0
:1069780033B8002458F8241021B90F48BDE8F0476F
:10698800FFF7EEB932462846FEF7C2FE013400286A
:10699800F0D189F800405546C4E700BF38790308AC
:1069A800706C00202E790308703603083D790308BF
:1069B80050390308677903084879030854390308EC
:1069C800FE7903082DE9F84F80460E4617462BF04E
:1069D8007BFF0446F0B94048404FDFF82081FFF7BD
:1069E80047FD0C25204605F0C7FD3368184205D041
:1069F80005FB047340469968FFF73AFD0134182CEB
:106A0800F0D1336813B93648FDF790FFBDE8F84F69
:106A1800FDF7E2BF024633494046FEF779FE0546D8
:106A2800B0B931482D4EDFF8C880FDF77FFF2C46FE
:106A38000C25204605F0A0FD384205D005FB04636F
:106A480040469968FFF714FD0134192CF1D1DDE7B0
:106A580098F800302D2B03BF08F1010804F1FF342A
:106A6800012500254FF0000A47F0807B1B4B0C22C4
:106A780002FB0A324046D2F8089022464946FEF701
:106A880047FEF8B9504605F077FD1BEA000F19D00C
:106A980075B1BAF1180F1CBF376807433760134840
:106AA800FDF744FF49461248BDE8F84FFFF7E1B942
:106AB800BAF1180F1CBF3568854335600D48FDF7DE
:106AC80035FFEFE70AF1010ABAF1190FCED10A48EA
:106AD800BDE8F84FFFF744B9557903084470030837
:106AE8005F790308387903083D7903086B7903084F
:106AF80067790308747903084879030866790308F5
:106B08006FF07F4200495DE71061002040F20222E9
:106B1800004957E7186100202DE9F047414D064626
:106B28002BF0D2FE404B95F82A801F680446B8F136
:106B3800000F15D0D5F82C90C4B93C483C4D3D4FBA
:106B4800FDF7F4FE012655F8241059B106FA04F3AE
:106B580013EA090F02D03846FFF78AFC0134F2E73E
:106B6800B946E9E7BDE8F047FDF736BF22463249A6
:106B78003046FEF7CDFD78B93048314C314DFDF740
:106B8800D5FE54F8041F0029ECD00B78002BF8D060
:106B98002846FFF76DFCF4E7B8F1000F03D1012395
:106BA800EF6285F82A303378DFF884A02D2B03BFF5
:106BB800013604F1FF344FF001094FF000094FF09E
:106BC80000085AF8287027B91F48BDE8F047FFF7B2
:106BD800C7B8224639463046FEF79AFDF8B9012370
:106BE80003FA08F2130604D51848BDE8F047FDF784
:106BF80007BFEB6AB9F1000F0BD023EA0203144870
:106C0800EB62FDF793FE39460E48BDE8F047FFF703
:106C180030B913430F48EB62FDF788FEF3E708F13C
:106C28000108CEE7B80E0020C03800207C790308A0
:106C3800C039030886790308387903083D790308C1
:106C4800BC39030867790308487903088A79030877
:106C58006B790308747903082DE9F04F87B0034670
:106C6800F9F784FB074620B1FFF7F2F807B0BDE853
:106C7800F08F05AA7F49DFF840A2DFF840B2184636
:106C88002CF0D6FBB84681463D463E464FF0FF34D1
:106C9800B9F1000F28D178482146FFF7E9FB774A78
:106CA80060B24B4602EBC30191F90610814200F035
:106CB800BD800133052BF5D1002E14BFB0464FF42B
:106CC8006148002D08BF03250023EDB20293CDE9EA
:106CD80000851A46194605F0F1FA0446002838D10D
:106CE8006748FDF78DFEC1E7B8F1030F07D8DFE865
:106CF80008F0020F14244846FAF7E2FA044605AAF7
:106D08005C4900202CF094FB08F101088146BFE79C
:106D18004846FAF7D5FA0646F1E751464846FEF7DF
:106D28001BFD08B145F0010559464846FEF714FD1C
:106D38000028E4D045F00205E1E748462BF0C4FD01
:106D4800504902464846FEF7E3FC002808BF0127E1
:106D5800D5E7414676B94C48FFF78AFB4B48FDF723
:106D68004FFE4B4B186803681B6A33B122464949EA
:106D7800984702E04848FFF77BFB484B4849494899
:106D8800434D002F18BF1946FFF773F837B128682D
:106D98000368DB6913B10022434998472D682846E8
:106DA80005F06CFA204605F069FA00210846FCF760
:106DB80015FF00210120FCF711FF2846FBF788FF8B
:106DC800A0B101210020FCF709FF2846FBF778FF56
:106DD80006462046FBF778FF0028FAD031462046C1
:106DE800FBF77AFF00210846FCF7F8FE2046FBF780
:106DF8006FFF0028E1D001210020FCF7EFFE2046BC
:106E0800FBF75EFF06462846FBF75EFF0028FAD030
:106E180031462846FBF760FF00210846FCF7DEFEF6
:106E2800CBE7A1682148FFF723FB0EE052F8334077
:106E3800002C3FF441AF002EF3D031461C48FFF739
:106E480017FB31462046F9F765FA5DB12179A94269
:106E580008D018482A46FFF70BFB2368E9B29B695C
:106E680020469847E36A0BB10023E362002E84D1E1
:106E780074E700BF457C0308AF790308E83B0020AE
:106E8800B8790308A9790308CD7903085B7A030860
:106E9800201100201D030008EA79030896790308E9
:106EA800FE7903087E7A03085F030008227A030844
:106EB800FF7903083D7A0308A3790308A679030834
:106EC8002DE9F041037903F06002202A2CD002D882
:106ED80052B1BDE8F081402A4AD0602AF9D127484A
:106EE800BDE8F041FEF7C5BF03F00703022B02D04F
:106EF800042B09D07BB9B0F80720B0F8051020485A
:106F0800BDE8F041FEF7B5BFD0F805101D48BDE853
:106F1800F041FEF7AEBFB0F90720B0F905101848E8
:106F2800BDE8F041FEF7A5BF4679174D174805EBB8
:106F3800C605FDF7FBFC95F8D07300240123A74292
:106F480003D8BDE8F041FDF747BDD5F8CC6356F846
:106F580024204FEA84084AB113B90D48FDF7E6FC2E
:106F680056F808100B48FFF783FA00230134E6E7C8
:106F780041790948BDE8F041FEF77BBFF37A030881
:106F8800B77A0308A17A030870360308CE7A030893
:106F9800DF7A030868790308E27A03082DE9F041EB
:106FA8001746027902F06003402B05460C462BD1A8
:106FB8000026554FDFF8708115E02B7903F00703A1
:106FC800022B15D0032B19D0012B14BFA15DA1579B
:106FD8003846FFF74DFA6B79013BB34202DD404674
:106FE800FDF7A4FC01366B79B342E6DCBDE8F0811D
:106FF80034F816103846FFF73BFAECE734F9161068
:107008003846FFF735FAE6E702F00702042A6DD89A
:10701800DFE802F0031F282A2D002478202B3ED019
:10702800602B4CD0002BE1D1B5F80560B5F807808E
:1070380035482146FFF71CFAA6424EDCA0454CDB3A
:10704800002FD3D0424631463048BDE8F041FFF723
:107058000FBA94F90040202B21D0602B2FD0002BA1
:10706800C4D14BE02488D9E7B4F90040F3E7266897
:10707800202B344613D0602B21D0002BB6D13146BB
:107088002348FFF7F5F9D5F805108E4225D8002FCB
:10709800ACD02048BDE8F041FFF7EAB900246A798E
:1070A8001D4B03EBC20393F8D023A24215DDD3F89E
:1070B800CC3353F82400BDE8F041FDF737BC6A79BA
:1070C8001441E30704D51548BDE8F041FFF7D0B9EE
:1070D8001348BDE8F041FFF7CBB9FDF77DFC224628
:1070E80029681048BDE8F041FEF7B6BE202BD5D080
:1070F800602BEDD0002B7FF479AF1C46B5F9056005
:10710800B5F9078094E700BFCB7A03081E7C030813
:10711800B47A03080B7B030870360308087B03085E
:10712800117B0308157B03082D7E030838B50D462F
:107138000446F9F7E5FB2A4601462046BDE83840F3
:107148002CE72DE9F74FDFF8C4B081468A460025C1
:10715800D8462B4B0D2418686C43FDF79BFB04EBBA
:107168000B031B7903F018034B4504D0B9F1000F4A
:107178003ED1182B3CD10D2303FB05820093B2F8B6
:107188000900F9F7A7FB444407462046F9F7F6F843
:10719800D7E901210646024401442046F9F726F9B9
:1071A8001AF0100F0246009B00D008BB03FB0583B2
:1071B8001AF0200F1B680FD072B9194611480093B6
:1071C8000192FFF755F97968019A31442046FFF793
:1071D800E5FEFDF701FC009B0B481946FFF748F94F
:1071E800B968002231442046FFF7D8FEFDF7F4FBCA
:1071F800013540F277139D42ABD103B0BDE8F08F63
:107208001C1100202F7B0308307B03081C3E030859
:10721800052838B50D460CD8064C60700648FEF7B0
:1072280037FEFDF7D9FB29461020FFF78AFFFF2319
:10723800637038BD00000020FE790308022838B5C5
:107248000D460CD8064C20700648FEF74DFEFDF79B
:10725800C3FB29460820FFF774FFFF23237038BDBE
:1072680000000020FE7903080CB407B510F02000D8
:107278000BD079B92320FDF751FB05A9049801919A
:10728800FEF740FDFDF7A8FB012003B05DF804EB15
:1072980002B070470020F8E70CB4C30607B500D564
:1072A80061B905A904980191FEF72CFDFDF794FB3F
:1072B800012003B05DF804EB02B070470020F8E746
:1072C8002DE9F04F354C87B08046354A23786088E1
:1072D80002EB8303D3F80491F9F7FCFAD0E901A390
:1072E8000493304B1B7813B9CDF810A09A4608F0D8
:1072F8004003DFF8BCB005930026A379002B08BF34
:1073080001239E4206DB284B08349C42DDD107B09E
:10731800BDE8F08F6279237906FB0323049A0136CE
:10732800D55CBAF1000F11D1B5FA85F77F090DB315
:1073380005F00F032D0940350293CDE900654B4652
:107348005A4639464046FFF7A7FFD6E71AF80330F2
:10735800EA1A57425741C3B103F00F021B094033E1
:107368000292CDE900635A464B4639464046FFF73C
:107378007BFFDCE7059B002BBFD100964B460B4AF1
:1073880039464046FFF788FFB7E700964B46074A5D
:1073980039464046FFF768FFC9E700BF6838030869
:1073A80070360308B80E002040390308507B0308E4
:1073B8003A7B03082DE9F04F87B005AA8C492CF0D9
:1073C80037F8064628B94120FFF77AFF07B0BDE82D
:1073D800F08F8849DFF86082FEF7D6F988BB8648C7
:1073E800864C874E874FFDF70BFB04F59C75A379F8
:1073F8002168A28808EB830301F13841B2FA82F2CE
:10740800890A4131D3F80431C2F11F023046FFF72F
:107418002FF8E17911B13846FFF72AF80834FDF75B
:10742800DBFAA542E3D1724905AA00202CF000F846
:107438007549FEF7A9F90028C8D16E48FFF725F865
:10744800C4E708F5FC770024B94617F8343008EB90
:107458008303E500D3F804A150462BF035FA5146D2
:1074680002463046FEF754F938B101341B2CECD1F2
:1074780031466648FEF774FCA8E705AA5C492BF07C
:10748800D7FFA8440746F9F71BFF98F8FE310646D0
:10749800002B40F09880002800F39F80A944B9F899
:1074A8000200F9F717FA3D78002D00F08980F3B251
:1074B800019399F8046099F80530019AD0F804808E
:1074C8005349384602FB0636FEF75EF960B908F8FC
:1074D800060018F80680B8F1000F16D14D48FDF7E0
:1074E8008FFA73E7012372E0602D8CBF613D413D47
:1074F800072D65D8781CF9F7E3FE0F2860D8013509
:1075080040EA051508F80650E3E74046FBF75AFF3E
:107518008146002854D04FEA1813403302933E4F57
:1075280008F00F030026039300252EE07888F9F76A
:10753800D1F97A793B7905FB03234268D15C41454F
:1075480022D1B44204D101998D421DD00021D154D9
:10755800DDE9021231485FFA85FB5FFA86FAFEF729
:1075680087FF59465046FEF7D9FFB44209D12C4847
:10757800FEF77EFF50465946FEF7D0FF2948FEF732
:1075880077FF2948FDF73CFA0135BB79002B08BF86
:1075980001239D42CADB01361B2E07F10807C3D120
:1075A800D9F80010B9F80420204801F13841B2FA9E
:1075B80082F2890AC2F11F024131FEF75AFC05E73F
:1075C800FEF746FC02E7002801DD9E4207DD0122A6
:1075D80017491848FEF7C4FBF8E6012882D105AA26
:1075E800034900202BF024FF013E074656E700BF61
:1075F800457C0308D2760308647B0308C03000206A
:10760800677B0308CA7A0308727B0308767B030842
:107618005F7B0308987B0308683803089E7B030890
:10762800C27B0308C57B03085BA50308CF7B03085F
:10763800927B0308BA750308703603082DE9F04FEA
:107648004A4085B098461D4FD34306460D46002450
:107658000393204604F090FF0E9B184228D0039B0A
:10766800174ADFF860A0034214BF4FF001094FF03A
:10767800000910EA050302934FF00C0303FB0423EF
:107688004946D3F808B0CDF800B014BF3A46524680
:1076980043463046FFF7E8FD029ACDF800B043466E
:1076A800002A14BF52463A4649463046FFF7F4FDD1
:1076B8000134182CCDD105B0BDE8F08F937C0308B8
:1076C80044700308DB7B030870B506462BF0FCF812
:1076D800114C054690B11122002120462BF071FF74
:1076E8002A460E4930462BF098FF38B1102D2A460D
:1076F800314628BF102220462BF0A1FF2378064AE6
:10770800002B08BF0121054B1CBF00211346012097
:10771800034ABDE87040BFE508210020E6A503083C
:10772800EA7B030870B505462BF0CEF8044690B105
:10773800112200210F482BF044FF22460E4928460B
:107748002BF06BFF38B1102C2246294628BF102297
:1077580008482BF074FF094B13F8112F002A064A2A
:1077680006BF012113460021054A0120BDE87040EB
:1077780092E500BF19210020E6A503080821002092
:10778800E27B03082DE9F04F002489B08346924636
:107798000D4626464FF019094FF46178BAF1000FEB
:1077A80022D004EB84030AEB030705223946284656
:1077B80007932BF0D3FE3A79079B19FB02820492B8
:1077C800FA781AF8033019FB02820392BA78029207
:1077D800B0FA80F67A78019276090093104A234627
:1077E80031465846FFF740FD2B790D4A19FB0383B4
:1077F8000493EB7819FB03830393AB7802936B78BC
:10780800019315F8053B0093314623465846013449
:10781800FFF742FD0A2CC1D109B0BDE8F08F00BFC7
:10782800F27B03082DE9F0478AB08246F8F79EFDFF
:10783800064638B1002247490120FFF7A3FF0AB0E6
:10784800BDE8F0875046F9F73BFD092804467ADC85
:10785800850005EB00080AF101008DF81F60F9F7B3
:1078680021FD3C4F824608EB07093E4650B1F9F727
:1078780027FD0D2806D89DF81F3008F807000133AA
:107888008DF81F305046F9F70DFD824658B1F9F7CB
:1078980017FD052807D82B19334458709DF81F3059
:1078A80001338DF81F305046F9F7FCFC824658B179
:1078B800F9F706FD082807D82B19334498709DF866
:1078C8001F3001338DF81F3008F103010DF11F023D
:1078D80031445046F9F7F7FC9DF81F20052A2AD1B4
:1078E800002308A9484608938DF824302BF036FE6B
:1078F8002B19334493F801C020B1BCF1000F1AD002
:107908009B78C3B1254472194FF46170117919231A
:1079180013FB01010491D17813FB010303939378BE
:107928000D4ACDE901C30021735D00930846234643
:10793800FFF7B2FC83E7002348F8073089F80430E2
:10794800FEF786FA7BE70923324604490448FEF726
:1079580007FA74E75C630020F27B0308927B030854
:10796800BA7503082DE9F047344F8CB006468946AE
:1079780015460024C4EBC40309EB03021068918880
:107988009279089040F30748ADF824108DF8262026
:10799800B8F1000F4AD0002D4DD02B440AA9186821
:1079A8009A880A909B79ADF82C2008A807228DF8B0
:1079B8002E302BF0D3FD9DF82E3006939DF92D30F7
:1079C80005939DF92C3004939DF82B3003939DF972
:1079D8002A300293B0FA80FA9DF8293001934FEAD1
:1079E8005A1A9DF8283000933A46234651463046A5
:1079F800FFF73AFC9DF8263006939DF9253005934C
:107A08009DF9243004939DF82330CDE902839DF835
:107A1800213001939DF8203000933A462346514681
:107A280030460134FFF738FC102CA3D10CB0BDE868
:107A3800F047FCF7D1BFAA46DCE700BF087C030883
:107A48002DE9F0478AB005462AF03EFF024630B9D4
:107A580085490120FFF786FF0AB0BDE8F0870522B7
:107A680082492846FDF754FE044670B90146702243
:107A78007D482BF0A6FD7E4B1C60DC609C615C623F
:107A88001C63DC639C645C65E6E70422794928464C
:107A9800FDF73EFE044620BB2846F9F703FC0746DF
:107AA8000028D9D02AF010FFDFF8EC81064658F8F4
:107AB80024501DB97048FEF753F9CDE732462946E0
:107AC8003846FDF725FE50B920461CF0EFFA294646
:107AD8006A48FEF7CEF96A48FFF7B2FFBCE70134FF
:107AE800E5E7072267492846FDF712FE0446002805
:107AF8006ED1284620212BF07BFD054680BB6248CD
:107B0800FEF7B6FC2C46614D214628460134FEF7A7
:107B1800AFFC0E2CF8D1FCF75FFF554EDFF87C91D7
:107B28005B4FDFF87C81002421464846FEF7A0FC25
:107B3800DFF870A1002532680123AB40134214BF5F
:107B48003946414650460135FEF792FC0E2DF2D1DA
:107B58000134FCF741FF082C06F10C06E4D17BE761
:107B680001AA4C494B4E2BF063FC02AD00283AD0D9
:107B7800022C15D1029A072A35D803990D2932D833
:107B88000378722B17D06E2B2DD10C235343384812
:107B9800012202FA01F1C25822EA0102C25013E09E
:107BA800F9F78EFB01AA45F82400314600202BF096
:107BB8003FFC0134DAE70C232D4C5343012000FA33
:107BC80001F1E0580843E0502E48FFF739FF43E73A
:107BD800284601AA2F492F4E2BF02AFC002402AD7B
:107BE80078B1082C02D1FEF733F935E7F9F768FBCD
:107BF80001AA45F82400314600202BF019FC013475
:107C0800EEE7082CEFD1029B0F2BECD8DDF80CE047
:107C1800BEF1070FE7D8049F0D2FE4D8059E06F1A3
:107C28006402C82ADFD8069DFF2DDCD8079864288F
:107C3800D9D808996429D6D88842D4DA099C032C63
:107C4800D1D8DFF824C0C3EBC3020CEB02030CF855
:107C580002E018715F709E70DD7059719C71084860
:107C6800FFF7EEFEF8E600BF305A0020A9790308B6
:107C78006C600020257C0308487903082A7C0308E7
:107C8800FE790308347C0308697903083C7C0308FF
:107C9800727C0308457C030854390308CB7A03082F
:107CA800837D0308417C03082DE9F04FDFF818B104
:107CB80089B08046894616460D4614460027002E90
:107CC8006DD00C22214628462BF048FC94F90B3045
:107CD800049394F90A300393B4F908300293B4F981
:107CE80006300193B0FA80FAB4F9043000934FEAF1
:107CF8005A1A3B465A4651464046FFF7B5FA95F997
:107D08000B30049395F90A300393B5F908300293C0
:107D1800B5F906300193B5F9043000935A463B464D
:107D2800514640460137FFF7B7FA082F05F10C0511
:107D380004F10C04C3D10024DFF890A0254686B3D3
:107D48000027012303FA07FB325959F8043053403E
:107D58003BEA030314BF0123002312EA0B0F079326
:107D680006D000972B46524607994046FFF77CFA03
:107D780059F804301BEA030F06D000972B465246E9
:107D880007994046FFF788FA01370E2FD9D10135F8
:107D9800082D04F10C04D2D109B0BDE8F08FB24629
:107DA800ADE73746012359F80420BB40134206D0FB
:107DB80000972B46524601214046FFF76DFA0137DE
:107DC8000E2FEFD1E3E700BF477C03085F7C030871
:107DD800F0B58BB00546F8F7C9FA002868D03549E0
:107DE800002201200BB0BDE8F0405DE72D2903D04B
:107DF800A1F13003092B56D8052C04DD0BB0BDE8E2
:107E0800F040FEF725B82846F9F75AFA0AAB621C83
:107E180003EB440424F80C0C15F8013F303B092B04
:107E2800FAD9144629780029E0D1062CE6D1BDF903
:107E38001C309AB2072AE1D8BDF91E40A4F2EE22FE
:107E480092B240F2DC508242D8D8BDF92050A5F257
:107E5800EE2292B28242D1D8BDF92260B442CDDC82
:107E6800B542CBDBBDF9247007F1640292B2C82A8F
:107E7800C4D8BDF926001128C0DCDFF838C00C22B0
:107E880002FB03C240B29480D58016819772D072EB
:107E9800CDE90370CDE901560094074A0846FFF77B
:107EA800FBF90BB0F0BD2029A8D101352246B8E76F
:107EB8000446B7E76C600020477C03082DE9F74FBC
:107EC800DFF864A081468B4617460E46002447B368
:107ED80007EB84080422414630462BF03FFBB8F8F4
:107EE80002300193B0FA80F537F8243000936D0919
:107EF8002346524629464846FFF7B6F97388019348
:107F08003BF824300093524623462946484601341C
:107F1800FFF7C2F9042C06F10406D8D103B0BDE876
:107F2800F08F3D46EAE700BF747C0308F7B50546C5
:107F3800F8F71CFA064630B12A490022012003B09E
:107F4800BDE8F040BAE728492846FDF71DFC38B9D6
:107F5800244B264AC3E90022C3E9022203B0F0BD3C
:107F68002846F9F7ADF90328044632D82846F9F728
:107F780099F9074660B1F9F7A3F90126054638468D
:107F8800F9F790F940B903B0BDE8F040FDF760BFDC
:107F980040F2EE250646F2E7F9F792F9002EF2D004
:107FA800A5F2EE2240F2DC539A42ECD8A0F2EE227F
:107FB8009A42E8D80B4B0E4A23F8245003EB84036B
:107FC80000215880CDE9005023460846FFF764F9A0
:107FD800C4E7084908480323324603B0BDE8F04027
:107FE800FDF7BEBE406F0020A9790308E803D0075B
:107FF800747C0308CA760308BA7503082DE9F04FA4
:108008002DED088BDFF80C9193B0804692460D4613
:108018001446002695ED008AB5EE408AF1EE10FA76
:1080280070D0D5ED019A95ED029AD5ED038ABAF193
:10803800000F3ED094ED000A94ED01BAD4ED02AAE7
:1080480094ED03AAB4EE408AF1EE10FA5FD1F4EE93
:108058004B9AF1EE10FA5AD1B4EE6A9AF1EE10FA90
:1080680055D1F4EE4A8AF1EE10FA0CBF0127002729
:108078000FA8FDF705FCB0EE4B0A83460CA8FDF7E8
:10808800FFFBB0EE6A0A059009A8FDF7F9FBB0EE10
:108098004A0A049006A8FDF7F3FB059B049A03908F
:1080A8000292CDE900B34A46334639464046FFF7C7
:1080B800DBF8B0EE480A0FA8FDF7E2FBB0EE690A5C
:1080C80007460CA8FDF7DCFBB0EE490A834609A871
:1080D800FDF7D6FBB0EE680A049006A8FDF7D0FBC2
:1080E800049B0390CDE901B3009733464A4600212B
:1080F80040460136FFF7D0F8082E05F1100504F1C7
:10810800100487D113B0BDEC088BBDE8F08F0027B1
:10811800AEE700BF857C03082DE9F0474B4FDFF839
:108128004881DFF8489104462046F8F71FF90646CB
:1081380028B1002246490120BDE8F0475EE7052244
:1081480039462046FDF7E4FA58B9414B00221A6037
:108158001A611A621A631A641A651A661A67BDE800
:10816800F087042241462046FDF7D2FA054620460C
:1081780015BBF9F797F806460028F0D02AF0A4FBBB
:108188002C465FFA80FA59F8245025B93148BDE8E1
:10819800F047FDF7E5BD524629463046FDF7B8FAE7
:1081A80040B9204611F098FF29462B482B4CFDF783
:1081B80060FEB9E70134E6E7F9F782F807280546D3
:1081C8003BD82046F9F76EF8064648B3F8F7C4F9E5
:1081D8001F4B03EB051383ED000A01243046F9F722
:1081E80061F8064638B1F8F7B7F9194B03EB0513F0
:1081F80083ED010A01343046F9F754F8064638B1E0
:10820800F8F7AAF9124B03EB051383ED020A0134C0
:108218003046F9F747F828B9BDE8F047FDF718BE2A
:108228000446DBE7F8F798F9094B032C03EB05152F
:1082380085ED030A3FF47DAFEEE732460723084990
:108248000848BDE8F047FDF78BBD00BFA9790308D2
:10825800C83A0020487903082A7C0308FE790308F5
:10826800927B0308BA750308257C03085439030870
:108278002DE9F04F834689B092460D4614460026F4
:108288004FF019094FF46178BAF1000F45D00A226E
:10829800214628462BF062F923890793E388069341
:1082A80023790593E3780493A3781D4A19FB038384
:1082B8000393637819FB0383029323780193B0FA3D
:1082C80080F7637900937F09334639465846FEF7AD
:1082D800CBFF2B890793EB8806932B790593EB78D3
:1082E8000493AB780E4A19FB038303936B7819FB4D
:1082F800038302932B7801936B79009339463346B5
:1083080058460136FEF7C8FF1E2E05F10A0504F18E
:108318000A04B9D109B0BDE8F08F5746D9E700BFC4
:10832800997C0308F0B58BB00746F8F71FF80446A8
:1083380030B100225B490120FFF79AFF0BB0F0BD76
:108348003846F8F7BDFF1D28054600F3A3800A2626
:108358004643781C8DF82740F8F7A4FF514C074690
:1083680050B1F8F7ADFF032806D8A31958719DF846
:10837800273001338DF827303846F8F793FF074642
:1083880058B1F8F79DFF0D2807D80A236B43E0542E
:108398009DF8273001338DF82730711C0DF1270225
:1083A80021443846F8F78FFFF8F77CFF074660B19D
:1083B800F8F786FF222808D80A2303FB0543D8705C
:1083C8009DF8273001338DF827303846F8F76AFFD3
:1083D800074660B1F8F774FF0D2808D80A2303FB95
:1083E800054318719DF8273001338DF827309DF823
:1083F8002730062B07D0A2190023A35153601381FD
:10840800FDF726FD9AE70A2606FB054600233846AF
:10841800F3803381F8F746FF074638B1F8F750FF85
:108428009DF82730F08001338DF827303846F8F76B
:1084380039FF50B1F8F744FF0A2303FB05431881BD
:108448009DF8273001338DF82730174B4FF0FF3256
:108458001A600A226A43A3184FF4617619890791B2
:10846800D988069119790591D978049198781921B4
:1084780011FB00600390587811FB00610291A25C27
:1084880001925B79009300212B46084A0846FEF7C3
:1084980003FF53E71D23224605490648FDF760FC04
:1084A8004CE700BF38610020A8080020997C030829
:1084B800927B0308BA7503082DE9F04F2E4EDFF8BA
:1084C800C0A087B0814690460D46144602F1280B9D
:1084D80095F9022000232949591891F9061091426B
:1084E80045D00833282BF6D108345C4505F108053A
:1084F800EED107B0BDE8F08F0822214628462BF0C0
:108508002DF8627994F9023056F822200492A27963
:1085180056F822200392227956F822200292E27815
:1085280056F822200192B0FA80F7228800927F093B
:10853800524639464846FEF797FE6A7995F9023061
:1085480056F822200492AA7956F8222003922A7912
:1085580056F822200292EA7856F8222001922A88B8
:108568000092394652464846FEF796FEBCE7B8F1F7
:10857800000FC1D14746E0E728740308E83B002014
:10858800BD7C03082DE9F04188B00346F7F7EEFEFD
:10859800044630B147490022012008B0BDE8F04147
:1085A8008AE7CDE9060018465D1CF8F789FE414BBD
:1085B80040B203EBC40696F90220824275D001341A
:1085C800052CF6D1002634462846F8F76BFE0746F8
:1085D80028B1F8F775FE0134ADF81800E4B2DFF8F9
:1085E800D88000253846F8F75DFE074600B3F8F74F
:1085F80067FE002258F822108842D3B203D0013215
:10860800102AF7D1002358F82320904210D1022DC8
:108618001AD0032D1DD05A1E012DD2B20FD00B2A0D
:1086280003D88DF81B300134E4B20135042DD9D1BB
:10863800052C14D808B0BDE8F041FDF709BC042AA0
:10864800F3D88DF81C30EEE7052BEED88DF81E30E8
:10865800E9E79A1E0D2AE8D88DF81D30E3E706AB46
:1086680003CB154A71609DF81D10306052F8211037
:1086780004919DF81E109DF91A3052F821100391AB
:108688009DF81C1052F8211002919DF81B1052F809
:10869800212001920021BDF8182000920846074ABF
:1086A800FEF7FAFD08B0BDE8F0818DF81A00012444
:1086B8008AE700BFBC3B002028740308BD7C030880
:1086C8002DE9F04FDFF8DCA087B0814690460D46D3
:1086D80014460026B8F1000F61D00622214628462C
:1086E8002AF03CFFB0FA80F720781AF05BFC83464A
:1086F80060797F091AF056FCBBF1000F1DD09BF87A
:108708000810A27894F803B094F801C04FF4617E81
:10871800192313FB02E213FB0BE394F804E000B106
:10872800007ACDE90223CDE904E0CDE9001C334607
:10873800524639464846FEF797FD28781AF032FC2B
:10874800834668791AF02EFCBBF1000F1DD09BF808
:108758000810AA7895F803B095F801C04FF4617E27
:10876800192313FB02E213FB0BE395F804E000B1B5
:10877800007ACDE90223CDE904E0CDE9001C3346B7
:10878800524639464846FEF787FD0136142E05F154
:10879800060504F106049DD107B0BDE8F08F4746F1
:1087A800CBE700BFDA7C03082DE9F04186B0074625
:1087B800F7F7DCFD044638B1002253490120FFF7E2
:1087C8007FFF06B0BDE8F0813846F8F779FD132839
:1087D800054600F3918006264643781C8DF817401D
:1087E800F8F760FD484C074660B1F8F769FDC0B27C
:1087F8001AF0BCFB30B10378A3559DF8173001334C
:108808008DF817303846F8F74DFD074660B1F8F790
:1088180057FD0D2808D8062303FB054358709DF81B
:10882800173001338DF81730B11C0DF117022144B0
:108838003846F8F748FDF8F735FD074660B1F8F710
:108848003FFD012808D8062303FB054318719DF84E
:10885800173001338DF817303846F8F723FD78B113
:10886800F8F72EFDC0B21AF081FB48B1062303FBCE
:10887800054302785A719DF8173001338DF8173087
:108888009DF81720042A4FF0060327D103FB054360
:1088980000221A715A7120F077FF06236B43E618FD
:1088A800E05C1AF07FFBF278B778192380464FF422
:1088B8006174707913FB074713FB02441AF072FBCB
:1088C800017A737898F80820039131790F48009756
:1088D800CDE901412946FDF7CCFA72E7052A04D112
:1088E80003FB054300225A71D5E7062AD3D0A21903
:1088F8000023A3519380CEE7132322460449054859
:10890800FDF72EFA5DE700BF486E0020DA7C030809
:10891800927B0308BA7503080EB400B584B005ABA2
:10892800019053F8042B0649039301A8FDF722F997
:10893800019B00221A7004B05DF804EB03B0704785
:10894800F907000810B44C09012250F8243001F04E
:108958001F0102FA01F123EA010340F824305DF80F
:10896800044B704710B44C09012250F8243001F030
:108978001F0102FA01F10B4340F824305DF8044B63
:10898800704700BF4B0901F01F0150F82320012355
:1089980003FA01F1114214BF18460020704700BFC6
:1089A80038B5064C064DAC4206D2616820461434F0
:1089B800F8F764FBAC42F8D338BD00BF70B90308C0
:1089C80020BE030808B5FFF7EBFF04F047FEBDE83B
:1089D8000840F8F71FBD2DE9F04F0F468DB0C1498B
:1089E8000646FCF7EBFE0546002840F01682BE4915
:1089F8003046FCF7E3FE0546002840F01082BB49EC
:108A08003046FCF7DBFE0546002840F00A82B849EC
:108A18003046FCF7D3FE0546002840F00482B549ED
:108A28003046FCF7CBFE002805460ABF012408247F
:108A380035460FB144F01004AF492846FCF7BEFE96
:108A4800002800F0F28144F02004F8F7F5FAFFF767
:108A5800A7FF14F0090F00F061820020FDF77CFDEC
:108A680014F48073039340F0EA81A448FBF7C8FF2D
:108A780004F01803182B40F0E581A148FBF7C0FF6C
:108A88000123029304F48473082B02D10020FDF71C
:108A980051FC14F080050BD19A4B1A78002A9A4A97
:108AA80006BF012113460021984A2046FEF7F4FB31
:108AB8002046FEF705FC002D40F04182944F954B6F
:108AC8003E781B78944D954AF01A464205EB83038D
:108AD8004641D3F8E03231462046FEF7C5FB3B78E5
:108AE8008E4A05EB83053146D5F8E0328C4D204699
:108AF800FEF7D2FBD5ED007A8A4AF5EE407AF1EE20
:108B080010FA0CBF012100212046FEF7C5FB2A46BA
:108B18008549864D2046FFF771FA854A85492046E2
:108B2800FFF7C2F895F90210834AB1FA81F14909B1
:108B38002046FEF7B1FB2A4680492046FEF712FF81
:108B48007F4B1F687F4B93F82A2002B1DF6A7E4B68
:108B5800DFF8F8A1D3F80090DFF84CB200265AF8F5
:108B68002650002D40F07181DFF840A22E4669EAB8
:108B7800070B764B53F82650002D40F08681744F32
:108B8800744E6FF07F4300933A683168724B204609
:108B9800FEF754FD40F202230093BA68B1686F4BA8
:108BA8006F4F2046FEF74AFD6E48DFF804C20126E3
:108BB8002B5CEA5D0CA919440DF1300E01F8202C4C
:108BC80015F80C108E440EF8102C16B1591A4E4296
:108BD8004E410135082DEBD13146002508AB624ADC
:108BE8008DF8185020468DF82850FEF73DFB04AB51
:108BF80031465D4ADFF8BCB1DFF8BC912046FEF78C
:108C08004BFB5A4A5A492046FFF756FC594A5A49DB
:108C18002046FFF755FD594A59492046FFF728FBDA
:108C2800584A59492046FFF749F9584A58492046B1
:108C3800FEF7A8FD0126574B5748DFF8DC800222D3
:108C4800991930442AF08AFC1BF815304344B0FACD
:108C580080F793F8F82019F81530022B4FEA5717C8
:108C680040F0378116F80B304FF0190A40F2EE2128
:108C78001AFB0313CDE9002339462B46474A204601
:108C8800FEF7F2FA16F80930444A40F2EE211AFBD0
:108C98000313019319F815309844394698F8F830B9
:108CA800009320462B46FEF7F7FA0135122D06F100
:108CB8000206C0D1134B3A4E13F8112F002A124A5C
:108CC80006BF012113460021364A2046FEF7E4FA82
:108CD80021460020FEF735FA14F0080F214600F06F
:108CE80015816BE0F37C0308FA7C0308027D030816
:108CF800087D0308727B0308117D03081F7D0308A4
:108D08002B7D03086C230020E6A50308EA7B0308F3
:108D180020700020706C0020703603083B7D03082B
:108D2800C83A0020447D0308844A0020305A0020B5
:108D38006C60002098650020537D0308286500209A
:108D4800284B0020B80E0020C0380020C039030886
:108D58001061002004650020777D03087E7D0308EC
:108D6800687403085424002092760308BC3B002052
:108D7800544A0020486E0020986F00203861002077
:108D8800D8630020406F0020306F00205C63002013
:108D9800A4630020736F00204F6F0020AD76030896
:108DA80090230020E27B0308607D03086C7D0308A4
:108DB800181F0020746F0020506F00200020FEF75D
:108DC8003DFA21460120FEF739FA5F4D214602207F
:108DD800FEF734FA33782B70039B13B95B48FDF721
:108DE80083F8FF232B700027F8B221460137FEF7DE
:108DF8000FFA062FF8D173786B70039B002B7CD188
:108E08005248FDF745F85248FBF790FDFF236B7079
:108E1800F8F7FCF80DB0BDE8F08F012409E602244C
:108E280007E6042405E6812403E64A492846FCF7B8
:108E3800C5FC00283FF409AE44F4807405E600231D
:108E480002931FE6012302931CE62B78DBB14FF057
:108E5800010808FA06F869EA070313EA080F14BFBD
:108E6800012100212B465A462046FEF7FDF967EA04
:108E7800090313EA080F5A462B4614BF01210021A3
:108E88002046FEF709FA013669E62B78FBB14FF068
:108E9800010808FA06F819EA080F0BD067EA09036F
:108EA80013EA080F52462B4614BF01210021204621
:108EB800FEF7DAF918EA070F09D01BEA080F2B4664
:108EC800524614BF012100212046FEF7E5F901367C
:108ED8004FE600922B4639461F4A2046FEF7C4F952
:108EE80019F815301C4A9844394698F8F830009318
:108EF80020462B46FEF7D0F9D7E6FF236B70029B7E
:108F0800002B85D01548FBF77BFD81E73078FEF70D
:108F180095F921467078FEF77BF9F0E7A20705D5A9
:108F28000F4B21461878FEF789F971E763077FF53B
:108F38006FAF0B4B21465878FEF76AF968E7214670
:108F48001820FEF7FEF8DAE700000020FE79030893
:108F5800367D03081A7D0308BD760308857D03085E
:108F680090230020012136E5002134E52DE9F74F53
:108F78003B4B3C4C1A785B78009022706370F8F792
:108F88005BF8FFF70DFD0025DFF8DCB0A8460D27DC
:108F9800354B00996F43DE19D6F800904846FCF728
:108FA800DBFB00283DD0B8F1000F01D0FBF714FD22
:108FB80049462E485F44FDF75BFA00213046FEF72C
:108FC800B5F8FBF709FD3B7903F01803082B3BD0F4
:108FD800102B3DD03046FDF773FF0D2303FB05B37F
:108FE800B3F80900F7F776FC0746C0B13046F7F743
:108FF800C5F9D7E901218246024401443046F7F712
:10900800F5F960B9019049461948FDF731FA7968D0
:10901800019A51443046FDF7C1FFFBF7DDFC08F12A
:109028000108013540F277139D42B0D1F7F7EEFF02
:10903800FF2323706370B8F1000F0DD10D4803B002
:10904800BDE8F04FFCF78CBE0B48FCF74DFFC1E7BD
:109058000948FCF71DFFBDE703B0BDE8F08F00BF6E
:10906800E4140020000000201C3E0308347B0308A1
:109078008F7D030848790308FE7903082DE9F74F27
:10908800814629F021FC054628B1012822D199F80A
:1090980000302A2B1ED17D48DFF808827C4FFBF771
:1090A800AFFC00244FF00D0909FB048638463168EF
:1090B800FDF7DEF9291C18BF01213046FEF736F806
:1090C8000134FBF789FC40F277139C42ECD103B0E2
:1090D800BDE8F08F3D2148462AF08AFA002800F0C2
:1090E800D080074617F8013C202B07F1FF3232D019
:1090F800A7EB09070130054601302B78202BFAD061
:10910800DFF8A0A14FF00008D346FFB20D2303FB00
:1091180008A42668304629F0D7FB3146024601905C
:109128004846FCF7F5FA0646002840F09D80019B6A
:10913800BB4240F09980237903F06001202951D087
:109148000BD8F1B15348FCF70BFE204603B0BDE83D
:10915800F04FFDF7B5BE1746C4E7402958D060293F
:10916800F0D14D4A02EBC606002796F8D0A3B946BF
:109178003B46574502D2B9F1000F35D0002BE1D05C
:109188000EE003F00706042E284618D113F0CAF99A
:10919800D4F8053083420146D4D32046F7F7C6FBFE
:1091A8000D2303FB08B83D48D8F80010FDF760F917
:1091B8000021204603B0BDE8F04FFDF7B7BFF8F730
:1091C8007FF8B4F805500146B4F80700AAB283B294
:1091D8001EB1022E1CBF2AB203B29142B2DB9942E1
:1091E800B0DCDAE76679BCE7D6F8CC2352F827007A
:1091F80060B129460193FCF7C7FA019B30B939469B
:1092080020464FF00109F7F791FB4B460137B0E7CD
:109218004FF00D0994F805A009FB08B95645BFDAC7
:10922800002DBDD02F4601353B78202BFAD02046A3
:10923800F7F766FB99F8043003F00703022B05469D
:109248000CD0032B0AD03846F8F73AF8A8552C2149
:1092580038462AF0CDF90136451CDFE73846F8F7DD
:109268002FF825F81600F2E708F1010840F2771305
:1092780098457FF44BAF0A4803B0BDE8F04FFCF7C0
:109288006FBD484603B0BDE8F04F6FE69F7D030809
:10929800347B0308BD7D030870360308B27D0308DC
:1092A800487903081C3E030810B50346F7F75EF833
:1092B800044628B9062208491846FCF729FA48B98D
:1092C800FFF76EFB054B002018701CB1BDE810407D
:1092D800FCF755BD10BD00BF347D0308791200208E
:1092E800074A084B10781B78074A834296BFC31A6F
:1092F800C3F180030020126818441044704700BF6F
:1093080004210020802000207C200020064A074BF2
:1093180010781B7883428ABFC3F18003C01AC01833
:10932800C0F17F00704700BF04210020802000208A
:10933800064808B54368DB68984705480549064A62
:10934800002303700B70136008BD00BFD82D0020E8
:1093580004210020802000207C20002010B5044635
:1093680000BF8068FAF7FCFB606840F2E933828945
:1093780000E0B3B10289013B12F0020F9BB2F8D0B2
:10938800017340F2E93300E05BB10289013B12F05E
:10939800010F9BB2F8D0037BA068FAF7E7FB00BF88
:1093A80010BDFAF78BFDA068FAF7E0FB00BF10BD0F
:1093B800F0B5077F836983B004464FF0020C0020A4
:1093C80000900E4615468DF804008DF800C0002F59
:1093D80034D01A0E8DF801200DEB0C02180C1F0A60
:1093E80093701070577006212046FAF7CDFD0621BC
:1093F8002068FFF7B3FF01236377236800BF9868ED
:10940800FAF7AEFB237F2268002B14BF0523042341
:10941800694650680022FAF763FD23683146002246
:1094280058682B46FAF75CFD23689868FAF79EFBA4
:1094380000BFA2692A44A26103B0F0BD0DF1010288
:10944800CCE700BF10B4144681611A4621465DF886
:10945800044BADE710B5044645F20821FAF794FD30
:1094680020680621FFF77AFF012363772068C72168
:10947800BDE8104072E700BF30B5027F83B000231B
:109488000446D82000938DF804308DF800005AB3B4
:109498000B0E8DF801300DF102030A0A080C9970C1
:1094A80018705A7041F288312046FAF76DFD06218E
:1094B8002068FFF753FF237F2568002B4FF0010337
:1094C80014BF05210421637700BFA868FAF748FB99
:1094D80000220B4668686946FAF702FDA868FAF7A1
:1094E80045FB00BF03B030BD0DF10103D5E700BF58
:1094F8000348436813B19B6A03B118470148704792
:10950800D82D00206C3B03081FB5FFF7F1FF044678
:10951800FFF7E6FEA38921880290A268019262887B
:10952800009262680248FCF7A4FC04B010BD00BFBA
:10953800CB7D03082DE9F04F87B04FEA820A0491EA
:10954800CDE9013000220B46514453F8040B8B42FD
:109558000244FAD1019B05922BB9424843681B6823
:109568009847002863D0FFF7C3FF43880393059B00
:10957800002B4AD03C4B029A3A4E1B68DDF814B0D7
:1095880092440399B3FBF1F901FB193303EB0B0286
:109598008A428CBFA1EB0309D946FFF7A9FF324BDA
:1095A800196883688B4248D973682E481B699847A5
:1095B8007168029C049D4F46AC4655F8043B304602
:1095C8001A468BB1D4F800E0D1F81480BB4271463A
:1095D8001FD2C04755F8042C2368716813442360D0
:1095E8000023BF1A45F8043C04345445E4D18B6980
:1095F800304698471C4A13684B441360019AABEBFA
:10960800090B3AB3BBF1000FBBD1059807B0BDE811
:10961800F08F4346E0463A4698472268D8F800302B
:1096280071683A44DF1B2260C8F80070DFE7019BCD
:109638000593059807B0BDE8F08F05980B490C4ACB
:10964800A0EB0B000590059800230B70137007B072
:10965800BDE8F08F059BA3EB0B030593059807B0B6
:10966800BDE8F08FD82D00207C20002004210020A8
:109678008020002070B5104D104E2B7831788B4229
:1096880084B016D00E4A03921A4402928CBF0C463C
:10969800CA1A04A98CBFC3F180020024012341F82F
:1096A800102D02A802220194FFF744FF0023337013
:1096B8002B7004B070BD00BF802000200421002062
:1096C800842000202DE9F04784B0FFF711FF83685C
:1096D80013B904B0BDE8F087FFF70AFF8568ED0A03
:1096E8001BD0DFF84C800026C14604AFD8F8043000
:1096F800AC196410D3F824A0E10210236A46484646
:10970800D0470F2809DD6B4653F8042B01320AD1E4
:109718009F42F9D12546AE42E8DBFFF7ABFF034B8A
:10972800ED021D60D5E7661CF5E700BF7C20002030
:10973800D82D002070B5194C194D237829789942F5
:1097480084B027D0174A03921A44029234BF0E46B7
:10975800CA1A04A934BFC3F180020026002341F8C5
:10976800102D02A802220196FFF7E4FE2378184480
:10977800C0B203062B7848BF80F080008342207077
:1097880002D0002004B070BD002301202B7023708C
:1097980004B070BD012004B070BD00BF802000205F
:1097A800042100208420002008B5FFF7A1FE80686E
:1097B800003018BF012008BD08B5FFF799FE806882
:1097C80000B908BD024843681B68984708BD00BF38
:1097D800D82D002008B5FFF7E7FFC8B10D48FBF703
:1097E8000FF90D4B1868FBF755F8FFF7A1FDFFF7C8
:1097F800E3FF48B1132002F0EDFEFBF7EDF8074850
:10980800BDE80840FBF7FCB86420F9F795F8EEE7E7
:1098180008BD00BF267E03081C1100202F7E030808
:10982800074A00235168814202F11C0204D0013327
:109838000C2BF7D100207047581CC0B2704700BFEE
:109848000400002001382DE9F0434FEAC00C394EDE
:10985800DFF804E1384FDEF81490DFF80081ACEB54
:10986800000406EB840483B06568BD420CBF012781
:109878000227A56847EA09074545CEF81470E16054
:1098880063613ED02D4B9D423DD014339D423CD068
:1098980014339D4232D014339D4239D014339D4243
:1098A80039D014339D4239D003F562739D423AD0C2
:1098B80014339D4239D014339D4232D014339D4223
:1098C80035D01F491F4B8D420CBF1D460025ACEB00
:1098D800000C06EB8C069209747CF56100210123CB
:1098E80001A88DF804408DF805208DF806108DF834
:1098F800073010F083FE03B0BDE8F0834FF4005545
:10990800E5E70225E3E72025E1E74FF40075DEE708
:109918004FF40035DBE74FF40015D8E74FF000753A
:10992800D5E7094DD3E7094DD1E7094DCFE7094DF3
:10993800CDE700BF00000020000002401C000240EC
:10994800580402400000021000020010020000103B
:109958002000001000200010001002400800024003
:109968000A4B0138C0EBC00003EB800070B4084C10
:10997800084E43686569B3420CBF012302232B4399
:1099880063610176427670BC704700BF000000201A
:1099980000100240000002402DE9F04F544C54F8EA
:1099A800204083B0002C5FD0E56DA1601F46904633
:1099B800504B6A686265236004F1620204F1E203B5
:1099C8006261A36180224FF48073C4E90323814656
:1099D800287E0DF0DBF9E86860B1FFF721FF09F197
:1099E8000102D2B20C21FFF7BBFF636DEA68A263E4
:1099F80024332365A86898B1FFF712FF09F1010223
:109A08000646D2B20B21FFF7ABFF2346EA7E3A495E
:109A18003046FFF717FF636DAA68E2632833E364F3
:109A280094F86100F9F7CEFC064694F86000F9F75F
:109A3800C9FC3A07824695F819B019D5C6B117F08E
:109A4800110F4FF00B0309F10100F07114BF4E2103
:109A58003E21B3715A463046F9F77AFDFB0743D5E4
:109A6800A36B6BB3E36B5BB3204603B0BDE8F08F29
:109A780017F0010F0CBF2E274E2718F0020F0AD03F
:109A88004EB10B2209F10103B271F37130465A4607
:109A98003946F9F75DFD18F0010FE1D0BAF1000F72
:109AA800DED00C2309F101008AF807008AF8063095
:109AB8005A4639465046F9F74BFDA36B002BD1D1D6
:109AC8002B7FAA7E8DF804209B090021012201A882
:109AD8008DF805308DF806108DF8072010F08EFDF2
:109AE800204603B0BDE8F08F3046FAF739F8B7E7FB
:109AF8002C5800207C3B0308390F00080348D0F895
:109B0800403113B100F59C701847704700000020E1
:109B18000348D0F8243113B100F58E701847704708
:109B2800000000200348D0F8083113B100F5807018
:109B380018477047000000200348D0F8EC300BB1FC
:109B4800E4301847704700BF000000200348D0F8F1
:109B5800D0300BB1C8301847704700BF0000002054
:109B68000348D0F8B4300BB1AC301847704700BF89
:109B7800000000200348D0F898300BB19030184707
:109B8800704700BF000000200248C36F0BB174305B
:109B980018477047000000200248036E0BB1583088
:109BA80018477047000000200248436C0BB13C3056
:109BB80018477047000000200248836A0BB1203024
:109BC80018477047000000200248C3680BB10430F2
:109BD8001847704700000020F0B44C4C049D00EB7F
:109BE800800004EB8004606800285FD0484F4E0076
:109BF8004FF42041F6B279628469240401F1FF31FF
:109C08004BD44168DFF814C146F4903401EA0C01E2
:109C18000C434FF420414460796202E0B1F1FF3F08
:109C280052D0846914F0020401F1FF31F6D04FF4E8
:109C38002041826279620A4602E012F1FF324CD377
:109C4800816911F04001F8D032494468DFF8CCC08E
:109C58007A6241EA0342013B1643DBB204EA0C0292
:109C6800013316432B44466082694FF4204112F0B9
:109C7800040201F1FF3107D14C1C36D0826912F081
:109C8800040201F1FF31F7D0426A05F8012BAB421B
:109C9800EAD14FF420427A620DE04C1CACD11E4A46
:109CA8007962138801339BB213800020F0BC70479F
:109CB80012F1FF3221D3836913F02003F8D0202357
:109CC800C3617A620120F1E7134A7962138801338C
:109CD8009BB220461380F0BC70470F4C7A622388F1
:109CE80001339BB208462380E0E70B4C7962238856
:109CF80001339BB210462380D8E707497A620A8865
:109D0800013292B218460A80D0E700BF5C580020A2
:109D1800B80E002000240002240F0020009800FC48
:109D2800F0B50E460178012985B0044653D00229C2
:109D380057D11D46836846F0800113B118689B8887
:109D48000385606840F2E933868901E0002B57D02B
:109D58000689013B16F0020F9BB2F7D0017340F25F
:109D6800E93301E0002B4BD00189013B11F0010FD1
:109D78009BB2F7D0037B60684FF0000C83894FF6E5
:109D8800FF764FF47A734FF0FF0E03E0013B9BB26E
:109D9800B34229D001898F07F8D580F80CE04FF439
:109DA8007A7302E0BBB2B3421ED00189C90703F13E
:109DB800FF37F7D5017BC9B20AB1117001320CF136
:109DC800010CAC45E6D1A368C3B11A689B889361BE
:109DD800012005B0F0BD90F90400411C01D0022813
:109DE80005DD002005B0F0BDFAF768F8EBE761790A
:109DF80000923246FFF7F0FE05B0F0BD0120F1E712
:109E08000392FAF75BF8039AB5E737B500F10C044B
:109E1800054600220A212046FAF708F91420F8F727
:109E28008BFD0F220A212046FAF700F90A20F8F7DD
:109E380083FD01AA032310212046FFF771FF0A20A2
:109E4800F8F77AFD9DF8043080336B839DF8053070
:109E58008033AB839DF806308033EB8300220A21E0
:109E68002046FAF7E3F80A20F8F766FD0DF1030239
:109E7800022120460DF0E0FC0DF1030209212046E5
:109E88000DF0DAFC11220A212046FAF7CFF801205A
:109E980003B030BD07B5032301AAF621FFF740FF41
:109EA8009DF805309DF804201B0243EA02439DF803
:109EB80006201343054AB2F92020C2F10802D34014
:109EC800034A136103B05DF804FB00BFEC6C00208B
:109ED800B80E002007B5022301AAF621FFF720FFDC
:109EE8009DF804209DF8053043EA0223024A938135
:109EF80003B05DF804FB00BFB80E002007B50323CC
:109F080001AA0021FFF70CFF9DF805309DF8040019
:109F18001B0243EA00439DF80600184303B05DF8AE
:109F280004FB08B5FFF7EAFF014B986108BD00BFC5
:109F3800B80E002008B5FFF7E1FF014B586108BDD6
:109F4800B80E0020F0B5037C012B85B004464DD037
:109F5800022B51D1836913B11A689B8813856069F4
:109F680040F2E933828901E0002B74D00289013B79
:109F780012F0020F9BB2F7D0C323037340F2E93308
:109F880001E0002B67D00289013B12F0010F9BB260
:109F9800F7D0037B60698389038999074FF0050728
:109FA80002AE4FF47A724FF0FF0C4FF6FF7506D4ED
:109FB800531E9BB21AB31A4603899907F8D580F83D
:109FC8000CC04FF47A7302E08BB2AB4217D002890F
:109FD800D20703F1FF31F7D5027BD2B20EB132704E
:109FE80001367A1E6FB117461A46E5E790F9140054
:109FF800431C01D0022824DD002005B0F0BDF9F78C
:10A008005DFFA36913B11A689B8893619DF80C00E2
:10A018009DF808609DF809109DF80A509DF80B20DE
:10A028009DF80D3041EA062143EA002342EA052261
:10A038000120A4F85010A4F85220A4F8543005B018
:10A04800F0BD02AB617D009343220623FFF7C4FDF8
:10A058000028DBD1D0E7F9F731FF9BE7F0B5037BA8
:10A06800012B85B004464DD0022B51D1436913B161
:10A078001A689B881385206940F2E933828901E0D8
:10A08800002B71D00289013B12F0020F9BB2F7D06E
:10A09800BB23037340F2E93301E0002B64D002894B
:10A0A800013B12F0010F9BB2F7D0037B2069838933
:10A0B800038999074FF0050702AE4FF47A724FF003
:10A0C800FF0C4FF6FF7506D4531E9BB21AB31A46FF
:10A0D80003899907F8D580F80CC04FF47A7302E029
:10A0E8008BB2AB4217D00289D20703F1FF31F7D503
:10A0F800027BD2B20EB1327001367A1E6FB11746AA
:10A108001A46E5E790F91000431C01D0022821DD2A
:10A11800002005B0F0BDF9F7D1FE636913B11A68E4
:10A128009B8893619DF80C009DF808609DF80910C4
:10A138009DF80A509DF80B209DF80D3041EA062144
:10A1480043EA002342EA052201206183A283E383D4
:10A1580005B0F0BD02AB617C00933B220623FFF7FC
:10A168003BFD0028DED1D3E7F9F7A8FE9EE700BF44
:10A178001749184B184A194810B4D1F8884044F4C4
:10A188007004C1F888401C6844F001041C605C68D5
:10A1980022405A601A6822F0847222F480321A60CF
:10A1A8001A6822F480221A605A6822F4FE025A6061
:10A1B800DA6A22F00F02DA621A6B002410404FF0BC
:10A1C800006218639C608A605DF8044B704700BFAA
:10A1D80000ED00E0001002400CC07FF8CCFC00FF4E
:10A1E80070470C4B1B78DB0700D570470A4A136889
:10A1F800002BFAD04FF47A7101FB03F39842F4D3A1
:10A20800064B1B781BB9064B99681B690B6000232A
:10A2180013607047994900205C510020505100207C
:10A22800344C0020704770B50B4C23689BB15A68BA
:10A23800821A002A0FDB0546002603E05A68AA1A8C
:10A24800002A08DB99681E731A682160184690472F
:10A258002368002BF2D170BD1C0F0020F8B52A220C
:10A2680004460021023029F0ACF90C4F00222346A5
:10A27800052104251046D65D9E700132052AD97045
:10A288001D719871597103F10803F4D101232380DA
:10A29800522384F82A3064232385F8BD246E0308EA
:10A2A800024B1A7959790FF03FBF00BF1C0F0020ED
:10A2B80008B51DF09DFC084B9B7943B1012B0AD1D1
:10A2C8000649074B0748084A0860DA6002E0044B71
:10A2D800054ADA60FEE708BD1C0F0020FC9F00203D
:10A2E80000ED00E0EFBEADDE0400FA052DE9F04F09
:10A2F8002DED028BA0F10A0385B00C46E72B00F286
:10A308009D87DFE813F0DC029B079B079B079B07F1
:10A318009B079B079B079B079B079B079B079B0725
:10A328009B079B079B079B079B079B079B079B0715
:10A338009B079B079B07BE029B079B079B07AF02D8
:10A348009B079B079B07A2029B0700049B079B0791
:10A358009B0717019B07B3069B0763049B074701ED
:10A368009B079B079B070D0505059B0788029B0715
:10A378009B079B029B079B079B079B079B077802F2
:10A388009B079B079B079B0759029B0715029B0787
:10A39800FE01E4019B079B079B079B079B079B0705
:10A3A8009B07A2019B075B019B078F039B07F10596
:10A3B8009B07C7059B079B079B079B07EE022C0380
:10A3C8002207CF06BC069B079B07300125019B0788
:10A3D8004507F9009B079B079B079B07E8009B071E
:10A3E8009B078D059B079B079B077D05AF05C80449
:10A3F8009B079B079B079B07B9049B07AA04880434
:10A408009B079B079B079B079B079B079B079B0734
:10A418009B079B079B079B079B079B079B07EE02D6
:10A428009B079B079B079B079B079B079B079B0714
:10A438009B079B079B079B079B079B079B079B0704
:10A448009B079B079B079B079B079B079B079B07F4
:10A458009B079B079B079B079B079B079B079B07E4
:10A468009B079B079B079B076F059B079B079B0702
:10A478009B079B079B079B079B079B079B079B07C4
:10A488009B079B079B079B079B079B079B079B07B4
:10A498009B079B079B079B079B079B079B079B07A4
:10A4A8009B079B079B079B079B079B079B079B0794
:10A4B8009B079B079B079B079B079B079B079B0784
:10A4C8009B079B079B079B079B079B079B074C05C5
:10A4D8009B0740051505A64952232268501C206099
:10A4E800137011F8013F002BF7D10125284605B05C
:10A4F800BDEC028BBDE8F08F9E48002201682568FC
:10A5080002EB42035B0019446E1C097A266029702D
:10A518000168256819446E1C497A2660297001680B
:10A5280025680B4401329B7A691C052A21602B702F
:10A53800E4D1DAE7202500212046FAF7A1FE013D03
:10A54800F9D123688C4A591C21601D7000F0AFBCFA
:10A558008A4B08461968FAF793FE20460021FAF755
:10A56800A7FE0125C2E7864D08462988FAF7A0FE0E
:10A5780069882046FAF79CFEB5F90430814AD91754
:10A5880082FB0323C1EBA301204689B2FAF790FEB0
:10A598000125ABE77C4D7D4E05F1280795F90210A2
:10A5A8007B4B93F906208A4203F1080300F05A8690
:10A5B8009E42F6D10835AF42F0D196E70B68754E4A
:10A5C800754A7178754D581C206019702368127887
:10A5D800591C21601A7023682A79591C21601A7045
:10A5E8002368AA78591C21601A7029882046FAF72E
:10A5F8005FFE298A2046FAF75BFE23680022591C71
:10A6080021601A702368EA78591C21601A7023683F
:10A618003279591C21601A702368F278591C21601C
:10A628001A7023683278591C21601A70718B204681
:10A63800FAF73EFE718A2046FAF73AFE2368327D21
:10A64800591C216001251A7050E7554B1E680023DC
:10A658008DF80830002E00F0B78602A930460BF0BE
:10A668002FFB336830465B68984733689B6807461A
:10A67800002B00F0CE863046984706462368494DA1
:10A688005A1C22601F7023682A78591C21601A708E
:10A6980023686A78591C21601A702368AA78591CA3
:10A6A80021601A7023689DF80820591C21601A70CF
:10A6B800A9882046FAF7FCFD23685A1C22601E7000
:10A6C80023682A7A591C216001251A700EE70A6846
:10A6D800354B36490125501C206015702268987842
:10A6E800561926601070226850192060157022686B
:10A6F800097850192060117019882046FAF7D8FD9A
:10A70800F4E60B6800255A1C0A601D700B685A1C79
:10A718000A601D700B685A1C0A6029461D70204685
:10A72800FAF7AEFD29462046FAF7AAFD0125DDE62F
:10A738001F4F3B78002B3FF4D8AEDFF87880002518
:10A748004646236818F81520591C21601A7071783C
:10A7580001EB810101EB810101F2EE212046FAF7BC
:10A76800A7FD3B780135AB4206F10206E9DCBCE601
:10A7780028510308001500208C1400202018002000
:10A788004C14002067666666BC3B0020103C002025
:10A79800E83B0020F83100207C6A0020503B002074
:10A7A8009C490020A0490020681700206A6A002000
:10A7B80044680020746F00208A4D0B682A79591C60
:10A7C80021601A7023686A79591C21601A702988D7
:10A7D8002046FAF76DFD2368AA79591C21601A7082
:10A7E80069882046FAF764FD2368EA79591C2160D4
:10A7F80001251A707AE6FEF7D7FF0546002840F0D3
:10A80800C78523685A1C0146226018702046FAF74B
:10A8180037FD294683E70B68734A581C5178206036
:10A8280019702368714A0021581C20601970236828
:10A838001279591C216001251A7057E6084608222A
:10A848006B49FAF705FD012550E60B68694A581C63
:10A8580011782060197023685278591C21600125ED
:10A868001A7043E6644D08462988FAF721FDA9883D
:10A878002046FAF71DFD29892046FAF719FD01251A
:10A8880034E65E4D05F17806287818F08BFB2368CE
:10A89800027A591C21601A7023686A78591C216051
:10A8A8001A702368AA78591C21601A702368EA78FC
:10A8B8000635591CAE4221601A70E5D115E6504D97
:10A8C800284628F001F800283FF40FAE2B4605442F
:10A8D800226813F8011B501C9D4220601170F7D1AB
:10A8E80003E6002306461D46DFF82C81DFF82CB16D
:10A8F800DFF82CA1CDE90033994603E00135282D76
:10A9080000F0CE8429464046EFB2FEF73BF8002817
:10A91800F4D0002240F20123ADF80820ADF80A3047
:10A9280040F6060240F60A33ADF80C20ADF80E30BA
:10A93800002D00F08684072F4FF0010300F28D846C
:10A9480002AA515DBBF800208B40134214BF0120BE
:10A958000020002840F07B8409F10109CEE7294B4B
:10A968001B8BB3F5006F00F20C85B3F5806F00F216
:10A978003C85B3F5007FB7EE008AF6EE007A28BF73
:10A98800B0EE678A204D05F10C06B5EC010A20EE01
:10A99800080A28F097FD81B22046FAF789FCAE42F2
:10A9A800F3D11A4D1A4F05F10C06B5EC010AD7ED93
:10A9B800077A80EE270A28F085FD81B22046FAF74B
:10A9C80077FCAE42F1D1134D05F10C06B5EC010A46
:10A9D80028F078FD81B22046FAF76AFCAE42F5D13C
:10A9E80083E500BF085900209C6A00205414002009
:10A9F800181F0020706C00208C580020486E002022
:10AA080008210020A01C0020CC1C0020243200209B
:10AA180030320020846C00204C4C0020101800209C
:10AA280099490020AF4E0B68B279AF4D591C21608F
:10AA38001A702B6820465988FAF73AFC2B6820468A
:10AA48001988FAF735FC71892046FAF731FCB18983
:10AA58002046FAF72DFC2B6820469988FAF728FC3F
:10AA68002B682046D988FAF723FCF1892046FAF7A3
:10AA78001FFC318A2046FAF71BFC2A68236892F8E3
:10AA88002620591C21601A702368B278591C21604D
:10AA98001A7023680022591C21601A70F188204618
:10AAA800FAF706FC31892046FAF702FC2368727D22
:10AAB800591C21601A702368B27D591C21601A70D4
:10AAC8002B682046B3F84C10FAF7F2FB23682A6883
:10AAD800591C92F8602021601A70B18B2046FAF751
:10AAE800E7FBF18B2046FAF7E3FB2B682046B3F827
:10AAF8006210FAF7DDFB2B682046B3F86410FAF70A
:10AB0800D7FB0125F2E4794D0B682A7A591C21609C
:10AB18001A70E98A2046FAF7CBFB698A2046FAF7C9
:10AB2800C7FBA98A2046FAF7C3FB23686A7B591C2E
:10AB380021601A70E98B2046FAF7BAFB298C204667
:10AB4800FAF7B6FB23682A7E591C21601A7023681D
:10AB5800AA7E591C21601A702B7F03EB83035900CE
:10AB680001F57A712046FAF7A3FB236800265A1CE0
:10AB7800226031461E702046FAF782FB23685A1C71
:10AB880022601E702368EA7E591C21601A702368AF
:10AB98006A7E591C21601A7023685A1C22601E7034
:10ABA80023685A1C22601E7023685A1C22601E707B
:10ABB80023685A1C22601E7023685A1C22601E706B
:10ABC80023685A1C226001251E708FE4484B03F548
:10ABD800967522685979501C20601170226819787E
:10ABE800501C2060117022685978501C2060117028
:10ABF80022689978501C206011702268D978501CFE
:10AC080020601170226819790A33501C9D42206017
:10AC18001170DED169E4374B1D6815F000653FF40B
:10AC280065AC0B68344E591C327821601A70337841
:10AC3800002B3FF45AAC0025E8B208F0BBFD2368AE
:10AC48004278591C21601A7081892046FAF730FB36
:10AC580033780135AB42EFDC47E4284B2849B3F998
:10AC6800003081FB0321DB17C3EBA101204689B229
:10AC7800FAF71EFB012539E4224D0846698AFAF7DE
:10AC880017FBA98A2046FAF713FBE98A2046FAF748
:10AC98000FFB01252AE423681B491848CA795D1C63
:10ACA80025601A7023685D1C25601A7023688078F7
:10ACB800164A5D1C2560187023681278581C20609D
:10ACC8001A7023680022581C20601A702368C979FA
:10ACD800581C206019702368591C216001251A70BE
:10ACE80004E400BFF831002000150020181F0020E0
:10ACF80038610020C03800207D1200208C6A0020B6
:10AD080067666666503B0020D4680020776900209B
:10AD18000B6801229918216015461A70FFF7E6BBE7
:10AD2800674B0846196AFAF7ABFA0125FFF7DEBB4D
:10AD3800644B03F1700522681978501C206011706B
:10AD480022685978501C2060117022689978501C2C
:10AD5800206011702268D978501C20601170226818
:10AD68001979501C2060117022685979501C206094
:10AD78001170226899790733501C9D422060117028
:10AD8800D9D1FFF7B2BB504D0846A989FAF790FA16
:10AD980069892046FAF78CFA0125FFF7A7BB0B68EB
:10ADA8004A4D591C1422216005F178061A7028783A
:10ADB80018F0F8F80746687918F0F4F823683A7A32
:10ADC800591C21601A7023682A79591C21601A704D
:10ADD8002368027A0635591CB54221601A70E6D1FB
:10ADE800FFF783BB0B683A4A591C127821601A7026
:10ADF8002368FF22591C216001251A70FFF776BBD2
:10AE0800344D08462988FAF753FA69882046FAF734
:10AE18004FFAA9882046FAF74BFA0125FFF766BBD7
:10AE28002D4D05F16006A9882046FAF741FAE98810
:10AE38002046FAF73DFA29892046FAF739FA2368B5
:10AE4800AA7A591C21601A702368EA7A591C216071
:10AE58001A7055F80C1B2046FAF712FAAE42E2D1E6
:10AE6800FFF743BB0A681D4B1A491878551C256023
:10AE7800107022685878551C2560107022689B78DD
:10AE8800501C206013702046C988FAF711FA012572
:10AE9800FFF72CBB0B680C4A11499078114A5D1CCE
:10AEA8002560187023684979581C20601970236838
:10AEB800D278591C216001251A70FFF717BB00BF13
:10AEC8003C130020305A0020641C0020486E0020EB
:10AED8005E6600208C5F00206C600020846A002081
:10AEE800482400208C6A002000212046FAF7E0F967
:10AEF80000212046FAF7DCF900212046FAF7D8F9B4
:10AF08002368964D00265A1C22601E7023682A6802
:10AF1800591C92F8462021601A7023682A68591C27
:10AF280092F8472021601A7023685A1C22601E700C
:10AF380023685A1C22601E7023685A1C22601E70E7
:10AF480023685A1C22601E702B682046198FFAF756
:10AF5800AFF92B682046D98EFAF7AAF92A68236830
:10AF680092F82D20591C21601A7023685A1C2260FF
:10AF78001E702B682046598EFAF79AF92B682046DE
:10AF8800998EFAF795F931462046FAF791F92A6829
:10AF9800236892F85120591C21601A7023685A1CA2
:10AFA80022601E7023685A1C22601E7023685A1C77
:10AFB80022601E7023685A1C22601E7023682A684B
:10AFC800591C92F84F2021601A7023682A68591C6E
:10AFD80092F8562021601A702B6820469989FAF752
:10AFE80067F92B682046598AFAF762F92B682046D8
:10AFF800198BFAF75DF92A68236892F83020591CF2
:10B0080021601A702A68236892F86E20591C216002
:10B018001A702A68236892F86F20591C21601A70E8
:10B028002A68236892F87020591C21601A702A68CF
:10B03800236892F87120591C21601A702A682368C5
:10B0480092F87220591C21601A702B6893F86B20B3
:10B058002368591C21601A702A68236892F86C20AA
:10B06800591C216001251A70FFF740BA0B683C4A49
:10B07800591CD27B216001251A70FFF737BA394F66
:10B088003B78002B3FF431AA374E002536F9021BD6
:10B09800204689B2FAF70CF93B780135AB42F5DC6A
:10B0A800FFF723BADFF8D8A0DFF8D8B02F4E304F1B
:10B0B8009FED308ADFF8D080DFED2F8ADFF8CC9063
:10B0C8000AF1C0050EE0FCEEE77A17EE903A99B265
:10B0D80020460AF1180AFAF7EBF8AA450BF1040B17
:10B0E8003FF403AA9AF811100029F1D03378DBED68
:10B0F800007A012BE7D13B68DB0440F12B81F5EEA8
:10B10800407AF1EE10FA00F04081F4EEC87AF1EEE0
:10B1180010FA00F13A81BDEEE77AF4EEE87AF1EE42
:10B1280010FA17EE103A00F26481A3F130026FF4BE
:10B13800F97303FB02F389FB03121A44D917C1EB15
:10B14800622101F2DB5189B2C2E7084610220B499D
:10B15800FAF77EF80125FFF7C9B900BF00150020EE
:10B16800181F002044680020CC1B0020C03C002091
:10B17800C03800200000404200E08244E86D002012
:10B188001839002034180020DB9B914121053483B5
:10B19800A14D0B682A68591CD27821601A702B6857
:10B1A80022689979531C2360002311702A6821684A
:10B1B8001A440133527A481C032B20600A70F5D1D7
:10B1C8002A682368127B591C21601A702A68236830
:10B1D8001278591C21601A702A6823685278591C01
:10B1E80021601A702B682046D989FAF761F82A6815
:10B1F8002368127A591C21601A702A6823685279C8
:10B20800591C21601A702A6823681279591C216018
:10B218001A702A682368D279591C21601A702A6822
:10B228002368127C591C21601A702A682368527C92
:10B23800591C216001251A70FFF758B90025FFF73E
:10B2480055B99AF8000000F00100FFF782BB4946A3
:10B258006846FDF787FBFFF77FBB38461EF04AFBC1
:10B26800FFF777BB23685A1C22601970298820468B
:10B27800FAF71EF82368EA78591C21601A702368C7
:10B288002A79591C21601A702368AA79591C2160EF
:10B298001A7023686A79591C21601A70FFF78AB9F5
:10B2A8005E4B5F4DB3F89C102046FAF701F85D4BF2
:10B2B80020461989F9F7FCFF5B4B19684B0103F02D
:10B2C8002002C1F340031343C1F3800243EA42035F
:10B2D800C1F3C00243EA8203C1F3401243EAC20346
:10B2E80001F0100119432046F9F7E2FF69460422EC
:10B2F8002046F9F7ADFF236829784C4A581C20608E
:10B30800197011886429A8BF64212046F9F7D0FF75
:10B31800962E5FD000212046F9F7CAFF2168B9F1BF
:10B32800190348BFA9F11203A3F3C4034A1C2260FE
:10B3380020461A460B7001A9F9F78AFF23683C4A90
:10B34800581C15212060197020461168F9F798FFDC
:10B35800FFF7CBB8F4EEC87AF1EE10FA37DBFDEE62
:10B36800E77A40F2E73217EE903A303B02FB03F3FC
:10B3780088FB0321DB17C3EB612101F2E93189B2B4
:10B38800A6E6B4EE008AFFF7FDBA40F2DC519FE66C
:10B39800FEF712FA0646FEF7ABF8236846F00206F7
:10B3A8005A1C226007461E7001882046F9F768FF7C
:10B3B800B9682046F9F764FFFDF792FF0146204679
:10B3C800F9F75EFFFFF792B8FF27FFF757B94FF479
:10B3D8007A717DE623680322591C21601A7023685C
:10B3E8006A78591C21601A7098E7B5EE008AFFF751
:10B3F800C9BAA3F5836240F2F31303FB02F389FB96
:10B4080003121A44D917C1EB622101F2DD5189B246
:10B418005EE61846FFF731B98C1E0020B4080020FC
:10B42800E41400201C0F00201C1800209A63002040
:10B43800A81B00208A4B1B7803B170472DE9F04FF9
:10B44800884D2DED028B2B6859058DB004D40DB0B5
:10B45800BDEC028BBDE8F08F834B1B7807460BB918
:10B4680025F0B6FE814B1B78012B44D0F7F746F93F
:10B478007F4B1E7800F57A70012E049067D07D4BC3
:10B488001B78002B40F0C1807B4D2A78002ADED142
:10B498007A4C94F82930012B40F2908094F82A00D5
:10B4A800774984F82A20C21801EB8202D269BAB11E
:10B4B800DFF8F481CDF814800CAEA8F1120946F833
:10B4C800209D48F2A50C152339463046A4F82CC017
:10B4D80084F82E309047002840F0738194F8293082
:10B4E800684A0133A2FB0312520802EB42029B1A7C
:10B4F80084F82930ABE7644B1B68002BB6D05F4C4F
:10B50800624A6369FB1A9342B0DDDFF8A091267E98
:10B51800D9F8008067610136F6B218F0020F267676
:10B5280040F0768218F0340F02D0B20700F053834F
:10B5380018F0080F40F0DB82730700F08F82282E86
:10B5480000F0F882524B5E201B6898478EE7514DF9
:10B558002868002893D04FF000098DF80890F7F775
:10B56800B7FB30B3DFF84881444C2868F7F7A8FBED
:10B5780083B27E2B00F0798198F800202968002A90
:10B5880040F00D8194F81DC0BCF1000F1BD01B2B9F
:10B59800627740F00B810846F7F79AFB002800F025
:10B5A8002C82286888F80060F7F792FB0028DCD125
:10B5B800002004AA02A909F07FF960E7304A02EBEB
:10B5C8008302D26973E77D2B00F0AB8294F82020C8
:10B5D80022B180F02003DBB284F820C0E28B94F81B
:10B5E8001CC01A44BCF1060F92B22AD804EB0C0E08
:10B5F80008460CF1010CE2838EF80C3084F81CC06C
:10B60800F7F766FB0028B0D1D2E7234C227832B195
:10B61800224B23491868F7F72FFB00232370DFF824
:10B62800948098F80040002C48D0DFF88CB0DBF804
:10B638006060002E40F02781104B88F800605F6240
:10B6480022E7D3B203EB1222FF2A88F80060E283D4
:10B6580040F0A5800846F7F73BFB1248A9E700BF72
:10B66800711B0020C038002078690020441F00208A
:10B67800511F00205C1F0020356700201C0F002090
:10B6880028510308ABAAAAAACC17002047E8010052
:10B6980038130020901E0020141F0020581F00207F
:10B6A800D41E0020280F00205D0F00201C18002049
:10B6B800640100205E1F0020681F0020894D2B7840
:10B6C800002B40F02581884C884D626A2978884B88
:10B6D80093FBF1F313449F42FFF4D6AE854A94F8E6
:10B6E8002830676212F8038018F0010F44D0DFF8A1
:10B6F80018929FED818AB9F9023007EE903AF8EE78
:10B70800E77A7E4B059367EE887A0CAEFDEEE77A12
:10B71800A3F13D0246F8202D17EE902A91B240F68B
:10B72800C80223F8402C1E2203F83E2C3046F9F7B5
:10B7380099FDB9F9003007EE903AF8EEE77A30460D
:10B7480067EE887AFDEEE77A17EE903A99B2F9F744
:10B7580089FDB9F9043007EE903AF8EEE77A3046F9
:10B7680067EE887AFDEEE77A17EE903A99B2F9F724
:10B7780079FD304609F068FB18F0020F40F07C8232
:10B7880018F0040F40F0FB8194F828302978013331
:10B7980093FBF1F201FB123384F8283074E6084673
:10B7A800F7F796FA00287FF4E0AE01E70D2B7FF457
:10B7B800F8AE0846E283F7F78BFA00287FF4D5AE97
:10B7C800F6E6049B4B4540F29C82A8F1130003F176
:10B7D800FF3C002141F2210710F8012F81EA0222E3
:10B7E80012B293B2002AACBF5B0087EA43039BB254
:10B7F8001A0454BF5B0087EA43039BB2190454BF81
:10B808005B0087EA43039BB21A0454BF5B0087EAD4
:10B8180043039BB2190454BF5B0087EA43039BB2FE
:10B828001A0454BF5B0087EA43039BB2190454BF50
:10B838005B0087EA43039BB21A0454BF5B0087EAA4
:10B848004303844599B2C7D13046F9F731FD2C49F5
:10B85800049E2C48761A152EA8BF1526324627F0C6
:10B868008CFE94F829302E703AE628688DF80890F6
:10B8780084F81C90667788F80090F7F729FA002872
:10B888007FF473AE94E60024DFF880A026464FF0DC
:10B8980050090BE01C44EFF3118389F31288DBF89D
:10B8A8006020944216DADBB283F311881BF8045047
:10B8B800601C29465844002208F0F8FE6B1C00283A
:10B8C800E8D051463A2008F053FE01350643F6B257
:10B8D8002C44E0E70022DBB2CBF8602083F3118828
:10B8E800AAE600BF5D1F00201C0F0020641F002077
:10B8F800A0860100601F002058A08B41D41E0020A4
:10B90800480F0020206700204C140020854E0108B5
:10B91800C24EC34B0093A6F13F014FF0C808CDE9D2
:10B92800021606F8408CBF4BBF4AC04904A8FCF772
:10B93800F3FF029E731C02933470029B2922591C48
:10B9480002911A70029BEA22591C02911A70029BFA
:10B958005A1C029204A883F8008026F0B5FF00F173
:10B96800010804A94246029827F007FE029A02EB52
:10B9780008030133029302F80840029B5A1C029202
:10B988001C70029B5A1C02921C70029B5A1C029249
:10B998001C70029B5A1C02921C70029B5A1C029239
:10B9A8001C70029B5A1C02921C70029B5A1C029229
:10B9B8001C70029B5A1C02921C70029B5A1C029219
:10B9C8001C70029B5A1C02921C70029B5A1C029209
:10B9D8001C70029B5A1C02921C70029B012299182F
:10B9E8000CA802911A7050F8283D9B1B337009F07F
:10B9F8002BFA8F4B2C705F6246E528688DF808603B
:10BA080088F80060F7F764F900287FF4AEADCFE559
:10BA1800702009F053FA00283FF484ADDFF854820F
:10BA28002426A8F12C0AF8EC017A9AED007A67EE40
:10BA3800877A3046FDEEE77A013617EE903AC3EB87
:10BA4800431103EB8103D90009B2F6B209F0E4F916
:10BA5800272EE8D1267ED9F8008063E5754B764914
:10BA68009B6A323381FB0321DB17C3EB611109B2F7
:10BA7800022009F0D1F9714B1B78DE0700F16C81C7
:10BA88006F4D704BA989A3FB01318908032009F088
:10BA9800C3F96B7A002B40F03681D9F800301807CB
:10BAA80023D504A9684809F07BF9BDF910101320C3
:10BAB80009F0B2F9BDF912101B2009F0ADF94E21B9
:10BAC800232009F0A9F904A95F4809F069F9BDF92B
:10BAD8001010122009F0A0F9BDF912101A2009F06F
:10BAE8009BF94521222009F097F9267E27E54FF496
:10BAF800007009F0E3F900283FF41EAD16F00308C2
:10BB08007FF41AAD514A0A23B2F9041091FBF3F1FC
:10BB1800142009F081F941461C2009F07DF9267EA0
:10BB28000AE5084684F82060F7F7D2F800287FF481
:10BB38001CAD3DE5464A474B1568474EA3FB052318
:10BB48009B0BA6FB03214909C1EB0111A3EB810360
:10BB5800190209B200231720237609F05DF93F4B3B
:10BB6800A3FB05239B09A6FB03125209C2EB021291
:10BB7800A3EB820319B2182009F04EF9E2E42F4A28
:10BB8800264B92F800900593A3F14006C821212284
:10BB9800A3F13D0A19F0010923F8401CB270CDF851
:10BBA80010A000F0FE802E4A1288510540F108814D
:10BBB8002C4A106843F83D0CF31D0493581C04905C
:10BBC80000210CA81970284A50F8203D9B1A737060
:10BBD80009F03AF9D8E54FF4806009F06FF90028C8
:10BBE8003FF4A6AC214A224BD2F8008062694FF09C
:10BBF800640A9A4298BF4FF00008102098FBFAF6A2
:10BC080031B209F009F90AFB168109B2212009F0BD
:10BC180003F9267ED9F800808AE400BFD41E0020EC
:10BC2800EB14002038A2030840A203084CA2030822
:10BC38001C0F0020B86C00201F85EB51994900208B
:10BC480070130020CDCCCCCC809698004C140020EA
:10BC5800C42D002073B2E74589888888D34D6210C7
:10BC68001018002058A20308951E00202018002054
:10BC78003F4B4C00CC1C0020B24BB34AB349D27A9C
:10BC8800059340F6C82023F8400C082003F83E0C22
:10BC98003D3B04930B88002A75D1AD490533A1FBC0
:10BCA800033104AEC9083046F9F7DCFADFF8A89288
:10BCB800A849D9F8003081FB0321DB17C3EBA101A8
:10BCC80089B23046F9F7CEFA12F0F2FFD9F80890A7
:10BCD800049B4FEA1942591C04911A70049B4FEABD
:10BCE8001922591C04911A70049B5A1C049283F857
:10BCF8000090049B5A1C04921870304609F0A4F86E
:10BD08003EE50021A0E5012009F0D8F8002864D11B
:10BD1800AB7A002B3FF4C1AE022009F0CFF840B156
:10BD28008D4A0A23116891FBF3F1282009B209F022
:10BD380073F8042009F0C2F800283FF4AEAEAB89CE
:10BD4800002B40F0D480844B996881F3100109B22C
:10BD5800042009F061F8A0E61DF0C4FF7F4B9FEDB9
:10BD6800807AD3ED037A67EE877AFCEEE77A17EEEE
:10BD7800903A99B220B92B6813F0100F18BF002120
:10BD880009B2784D82E67849714A097893FBF1F156
:10BD98000531A2FB013104AEC9083046F9F762FA51
:10BDA80084E7724A1268002A5AD0714A106843F828
:10BDB8003D0CF31D591C2A221A7004910B46FDE60E
:10BDC800110540F198806B4A118823F83D1C927840
:10BDD8008AF80220B31D0493F0E6634EDFF86C8105
:10BDE8003278002A5ED11346110189B241EA032153
:10BDF800C3F30323194309B20620628309F00CF840
:10BE08005148618B90F808C0B8F800303278013199
:10BE1800BCF1010F03F105034FF00A06618393FBA0
:10BE2800F6F399B22BD0C37A01EB81018EB213B12C
:10BE38000AB196FBF2F64FF0640A3A20B6FBFAF81C
:10BE48000FFA88F108F0E8FF0AFB186189B20A23A3
:10BE580005313B2091FBF3F109B208F0DDFF57E70C
:10BE6800454A1288500500F19780100560D4D00526
:10BE780010D5424A106843F83D0CF31D9AE7C07A82
:10BE880018B112B193FBF2F399B209B2392008F054
:10BE9800C3FF3DE7D10715D5394A106843F83D0C73
:10BEA800F31D87E7618BB8F8003091FBF2F04FF093
:10BEB800640C02FB10100CFB0323510082B2B3FB8D
:10BEC800F1F391E7910728D5DFF8C8B0584626F076
:10BED800FBFC5946804602462A4827F04EFB0AEBEF
:10BEE80008030493B9F1000F3FF464AF66E612F05B
:10BEF800DFFE01B22CE7D10506D5204A106843F8C9
:10BF08003D0CF31D049359E6D007DBD51C4A106895
:10BF180043F83D0CF31D049350E61B4A1B4B92F863
:10BF280000B01B4ABBF1000F14BF9B469346CDE7F8
:10BF3800104A1188927823F83D1C8AF80220B31D14
:10BF480038E700BFD41E0020E4170020081800209E
:10BF5800CDCCCCCC67666666D0170020C86D0020B3
:10BF6800CDCC4C3E701300200E180020A81B0020DA
:10BF780060A2030868A20308101800206CA2030836
:10BF880074A20308971E00201218002028A2030894
:10BF98002CA2030834A20308024A106843F83D0C97
:10BFA800F31D07E758A203082DE9F0415E4C636CC6
:10BFB80046F2A712C31A93422DED028B03D8BDECAB
:10BFC800028BBDE8F081594B60641B6813F00403D1
:10BFD8002CD11846564A94F85410127812F00102DF
:10BFE80017D0F1B90125C4E916010A46084684F8B4
:10BFF80054500BB14F4B18604F4B1B780E2BDED1B2
:10C00800BDEC028B4D4B1E2158809A801980BDE8EB
:10C01800F08131B1D4E9165184F85420401B4A42CA
:10C02800E7E7D4E91612401A5242E2E7DFF82C811A
:10C03800434E98F806303788A56C013BB5FBF3F5FD
:10C048009FB3404A9FED400A5368002B1946B8BF7A
:10C05800D91DA3EBE1031D44002D2B46B8BFEB1DF2
:10C06800DB1007EE903AF8EEE77A556027EE800A83
:10C07800F9F728F9DFED357A20EE270AF9F768F99C
:10C08800F7EE007A77EEC07A9FED310A236D67EEFE
:10C09800807A9D42FDEEE77AC4ED137A3FD0013FE6
:10C0A800002337802565184694E707EE905A9FEDE0
:10C0B800260A284DF8EE677AB7EE008A27EE800A3E
:10C0C800F9F700F9DFED217A20EE270AF9F740F9B0
:10C0D800DFED1F7A38EE400A20EE270A27F0F2F942
:10C0E800B8F80830DFED1C6A07EE103AE36CC01AA6
:10C0F800B8EEC77A07EE900AA7EE668AB8EEE70AA6
:10C10800D5ED097AF8EEE77A20EE080A67EEA67A06
:10C11800A7EE870A27F0D6F9012368625AE70022BA
:10C1280013463280104655E71C0F00201C180020CB
:10C1380099490020201800201C4A0020204A00208D
:10C14800206100206401002008942537B1DC423EBC
:10C15800D048874AB86C00206F12833A48240020E0
:10C168002DE9F8432E4B1B685B0701D4BDE8F88323
:10C178002C4C2D4D94F86090B9F1010F3CD1EB692E
:10C18800284698472B69284698472B6A04F164018A
:10C1980004F168009847254AA66C9179D4E91B8375
:10C1A800D4E9192008F10107AA625A1C8F4208BF76
:10C1B8000027032AE8622AD01D49226794F87420D0
:10C1C80041F823004ABB04EB880804EB8703C8F84E
:10C1D80078009A6FAB89E766B61A30440022A064EB
:10C1E80084F86020002BC1D0124A642B1268B8BFB3
:10C1F80064231361BDE8F8836B6928469847AB69E7
:10C20800284698470122EB8984F86020EAE7084A23
:10C2180084F874900023906023670DF053FED2E7F2
:10C228001C1800201C0F0020B86C00204824002097
:10C23800BC3A00204870002008B50E4B1978012937
:10C2480013D00DD3022902D10020F6F74FFDF6F7DF
:10C2580055FA094B00F5F42000F59070186008BDF8
:10C2680000210846F7F7BAFCF1E70020F7F7B6FC1B
:10C27800EDE700BF9C630020A063002010B50446D2
:10C288002046F6F719FD00B110BD0A20F6F754FB59
:10C29800F6E710B5084A002352F83310884202EB3B
:10C2A800C30403D00133052BF6D110BD0021C162B0
:10C2B800A18042F83310F8E7E83B00202DE9F04F61
:10C2C80091B092469DF86C509DF87040964A039143
:10C2D80007469B464FF000084FEAC80302931344F1
:10C2E80093F90610B94230D008F10108B8F1050FEA
:10C2F800F2D14FF0000912E11F2FFAD1CDE9005415
:10C308001A9B5A465146012012F07CF88146F9E002
:10C31800506820EA0101516073E020211162116820
:10C3280041F020011160B2E0D9F854100A6842F0D7
:10C3380080020A60E0E0CDE900541A9B5A46514653
:10C34800304612F05FF88146DCE09E88002ED0D19E
:10C358001E2FF0D0D0DC022FCBD823462A461A99BC
:10C36800F8B2FDF719FB8146002800F0D8800122B9
:10C378001A9B80F8582005714471C0E90766C0E926
:10C388000966C0E90BAB8360406D026814F0040FC6
:10C3980022F0010202600CBF00224FF48052069284
:10C3A8002203240204F4806402F40052089415F075
:10C3B8000104079216BF04220994099215F0020598
:10C3C80005930A9603D0099A42F00802099205A932
:10C3D8000FF084FB99F8042099F8056012F0020F19
:10C3E8000CBF00214FF4003106F00100D30748BF0D
:10C3F80041F48031D9F85420002889D0506801438D
:10C408005160916830074CBF41F0080121F00801E4
:10C418009160116841F001011160002C37D0D9F802
:10C42800381000293FF479AF05A80EF0C3FAD9F8FF
:10C43800502005924FF4805300228021CDE90E321E
:10C4480009920B920A910C92D9F80C1007922022AB
:10C458000D92D9F83800D9F814200692ADF82010BA
:10C468000EF0D6FA05A9D9F838000EF0B1FAD9F8C5
:10C478003820D9F85400116841F001011160816831
:10C4880041F040018160526892B2C9F84820002DFD
:10C4980032D0D9F83C20002A3FF446AF05A80EF068
:10C4A80089FAD9F84C20059200244FF48052CDE93E
:10C4B8000E2480220A92D9F81020ADF82020D9F84D
:10C4C8003C000994102207920B940C940D940EF0E2
:10C4D8009FFA05A9D9F83C000EF07AFAD9F83C2061
:10C4E800116841F002011160D9F854105460546089
:10C4F8008A6842F080028A60D9F854100A6842F0CB
:10C5080001020A60B9F1000F09D0029B89F8347062
:10C518001A46054B039943F838901A4491804846C7
:10C5280011B0BDE8F08F00BFE83B002038B10388A8
:10C5380013EA010003D08B420CBF01200220704790
:10C5480070B50B4C0B4D0023052BDAB202D12370CA
:10C5580000200AE05E1C05EBC30135F833300132D8
:10C568001842D2B202D00846227070BD3346EBE7BB
:10C57800F0510020BC3B002018280AD800EB4000EE
:10C58800054B13F8200028B10123013803FA00F005
:10C5980070470020704700BF4470030810B50020A2
:10C5A800F7F7F2FA064A074B002414701C70FFF7DD
:10C5B80043FE0549054A064B0C6014801C6010BDFB
:10C5C800731C00209C63002094630020906300206B
:10C5D8001C610020002830D0194B1B6813F400336D
:10C5E80024D101229042174908D00133192B03EBBB
:10C5F800430223D011F822209042F6D130B4124CD5
:10C60800104A2068590030B14578C81802EB8000FC
:10C618004078A84208D20B440C480D4902EB83022B
:10C628000023226003800B6030BC7047094B1B78E5
:10C63800032B02D001220023D4E7AFE7704700BFE5
:10C6480010610020447003081C61002090630020E2
:10C6580094630020131800202DE9F84306460B20A8
:10C668001DF048F9E8B9474D2C68C4B1464F3B68FE
:10C67800B34214D8DFF8349199F800305BB3DFF88F
:10C6880030816268B8F80030D25C72B9002242F298
:10C698001071013301FB0266A8F800303E60BDE866
:10C6A800F8830A20FFF796FFDDE70020F7F76CFA1A
:10C6B800364A0023137089F80030FFF7BDFD2A6859
:10C6C800B8F800305268D25CFE2A56D10023A8F888
:10C6D8000030BDE8F8831BF01DFFD0B923780A2B82
:10C6E80040D0022B15D12A4A93689B0711D4294BB5
:10C6F80029491B68F31A8B420BD9284B1B6843B98D
:10C7080027482849066012790978FF2011F012FAA3
:10C718002C68DFF89C806268B8F80030D25C002A88
:10C72800B4D023781A4A013B0124126804FA03F3AF
:10C7380013421CD0154B01221A70FFF77DFDB8F883
:10C7480000302A68002BBDD11178481F012801D973
:10C758001829B7D1F5F7D2FF134B2A681860B8F833
:10C768000030AFE70A4A93689905C0D5D1E720465B
:10C77800F7F70AFA89F80040DCE7FF2A87D1BDE815
:10C78800F8430BE71C610020946300209C630020A1
:10C7980010610020544C0020804F1200581C0020CB
:10C7A8005C1C00207D120020786C0020731C002087
:10C7B8009063002040004028094A30B4A8BF4020B8
:10C7C800002302251424D5540233D118834201F8DA
:10C7D800014CF8D3FF21D1540E2030BCFAE600BF3B
:10C7E8001463002010B5094C238823EA00009842FE
:10C7F800208009D0064B41F20241FF2219809A702D
:10C808000E20FFF7E7FE2388184610BD10180020F9
:10C818001463002010B5094C2388184398422080DF
:10C8280009D0074B41F20241FF2219809A700E206D
:10C83800FFF7D0FE2388184610BD00BF101800204F
:10C8480014630020024A136818431060704700BF41
:10C85800A81B00202DE9F04FE04D2DED068B2B781D
:10C8680091B0044643B1DFF8CCA3DAF80C30504657
:10C87800984780F001002870D94B1A78002A00F0F8
:10C888004882D849D848D94E0D7804F5EC425F3231
:10C898000260002032681870002D00F0F581944283
:10C8A80001D9013D0D7020461DF01AFC002800F04A
:10C8B8003082CF4DCF4AD5F8C031C5F8C041E41A0F
:10C8C80047F230539C421668CB48CC49B6F80EC0A4
:10C8D800CB4FA8BF1C46B4F57A7FB0F90630B8BF75
:10C8E8004FF47A740C8063454FF001043C7080F279
:10C8F8002882C44A4FF07E511160C34AC349B0F937
:10C9080000804E8A92F9044092F800E092F801C043
:10C91800002CA8EB060214BF01274FF0FF37002AAE
:10C92800B8BF5242B2F5FA7FA8BF4FF4FA72724507
:10C93800C6BFA2EB0E0207EE902ADFEDB57AB54C22
:10C94800C8BFF8EEE77A4645B0F90280C4ED007A30
:10C95800A8EB0602C4BFF1EE677AC4ED007A002A9C
:10C96800B8BF5242B2F5FA7FA8BF4FF4FA729645A3
:10C97800BABFA2EB0E0207EE902ADFEDA57AB0F956
:10C988000400B8BFF8EEE77AB045A0EB0602C4EDA4
:10C99800017ABCBFF1EE677AC4ED017A002AB8BF0C
:10C9A8005242B2F5FA7FA8BF4FF4FA72944580F26A
:10C9B800E181A2EB0C0C07FB0CFC07EE90CAF8EE29
:10C9C800E77A954AC4ED027A86421068C4BFF1EE50
:10C9D800677AC4ED027A10F4805000F09F81B3F5B5
:10C9E800FA6FA8BF4FF4FA63B3F57A7FB8BF4FF474
:10C9F8007A73A3F57A71894B1A78002A40F09781E7
:10CA0800874FDFF834C287FB0123CA17C2EB6313D1
:10CA18005A1C6FF0630E3CF912203CF913C00EFB50
:10CA28000313A2EB0C0203FB02F387FB0327DB17BC
:10CA3800C3EB671363441BB207EE903AB8EEE78A7C
:10CA480084ED038A002840F0B581764B1B885A068E
:10CA580040F10F8140F603027349D4ED011A91EDBC
:10CA6800018AD1ED033A91ED029AD1ED005A94ED85
:10CA7800002A13406D4A08BFD4ED022A92ED014AFC
:10CA880092ED026AD2ED006A92ED030A18BFDFED5B
:10CA9800602A674A38EE635A74EE460A76EE807A60
:10CAA80065EE200A75EEC94A35EE89AA76EEC09A77
:10CAB80064EEA74AB0EE603AAAEE293AB0EE645A9C
:10CAC80038EE237A74EE067AAAEE295AA7EE273AA8
:10CAD800A7EE675AB0EE601A97EE271A33EE243A9B
:10CAE800F6EE008A75EE88AA28EEC33A35EE605A4B
:10CAF80076EE840AB0EE417AAAEE691AAAEEA03A56
:10CB080077EE647A76EE400A73EEC9AA25EE285AC3
:10CB1800EAEE297AAAEEA05A71EE244A36EEC44A01
:10CB280063EE036A73EE893A64EEA84A75EEC85A52
:10CB380036EE006A67EEA87AB0EE667AE3EE844ACB
:10CB480095EE057AE5EE056AE5EE867AB1EE648A39
:10CB5800F0EE665AF0EE476AB1EE674AE8EE246AEC
:10CB680063EE270A67EEA43AE4EE275AB1EE450AC7
:10CB7800B0EE606AB0EE631AA4EE277A23EE244A78
:10CB8800E7EEA76AA5EE246AA0EE031AE8EE245A97
:10CB9800B0EE448A31EEA19AE0EE240AA5EE278A87
:10CBA80066EEA16A72EE028AE5EE033A61EE211A98
:10CBB80026EE096AA4EEA47AA0EE274AA2EE256A18
:10CBC800E8EEA06AE2EE081A73EEA33A27EE227A9C
:10CBD80034EE044AF0EE005A30E000BF5C680020F2
:10CBE80064680020FC6D002060680020F86D00205B
:10CBF8001C0F00208C1E0020CC1B00200A52002095
:10CC080008520020145D0020846A0020181F0020AC
:10CC180000000000C86D0020C0380020904B0020A4
:10CC28001F85EB511018002074080020840800208C
:10CC38009408002044680020CC600020E2EEA36A3B
:10CC4800A4EE226AA1EEA57AC5ED726AC4ED016A66
:10CC580085ED716A84ED006A85ED737A82ED005A7C
:10CC680082ED013AC2ED027AC2ED034A002B00F0D0
:10CC7800DA81684B1B78DB077FD411B0BDEC068BDB
:10CC8800BDE8F04F1FF096BD94427FF60CAE624BA4
:10CC98001E78002E00F0E280DFF8B8A1DFF8B0B10E
:10CCA800DFF8A881DFF8B091574628E018F805109A
:10CCB8009847032D03462ADCC8B109EB850339F8E8
:10CCC80025105A88401A4FF47A7303FB00F0521A61
:10CCD80040F6CA0390FBF2F000F57A709842A8BFBC
:10CCE800184640F2EE239842B8BF184600B24A4BA5
:10CCF8002BF8020B1E780135B54280F2AF80072D64
:10CD08003846DAF80430D1DDE9B29847034618B25C
:10CD1800EDE711B0BDEC068BBDE8F08F8A8A93422F
:10CD280038DA3E4B1A780146002A3FF469AE5B7840
:10CD38003B4A01FB03F382FB0321DB17C3EB6111C1
:10CD48005EE6B3F5FA6F327B9FED367ABFBFA3EB91
:10CD58000C014A43CCF5FA6192FBF1F2C2F164028C
:10CD680007EE902AF8EEE77A2F4A67EE877AC2ED47
:10CD7800007AC2E5DFED2D7A23E62D4A2D4B117896
:10CD8800186801F0010111B0BDEC068BBDE8F04F49
:10CD9800F6F7F2BEB3F5FA6FD4BFC2EB0303C2F5E0
:10CDA800FA634FF47A71C2F5FA6201FB03F3B3FB3D
:10CDB800F2F120E6204BDB78002B7FF446AE1F4BC8
:10CDC8001F481F7B1521FBF7DDFD002F40F0338145
:10CDD80000283FF43AAEDFED1B7A1B4978EE677AFC
:10CDE800C6F5FA63FDEEE77A1AB217EE903A1BB26F
:10CDF8001B0381FB0301DB17C3EBA11302FB03F346
:10CE080043F30F33334407EE903AF8EEE77AC4ED74
:10CE1800037A1AE6994900202C6F0020904B0020D5
:10CE28001F85EB510AD7233C145D00200000000049
:10CE38008C2D0020902D00207C1700208C5F002076
:10CE48003C6A002000007A44D34D6210181F00206D
:10CE58005410002044680020406F0020B94B1A7815
:10CE6800B94BD3F80090002A40F0E0801346B74948
:10CE7800097804912A2904D1B548B6490078488030
:10CE88000A80B54A01251570002E00F0AB81B34A1F
:10CE9800B34F10780390B348DFF800C3C18B0191FA
:10CEA800018C0291418A03980A91397B0D910746BA
:10CEB800ACFB07714908079201EB4101AA4ADFF868
:10CEC800E0A21268DFF8B4B20B95411AC8B206F1B5
:10CED800FF380590CDE90864400042F20101069050
:10CEE800B8F1030F02F480500C9002EA0102A8BFC7
:10CEF8004FF003080025002B00F0DD809B490198C6
:10CF080031F8151081424FEA4507C0F0D4800298E5
:10CF1800814200F2D08009F596704AF8250009B2DE
:10CF2800002A40F0E8802BF8071001354545E2DD7E
:10CF3800DDE90864AE4227DD8D4FDFF840B2069484
:10CF480005EB450107EB4107002B00F09980874965
:10CF5800019831F8151088424FEA450800F2908090
:10CF680002988842C0F08C8009F596704AF825002E
:10CF780009B2002A40F016812BF808100135AE429C
:10CF880007F10607E0D1069C734B1B78002B40F095
:10CF98002B816F4B012204201A70FFF753FC754A4E
:10CFA800694BD2E901101B68D3601B1A8B4202D966
:10CFB800002382F82130704B1E78644B1B78049351
:10CFC800002E00F02881664A674B117B1B68654A72
:10CFD80003F48053B2F81E80578A002900F0468176
:10CFE8006649674D83B1ACE1022A40F02781427857
:10CFF80002EB820202EB820202F2EE2201339E422F
:10D0080021F8022B00F0078115F8132005EB4300E7
:10D01800002AE9D1DAB2022A40F26081032A40F0FC
:10D028000D814246EAE784ED027A22E6484B1B78F6
:10D0380083F001031BE7DFED537A534A38EE678A22
:10D04800BDEEC88A18EE103A1BB21B0382FB03120E
:10D05800DB17C3EBA213002800F02A81C6F57A7209
:10D0680012B203FB02F343F30F33334407EE903A53
:10D07800464BF8EEE77A0122C4ED037A1A70E4E42D
:10D088005AF82510A9EB01010029FFF677AF3C48B3
:10D0980010F815104FEA45084044002900F0D080E8
:10D0A800022940F0C880417801EB810101EB810140
:10D0B80001F2EE215CE75AF82510A9EB01010029DD
:10D0C800FFF633AF2E4810F815106F0038440029CA
:10D0D80000F0C180022940F0AB80417801EB81016A
:10D0E80001EB810101F2EE211B4C0020207009B2F6
:10D0F800002A3FF418AF1E48254C069E94F8A4E178
:10D1080007EB050C00EB4C008153BEF1000F06D174
:10D11800039E022E7FF607AF0B9984F8A41141886D
:10D12800B0F804E0124830F81C007144014408B219
:10D13800184981FB0041184CA1EBE071E05309B29A
:10D14800F1E600BF28680020C42D00201C4A0020FA
:10D15800B0080020204A0020446A0020FD6D00200D
:10D168008C5F0020181F0020C038002054100020B9
:10D17800781000207C1700202C6F0020CC1B00208A
:10D18800746F002000007A44D34D62107052002062
:10D198001C0F002056555555C4100020ABAAAAAA4A
:10D1A800006E00208B48059C90F8A40127F8141005
:10D1B80038B9039C022C7FF6DFAE8648012180F83F
:10D1C800A4117988B7F800C0B8886144014408B24E
:10D1D800814981FB0041814CA1EBE07124F80800F2
:10D1E80009B2C9E67E4B07937E480621FBF7CAFBC6
:10D1F80000287FF4CEAE7C4A7C4BD1681B689360D4
:10D208005B1AC82B07D97A490B68012023F004035D
:10D218000B6082F82100049B2A2B03D1754A764BB8
:10D22800D288DA80079A137801331370FFF73BBB73
:10D238003BF8071058E73BF8081099E60A88DDE63E
:10D24800E9B2022948D90329F5D10C99002940F0FF
:10D258009C8001998CE6E9B202293BD90329E7D1E0
:10D268000C99002940F0A38001993DE7002B39D1A2
:10D278006049624D0DE0022A18D1427802EB820221
:10D2880002EB820202F2EE2201339E4221F8022BC7
:10D29800C1D015F8132005EB4300002AEBD1DAB210
:10D2A800022A1DD9032A01D14246EDE70A88EBE795
:10D2B800C6F5FA6212B203FB02F343F30F333344A9
:10D2C80007EE903A4E4BF8EEE77A1870C4ED037A01
:10D2D800FFF7BBBB0A9907E70A9949E63A468DE684
:10D2E8003A46D1E7DFF80CA1444DDFF8F8B089469B
:10D2F8000EE0022B22D1507800EB800000EB80007A
:10D3080000F2EE2009F10109B1452AF8020B82D09A
:10D3180015F8193005EB4902002BEAD15FFA89F3B9
:10D32800022B2ED9032B4FF01501584606D1FBF7D7
:10D3380029FB00280CBF38464046E3E7BAF800004E
:10D34800E0E700230EE0022A19D1427802EB8202BC
:10D3580002EB820202F2EE2201339E4221F8022BF6
:10D368003FF459AF15F8132005EB4300002AEAD122
:10D37800DAB2022A07D9032A01D14246ECE70A8821
:10D38800EAE73846BEE73A46E6E715211548CDE90B
:10D398000832FBF7F7FADDE9083200287FF459AFC5
:10D3A8000D99019800290A9918BF0146E0E5152151
:10D3B8000C48CDE90E32FBF7E5FADDE90E3200281C
:10D3C8007FF452AF0D99019800290A9918BF0146B8
:10D3D8008AE600BF1C0F002056555555C410002082
:10D3E800FD6D00203C6A00207C170020C42D002021
:10D3F800A81B0020CC1B0020204A0020746F0020AE
:10D4080070520020F8B56D4B6D4E6E486E4D01247C
:10D41800642200211C7026F0D4F86C4A6C49002361
:10D4280030460B60136011F0F5FD2146204611F0DF
:10D438003FFE2146062011F03BFE6C7A654B211C0D
:10D448001A8D654B93FBF2F318BF0121642BB8BF0B
:10D4580064230820C6F8903111F02AFEAF7A391CEF
:10D468004FF0090018BF012111F022FEAB7B002B01
:10D4780064D05A4D002C6BD1391C18BF0121584C6F
:10D488000A2011F015FE2368DF0772D4980700F10F
:10D498008480D9067AD40121052011F009FE0021E3
:10D4A800072011F005FE01210B2011F001FE216873
:10D4B8000C20C1F3C00111F0FBFD21680D20C1F360
:10D4C800800111F0F5FD23685A0756BF296801212C
:10D4D800C1F3C0110F2011F0EBFD29684B0539D4B9
:10D4E800C1F30041112011F0E3FD296811F48021F6
:10D4F80004D03C4B1968003118BF0121122011F0EB
:10D50800D7FD29681320C1F3C06111F0D1FD0121B5
:10D51800142011F0CDFD0121152011F0C9FD0121C4
:10D52800162011F0C5FD304B196800314FF0170077
:10D5380018BF0121BDE8F84011F0BABDEB7B274DBB
:10D54800002B97D1296811F4802198D0002C93D012
:10D55800012194E70121102011F0AAFD234B29682D
:10D568001B7A083B012B9CBF4FF4FA63C6F81034B2
:10D57800B6E71F4B1B68642BB8BF64230121022048
:10D58800C6F8903011F094FD23687FE729680E20D3
:10D59800C1F3402111F08CFD7DE70121032011F03A
:10D5A80087FD144B9B6A642BB8BF642301210420B8
:10D5B800C6F8D03011F07CFD23686AE7C851002016
:10D5C800B40800206451002070130020DC510020B2
:10D5D80060510020BC3B002040420F00C0380020B2
:10D5E8001C18002058180020D81F0020181F0020E1
:10D5F80020320020A01C002008B501210020F6F7E9
:10D60800EDFA01210846F6F7E9FA01210220F6F7BA
:10D61800E5FA114B1B7803F00503052B18D0002100
:10D628000846F6F7DBFA00210120F6F7D7FA0021C1
:10D638000220F6F7D3FA3220F5F77EF90020F5F745
:10D6480055FB0120F5F752FB0220F5F74FFBF2E7F7
:10D658001AF064FBE3E700BF285800202DE9F04FDB
:10D668008DB0F7F7D7FADFF87891584FDFF8748163
:10D6780024F0D6FC564A574B128DADF80620A3EB82
:10D68800090300934FF0030A0026CDE90866CDE9A7
:10D698000A66009BCDF818900793D8F810301B063F
:10D6A80006D54D4BC8F8043003F18833C8F8043068
:10D6B80001238DF82C303423C8F80C300222BDF831
:10D6C8000630ADF8083002A906A8F7F77DFD02225A
:10D6D80002A94FF6FF70F8F7FFF9404BBB428346AB
:10D6E80029D21C46658823888DF81560C5F30B057B
:10D6F800C3F30B00A91D1B0B0622ADF81010ADF8E3
:10D70800120004A906A88DF81430F7F75DFD5846F5
:10D71800062204A9F8F7E0F9616883462A4606A8B4
:10D72800F7F752FD616858462A46F8F7D5F91434D8
:10D73800BC428346D6D3022203A906A8ADF80C60E2
:10D74800F7F742FD022203A95846F8F7C5F940BA8F
:10D75800C343022204A906A8ADF81030F7F734FD38
:10D76800099820BB0A989DF82C305BB990B1BAF1A2
:10D77800010A8AD10520F4F72DFD24F0E7FB0DB04E
:10D78800BDE8F08FD8F8103043F08003C8F81030A7
:10D798000028ECD199F80030AC2BEBD199F8013086
:10D7A800BE2BE7D1F8F7B2F90028E6D1E2E708ABDB
:10D7B800C0F104020021184425F003FF089906A8C7
:10D7C800F7F7A8FCCDE90960CDE700BF20BE030844
:10D7D80028510308000004082301674570B90308AD
:10D7E80000F00308002002402DE9F047D64C2DED4B
:10D7F800028BA36820469847002800F0D180D34BBD
:10D808001B780122042B84F8382000F0CD80B4F96D
:10D818001A3006EE903AB4F91C3007EE103AB4F913
:10D828001E3007EE903AF8EEE66AB8EEC77AF8EEE0
:10D83800E77AC4ED0B6A84ED0C7AC4ED0D7AC44B1B
:10D848001B88002B60D0C34B94ED0B2AD4ED0C2A17
:10D8580094ED0D3A93ED008AD3ED054A93ED090A4C
:10D86800D3ED0E3AD3ED120A93ED174A93ED011A50
:10D8780093ED065AD3ED0A1A93ED0F6AD3ED137A96
:10D8880093ED187AD3ED045AD3ED0D6AE8EE024A07
:10D89800E0EE223AA3EE204AA1EE025AA1EEA26AD5
:10D8A800A3EE277A93ED038AD3ED167A93ED020A55
:10D8B800D3ED0C0A93ED0B1AD3ED151AC4ED0B4AF0
:10D8C80065EEE45AA8EE645A66EEE36AD3ED144AAC
:10D8D80083ED055A67EEC47AE0EE025AA0EEE36AD9
:10D8E800E1EE226AA4EE617AE3EE247AC3ED065AE9
:10D8F800C4ED0C3A83ED0E6AC3ED0F6A83ED177A17
:10D90800C3ED187A84ED0D4A934F94F8221093488A
:10D91800934E23F073FC3B88D6F8D051002B40F08F
:10D928009880904B1B685A075BD4B5F9003094ED8A
:10D938000C6A94ED0D7A94ED0B5A8B4905EE903AEA
:10D94800B5F902300A6806EE903AB5F9043007EEE8
:10D95800903AF8EEE55A854BF8EEE66AF8EEE77A83
:10D96800D3ED003A93ED014AD3ED024A75EE655ABC
:10D9780076EE666A77EE677AC4ED0B5A34EE266A5D
:10D9880073EEA55A34EEA77A0132C3ED005AC4EDFE
:10D998000C6A83ED016AC4ED0D7A83ED027A0A60A0
:10D9A800BDEC028BBDE8F087B4F91A00B4F91C107D
:10D9B800B4F91E206E4B07EE900AF8EEE76A07EE00
:10D9C800901AB8EEE77A07EE902AF8EEE77AC4EDF7
:10D9D8000B6A188059809A8084ED0C7AC4ED0D7A10
:10D9E8002DE7644F3B88322B00F0CE80002B40F0AF
:10D9F8001A8161480378002B97D0604FD6F8F4312C
:10DA0800D6F8EC21D6F8F01187FB03ECDB17C3EB53
:10DA18002C13B4F818C0A3EB0C03AB8087FB02C32C
:10DA280087FB01C7C917C1EB2711D217544F69806B
:10DA3800C2EB2312002303702A807B81BB81FFF78E
:10DA48000DFEF7F7F9FA0120FEF7B4FED6F8D0512B
:10DA58006BE7B3F5C87F18BFD6ED757AD4ED0B6ABE
:10DA68000CBF9FED487AB8EEE77ADFED467A0023DF
:10DA7800C4ED0B7A2B803B88B7F8008037EE267A06
:10DA8800B3F5C87F18BFD6ED767ABDEEC77A18BF52
:10DA9800F8EEE77A17EE102A86ED757A94ED0C7A8F
:10DAA80077EE877A0021FDEEE77A0020B8F5C87F87
:10DAB800216317EE903A6880C6ED767A00F0AA8066
:10DAC800D6ED777A94ED0D7A6163F8EEE77AB8F1DE
:10DAD800010F77EE877AA880FDEEE77A17EE901AA5
:10DAE800C6ED777A2BD1DFF894C0B4F818E0C831C6
:10DAF8008CFB01A9C832C833C917C1EBE9118CFBEB
:10DB080002A98CFB03ACDB17C3EBEC13D217DFF8CD
:10DB180070C06B80A1EB0E01C2EBE912A9802A80CC
:10DB2800ACF80A00ACF80C00FFF798FDF7F784FA98
:10DB38004046FEF73FFEB7F80080D6F8D05108F10E
:10DB4800FF38A7F80080ECE6A01C00201C4A002043
:10DB5800DC680020E068002026610020CC1C002042
:10DB68001C0F0020C0380020EC5F0020F05F002070
:10DB7800204A002028610020246100201F85EB51E5
:10DB8800641C002000000000514B2A68D3F80A30BA
:10DB9800C6F8E8319FED4F7AB5F90430C6F8E021B0
:10DBA800A6F8E431DFED4B7AD4ED0B6AC4ED0B7ABD
:10DBB80000232B803B8837EE267A322B18BFD6ED10
:10DBC8007C7A3B88BDEEC77A18BFF8EEE77A86ED17
:10DBD8007B7A94ED0C7A77EE877A0021FDEEE77A6E
:10DBE8000022322B2163C6ED7C7A6A8042D0D6EDC2
:10DBF8007D7A94ED0D7A6163F8EEE77A012B77EE82
:10DC0800877AAA80FDEEE77AC6ED7D7A10D0013BCF
:10DC18003B80EEE6D4ED0D7A6163FDEEE77AA880ED
:10DC2800C6ED777A8BE7D6ED7B7AB8EEE77AB9E777
:10DC380029492A480968DFF8B8C003708B038CF8B3
:10DC480000203DD4264900220B4618780B2803F102
:10DC58000C0318D00132192AF7D1D6F8E0312B601D
:10DC68001B4AB6F9E401D6F8E811A8803B88C2F847
:10DC78000A10CCE7D4ED0D7A6163FDEEE77AAA804D
:10DC8800C6ED7D7AC3E71748D0F800C05300BCF151
:10DC9800000F09D003EB020E01EB8E0E9CF801C0B9
:10DCA8009EF801E0E645D8D21344DFF848C00E4A92
:10DCB80001EB830100230160ACF800301360CCE76E
:10DCC8000A4B1B78032BBDD1FEF768FCC5E700BFE4
:10DCD800641C002000000000106100202361002067
:10DCE800447003081C61002094630020131800206E
:10DCF8002A61002090630020022838B504460FD816
:10DD0800C0EB0013094A0A490A4D0C70C0EB8303A3
:10DD180002EB430318462B6017F06EFF1AF006FB60
:10DD2800601CC0B2BDE83840FEF744BD10150020A5
:10DD3800E4140020001500202DE9F047B0F9085040
:10DD48000D81EDB2382D8CB00C4600F014830646D8
:10DD5800914645D9812D00F0FA8000F28D80542D2E
:10DD680000F0688140F2E1816E2D00F0B882802DCC
:10DD780040F0DD819F4B1F78023717F0FF0700F056
:10DD880090809D4EDFF88082DFF89CA2DFF89C929D
:10DD980037440A25013616E0322D00F06E83A5F1CE
:10DDA8003C00C0B2132840F2A98300232268511C0A
:10DDB800216015702268B74202F1010121601370D9
:10DDC8006FD016F8015B0A2DE6D1B9F8003005339B
:10DDD800A8FB0323DB08FF2BA8BFFF23DBB2E5E783
:10DDE800042D00F0EE8240F20C82202D60D040F22B
:10DDF8005882242D00F06A82282D40F098810B6803
:10DE0800DFF82C827D4E591C022221601A7023688B
:10DE180006275A1C22601F7023680A22591C216099
:10DE28001A70236801255A1922601D70B8F800106D
:10DE38002046F7F73DFAB8F802102046F7F738FA07
:10DE480023685A1922601F702368502259192160CB
:10DE58001A7023680022591921601A7031882046E7
:10DE6800F7F726FA71882046F7F722FA2B46284654
:10DE7800A3810CB0BDE8F087A02D56D040F2D88120
:10DE8800B82D00F06782FE2D40F051815C4D05F100
:10DE9800080635F9021B204689B2F7F709FAAE429F
:10DEA800F7D101252B462846A3810CB0BDE8F087A1
:10DEB800544D55496A8823680532A1FB0202C2F312
:10DEC800C702581C20601A702A8823680532A1FBF3
:10DED8000202C2F3C702581C20601A70AB8822687D
:10DEE8000533A1FB0313C3F3C703511C216013704F
:10DEF800A9892046F7F7DCF923686A7A591C21605A
:10DF08001A702368AA7A591C21601A7069882046F9
:10DF1800F7F7CEF929882046F7F7CAF9A9882046E5
:10DF28000125F7F7C5F92B46A1E7384B08461968CC
:10DF3800F7F7A6F9364B20461968F7F7A1F9354BDC
:10DF4800204619680125F7F79BF92B468FE7294BDF
:10DF58001E78043616F0FF06A3D02F4B2F4F1E4411
:10DF680003F101094FF00A0824E0B8F1500F00F05E
:10DF78008782B8F15A0F00F0CC82B8F1320F00F066
:10DF8800E582A8F13C00C0B2132840F2F1820025D6
:10DF9800294623685A1C2260204683F80080F7F738
:10DFA80087F929462046F7F783F94E453FF479AFBC
:10DFB80019F8018BB8F10A0FD7D1194B19499D6887
:10DFC8001A68087805EB85054FF6FF716D008D42DC
:10DFD800A8BF0D469142A8BF114625EAE57521EA7A
:10DFE800E1712328ADB289B2D3D10548DB688380BB
:10DFF800C280CEE77D12002054510308D8140020B7
:10E00800204A002070130020CDCCCCCCACF7FF1FE9
:10E01800B0F7FF1FB4F7FF1F64510308E451002055
:10E02800B44B00201C4A0020984B0020A44B002031
:10E03800D01400200B68BC4F591C012221601A70B3
:10E04800236800259A1822601D70236897F86D20B0
:10E05800591C21601A70236897F86C20591C21609C
:10E068001A70B7F868102046F7F722F923685A1C87
:10E0780022601D7023683422591C21601A70B7F879
:10E088006A102046F7F714F9BD1E07F1660635F841
:10E09800021F2046F7F70CF9AE42F8D12268142186
:10E0A800531C2360012500231170F96F226805FABB
:10E0B80003F0084203F1010314BF01210021501CA1
:10E0C800142B20601170F0D123680222591C2160A2
:10E0D8001A70B7F86E102046F7F7EAF8B7F870101C
:10E0E8002046F7F7E5F8B7F874102046F7F7E0F898
:10E0F80023680D22591C21601A70796F2046F7F7A2
:10E10800BFF823685A1C22601D7023685A1C2260BD
:10E118001D7022680021531C0125236028462B46C8
:10E128001170A3810CB0BDE8F087522DF1D02146C3
:10E138002846FCF7DBF8824600287FF4B2AE742D3F
:10E14800D6E9008700F0058240F2EA81772D00F0D9
:10E158008281E62D40F0A981B84500F06B82D4E9B0
:10E16800003CACEB03030097019705465F1E43464E
:10E178000022974203F1010E04A968461ADDC6F889
:10E1880000E093F800E02368ADF808E0CDE9043C2E
:10E19800FFF7D2FD2268049BD4F804C09B1A013310
:10E1A80003F0FF03FF1AD6E900325CBF0135EDB278
:10E1B8009A42DDD1C6F80080CDF814C02768E5B1D1
:10E1C8004FF00008C14607F1010ACDF810A087F802
:10E1D800009033685A1C32601B78ADF80830002272
:10E1E80004A96846FFF7A8FD049B08F10108A3EB02
:10E1F8000A033B704545049FE5D1012527602B465E
:10E2080035E6022D00F01F8100F21081012D8ED11C
:10E218000B680022591C21601A7023685A1C22605E
:10E228001D7022682921531C23602B4611701EE69D
:10E23800822D7FF47CAF0B683C4A3D4D11783D4AF6
:10E248003D4E581C2060197091892046F7F730F828
:10E258002B883A4922680533A1FB0313DB08FF2BFF
:10E2680002F10101A8BFFF2321601370B16881F397
:10E27800100189B22046F7F71BF8316801F30F0146
:10E2880089B22046F7F714F823682D4A591C1278EA
:10E2980021601A70298820460125F7F709F82B46CE
:10E2A80001E6052D7FF443AF0B2226492046F6F7F9
:10E2B800CFFF082224492046F6F7CAFF0125072286
:10E2C80022492046F6F7C4FF2B46D0E5204B93F8A9
:10E2D800F821002A00F0CE80D3F8FC1145E0144D57
:10E2E80016492B882268144E0533A1FB0313DB085B
:10E2F800FF2B02F10101A8BFFF2321601370B16851
:10E3080081F3100189B22046F6F7D2FF23F05CFAB8
:10E3180001462046F6F7CCFF316801F30F0189B2B8
:10E328002046F6F7C5FFB5E7881300200E18002031
:10E338000818002070130020D0170020CDCCCCCCBA
:10E348001318002090A203089CA20308A8A203089F
:10E358001C0F0020B94D08462968F6F791FF23687D
:10E368002A79591C21601A70A96820460125F6F7F8
:10E3780087FF2B4697E50A68B14B0125511C2160A0
:10E3880015702268052150192060117022680A2131
:10E3980050192060117022680021501920601170F6
:10E3A800226819785019206011702268597850191C
:10E3B8002060117022689978531923602B461170D8
:10E3C80055E52A469F492046F6F742FF0021204698
:10E3D800F6F76EFF23689C4900255A1C22601D70C1
:10E3E800236802265A1C22601E7023680A22581CC1
:10E3F80020601A702046F6F72BFF23685A1C22600B
:10E408001D7023685A1C226029461D70202204A80A
:10E4180025F0D7F8202204A92046F6F719FF22682C
:10E428000125531923602B46167020E50B6804223A
:10E43800591C21601A7023680022591C21601A7027
:10E448002268062167E60422804920460125F6F75E
:10E45800FFFE2B460BE5B8451BBF08F101033360EF
:10E46800014698F800107A4A2046012514F044FD28
:10E478002B46FCE4774B196877E7BAF80030A6E436
:10E48800754A9568116805EB85056D004FF6FF73B1
:10E498009D42A8BF1D469942A8BF194625EAE575C1
:10E4A80021EAE171ADB289B273E5F52D00F0E280A1
:10E4B800472DA7EB080967D0392D00F0738100F2CA
:10E4C800B380212D00F09A83292D40F0AF8108F107
:10E4D8000103336098F800300A2B00F02384502B96
:10E4E80040F016843046F6F7A1FE5C4F388030467F
:10E4F800F6F79CFE012578802B46B8E405F05AF91A
:10E5080000283FF452AC03780A2B3FF64EAC438800
:10E518005DE4534AD2E9001303EB83035D00B5E7DA
:10E52800442DC2D1B84540F0FF804E4B0246987149
:10E538002368591C21601A70B9F1000F3FF4B1AC7F
:10E54800494BC9F8003001252B4690E4D7E9001360
:10E55800E2E7B8451BBF08F101033360014698F8AC
:10E568000010424A2046012514F0C6FC2B467EE4E2
:10E5780005F020F900283FF40AAD03780A2B3FF68E
:10E5880006ADD0E90131C7E73046F6F737FEB9F1F5
:10E59800050F074600F2F7808025A8464FF0010ACC
:10E5A800D4E900239B1A103BAB42B8BF1FFA83F88B
:10E5B800FAF79EFF8368DB1B98453946204688BFDB
:10E5C8001FFA83F8F6F75CFE2668BAF1000F00F030
:10E5D800B680FAF78DFF836807EB08029A4240F28B
:10E5E8004B83B146FAF784FF8368A3EB0708FBF770
:10E5F80041F81F483946476843464A467F6AB84744
:10E60800BAF1000F00F0B780236885420344236005
:10E618007FF747AC002100E0236801305A1CA8426C
:10E6280022601970F8D13CE4552D00F0D080572DA8
:10E6380040F0FC804FF0FF352B4618E410610020B5
:10E64800CC140020EB14002084A203087CA2030849
:10E6580055CF0108C0380020CC4B0020D81400202A
:10E66800D84B00201C0F0020B9A20008BDD7010814
:10E67800D82D0020B84540F00983654BFF221A7158
:10E688004FF00008634D10F03BF8414620226248E5
:10E6980085F8008024F095FF8DF810809DF81030E3
:10E6A800072B00F2B1835D4F5B4E42469DF8103058
:10E6B80003EB430307EBC3035B7CE3B19DF8103026
:10E6C80003EB430307EBC30320215B699BB19DF870
:10E6D800103003EB430307EBC303586946F82200E5
:10E6E800F5F7C4F82B7856F82300F5F73FFA2A789F
:10E6F8000132D2B22A709DF810300133DBB28DF8A6
:10E7080010309DF81030072BD0D92368591C216090
:10E718001A70B9F1000F3FF4C4AB414BC9F800308F
:10E7280001252B46FFF7A3BB08F10103336098F8D6
:10E738000020374B012A9A717FF6FAAE7AE74146F4
:10E748002046F6F7B5FD23685A1C226083F800A01E
:10E75800D4F80090FAF7CCFE836807EB08029A42D7
:10E768003FF640AFFAF786FF2E48456843464A46CB
:10E7780039466D6AA847236830800125184420600F
:10E788002B46FFF774BB3046F6F750FDD6E900324A
:10E798009A42804601D1454602E73046F6F752FDD7
:10E7A8004546FDE608F10103336098F800300A2B6E
:10E7B80000F097823046F6F745FD3046F6F742FD01
:10E7C80001253046F6F73EFD2B46FFF750BB08F112
:10E7D8000103336098F80070FF2F00F0BE82FE2F0F
:10E7E80000F0A6823046F6F721FDD6E90032D21AAB
:10E7F800002A00F3F482332F3FF61CAF0A4B0125A1
:10E8080023F8170006F048FD2B46FFF730BB00BF82
:10E818001C0F00202B6A00204C69002018390020AA
:10E8280079F20208D82D0020881300200B3DEF2D27
:10E838003FF600AF01A353F825F000BF7DF50008AF
:10E848003DE600083DE600083DE600083DE6000814
:10E858003DE600083DE600083DE600083DE6000804
:10E868003DE600083DE600083DE600083DE60008F4
:10E878003DE600083DE600083DE600083DE60008E4
:10E888003DE600083DE600083DE600083DE60008D4
:10E898003DE600083DE600083DE60008F9F40008FA
:10E8A8003DE60008D5F400083DE60008B3F400088A
:10E8B8003DE600083DE600083DE6000883F4000850
:10E8C8003DE600087DF300083DE600083DE6000847
:10E8D8003DE6000845F300083DE6000833F300086C
:10E8E8003DE60008B5F200083DE60008E7F100083B
:10E8F8003DE600083DE600083DE600083DE6000864
:10E90800ABDE00083DE600088DF100083DE6000892
:10E918003DE600086DF100083DE600083DE6000808
:10E928003DE600083DE600083DE600083DE6000833
:10E9380061F100083DE600083DE600083DE60008F4
:10E948001DF100083DE60008CBF000083DE6000890
:10E958003DE600082DFB00083DE600083DE60008FE
:10E968003DE600083DE600083DE600083DE60008F3
:10E978003DE6000879FA00083DE6000897F9000826
:10E988003DE6000845F800083DE6000887F600085F
:10E998003DE6000857F6000835F60008A9F5000816
:10E9A8003DE600083DE600083DE600083DE60008B3
:10E9B8003DE600083DE600083DE600083DE60008A3
:10E9C8003DE600083DE600083DE600083DE6000893
:10E9D8003DE600083DE600083DE600083DE6000883
:10E9E8003DE600083DE600083DE600083DE6000873
:10E9F8003DE600083DE600083DE600083DE6000863
:10EA08003DE600083DE600083DE600083DE6000852
:10EA18003DE600083DE600083DE600083DE6000842
:10EA28003DE600083DE600083DE600083DE6000832
:10EA38003DE600083DE600083DE600083DE6000822
:10EA48003DE600083DE600083DE600083DE6000812
:10EA58003DE600083DE600083DE600083DE6000802
:10EA68003DE600083DE600083DE600083DE60008F2
:10EA78003DE600083DE600083DE600083DE60008E2
:10EA88003DE600083DE600083DE600083DE60008D2
:10EA98003DE600083DE600083DE600083DE60008C2
:10EAA8003DE600083DE600083DE600083DE60008B2
:10EAB8003DE600083DE600083DE600083DE60008A2
:10EAC8003DE600083DE600083DE600083DE6000892
:10EAD8003DE600083DE600083DE600083DE6000882
:10EAE8003DE600083DE600083DE6000881FD000817
:10EAF8003DE60008F7FC000837FD00083DE6000881
:10EB08003DE600083DE600083DE600083DE6000851
:10EB18003DE600083DE600083DE600083DE6000841
:10EB28003DE600083DE600083DE600083DE6000831
:10EB3800ABDE00083DE6000875FB00083DE600086E
:10EB4800FDFB0008E3FB0008ABFC00083DE60008FD
:10EB5800B1F000083DE6000885F0000873F00008F1
:10EB68000FF000083DE60008E7EF00083DE6000862
:10EB78003DE60008D3EF00089DEF00082DEF0008E0
:10EB8800FDEE00083DE60008DBEE00083DE6000863
:10EB9800C3EE00083DE600083DE600083DE6000833
:10EBA8003DE600083DE600083DE600083DE60008B1
:10EBB8003DE600083DE600083DE600083DE60008A1
:10EBC8003DE600083DE600083DE60008A9EE00081D
:10EBD8003DE600083DE6000831EE00083DE6000885
:10EBE8003DE600083DE600083DE600083DE6000871
:10EBF8003DE600083DE60008BDF10008424608F180
:10EC08000103336012F8023BCB4F03EB83035B0035
:10EC18007B80326098F8013003EB830308F103022C
:10EC28005B003B80326098F8023003EB83035B00A3
:10EC38003046BB80F6F7FAFA3268B8811346511CA1
:10EC4800316013F8021B797233605278BA727268B5
:10EC5800D31A052B7FF725A93046F6F7E7FA78800F
:10EC68003046F6F7E3FA38803046F6F7DFFA012542
:10EC7800B8802B46FFF7FBB8FAF7FCFCAF483246E2
:10EC8800466843463946766AB047BDE4424608F1CD
:10EC98000103336012F8023BA949326098F8012059
:10ECA8004A71042B0B7103D9FF2B7FF432AAE7E4D6
:10ECB800A4490978914205D8022B7FF42AAAFF2A91
:10ECC8007FF427AA236801255A1922601D70B9F11B
:10ECD800000F3FF4E6A89C4BC9F800302B46FFF71D
:10ECE800C6B808F102033360984B98F801201A70EF
:10ECF80008F10302326098F802205A7008F1040201
:10ED0800326098F803209A7001252B46FFF7AFB8B8
:10ED18003046F6F78BFA01253046F6F787FA2B4688
:10ED2800FFF7A5B83046F6F781FA894FFFF7DEBB43
:10ED380008F10203336098F80150022D3FF67AACCF
:10ED48003046F6F773FA834B03EB45034FF0FF3574
:10ED5800A3F86E002B46FFF78AB83046F6F772FA2A
:10ED680033687C4F1A46591C316012F8021B87F829
:10ED78006D1032605B7887F86C303046F6F756FADB
:10ED8800A7F868003046F6F751FA3046F6F74EFA1B
:10ED9800D6E90083A3EB0802012AA7F86A0005DD7B
:10EDA8003046F6F743FAD6E900837867A3EB080202
:10EDB800032A2BDCA3EB0803002B7FF772A830464D
:10EDC800F6F740FAD6E900239B1A002B7FF769A8CB
:10EDD80030460125F6F736FA2B46FFF748B85A1C95
:10EDE80032601B78002B7FF406AD132F3FF603AD7E
:10EDF80098B9584A0125D36F05FA07F723EA07039C
:10EE0800D3672B46FFF733B842467EE43046F6F721
:10EE1800F5F9D6E900837867CCE73846012506F08E
:10EE280071FA2B46FFF723B808F10103336098F80D
:10EE380000300F2B3FF6FEAB08F102023260C3EB45
:10EE4800C303454A98F80110D15408F10301316011
:10EE5800134498F802205A7008F10402326098F8B6
:10EE680003209A7008F10502326098F80420DA70DD
:10EE780008F10602326098F805201A7108F10702B5
:10EE8800326098F806205A7108F10802326098F842
:10EE980007209A71012515F033F92B46FEF7E7BFD5
:10EEA8003046F6F7C3F92D4FB8813046F6F7BEF96C
:10EEB800012578812B46FEF7DABF3046F6F7B6F91A
:10EEC800274A00EB80004300012513802B46FEF7FC
:10EED800CEBF3046F6F7AAF9224F78823046F6F7C9
:10EEE800A5F9B8823046F6F7A1F90125F8822B4634
:10EEF800FEF7BDBF08F101033360304698F8007093
:10EF0800F6F7A0F9D6E900134A1C326014480978CC
:10EF180081709B1A022B2DDC134B0125DF712B46C8
:10EF2800FEF7A5BF114B124918687622012524F077
:10EF380024FB2B46FEF79BBF70130020D82D002022
:10EF48001C0F00207D120020A9A20008CC1400206C
:10EF5800D014002088130020305A0020641C0020A0
:10EF68008C6A0020503B0020D46800200015002047
:10EF7800F46E03083046F6F765F93368BC4A591C45
:10EF880031601B78D37130460125F6F75BF92B46C3
:10EF9800FEF76DBF424608F101033360B54B12F826
:10EFA800021B1970326098F801205A7008F10302A8
:10EFB800326098F802209A703046F6F737F9AE4B6F
:10EFC8000125D8802B46FEF752BF3046F6F72EF9BA
:10EFD800A94F38803046F6F729F9788044E6DFF8FB
:10EFE800C482A64F002598F800309D423046BEF6F0
:10EFF80058AFF6F71BF918F087FD07EB850383ED8B
:10F00800000A0135EFE7B9F10D0F7FF413AB08F1F2
:10F018000103336098F80050072D3FF60BABDFF87B
:10F02800888230460C27F6F701F907FB05F708EB4D
:10F038000705A8803046F6F7F9F8E8803046F6F775
:10F04800F5F8336828811A46591C316012F8021BFA
:10F05800A97232605B78EB723046F6F7CFF801257B
:10F0680048F807002B46FEF702BF3046F6F7DEF8F1
:10F07800834B012518802B46FEF7F9BE08F10103E2
:10F08800336098F80000070600F119867D4B1B785D
:10F09800DE073EF506AF032828BF00200125FEF74E
:10F0A8002BFE2B46FEF7E3BE764B1B78DD073EF5BD
:10F0B800F8AE0125F9F786FCF5F7BEFF2B46FEF7FB
:10F0C800D6BE08F10103336098F80070112F3FF69F
:10F0D800B1AA08F1020333606B4D98F8013005F8C6
:10F0E80017303046F6F7A2F840F6CA039842A8BF90
:10F0F800184640F2EE2305EB47019842B8BF184680
:10F1080001251923A0F2EE2292FBF3F22B464A7056
:10F11800FEF7ADBE434608F101025C4D326013F8BC
:10F12800022B2A71336098F801306B713046F6F77C
:10F138007DF8336828805A1C32601B78AB713046E2
:10F14800F6F774F8336868805A1C32601B78EB71E4
:10F1580001252B46FEF78BBE0125FAF7E9F82B4669
:10F16800FEF785BE4A4D002301E0D6F8008008F17D
:10F178000102326098F80020EA540133082BF4D1D8
:10F18800FEF78FBE08F101033360424B98F8002068
:10F198005A703046F6F756F8D6E900329A423EF4ED
:10F1A80080AE5A1C32603C4A1B78137101252B46ED
:10F1B800FEF75DBE334B1B78DA073FF53BAA374BAA
:10F1C80093F8F821002A00F0AD80D3F8FC01F2F79B
:10F1D8001BF90125F5F730FF2B46FEF748BE07253A
:10F1E800B9FBF5F5C5EBC50399457FF423AADFF80C
:10F1F800B0A0EDB2002D3EF454AE08F10103336027
:10F2080098F90020264B4FF0000993F9021091421B
:10F2180003F1080306D009F10109B9F1050FF4D18A
:10F22800FFF708BA0AEBC9073046BA70F5F7FEFFD0
:10F23800D6F800802AF83900434608F10102326006
:10F2480013F8022BFA70336098F801303B7108F11B
:10F258000303336098F80230BB71434608F1040891
:10F26800C6F80080013DDB787B71EDB2C2E700BFD4
:10F27800D4680020846A00208C5F0020645F00202E
:10F288005663002099490020746F00200859002017
:10F29800181F00209C6A0020541400201C0F002016
:10F2A800BC3B00207D1200206C60002008F10103A7
:10F2B800336098F800001D283FF6BCA908F1020346
:10F2C800336098F8011003293FF6B4A9CB4ACC4F14
:10F2D8000A2303FB00F3D01808F1030541713560D8
:10F2E80098F80210D15408F10403336098F80330F9
:10F2F800437008F10503336098F80430837008F10F
:10F308000603336098F80530C37008F107033360CB
:10F3180098F80630037101254FF0FF333B602B4608
:10F32800FEF7A5BDFEF79AF953E708F1010333602C
:10F33800B44B98F80020DA73FEF7B3BD08F1010367
:10F34800336098F800301F2B3FF674A9B9F1050F08
:10F358007FF470A93046F5F751FFD6E90032D21A8A
:10F36800002A7EF79EAD5A1C3260A74A1B78D370DC
:10F37800FEF797BD08F10103A24D336098F80030FD
:10F388002B723046F5F752FFE8823046F5F74EFF0C
:10F3980068823046F5F74AFF3368A8825A1C326003
:10F3A8001B786B7373689A1A032A42DCD6F80080BC
:10F3B800A3EB0802052A2CDC002A7EF772AD08F1BF
:10F3C8000102326098F80020EA76D6F80080A3EBB4
:10F3D8000803052B16DD08F10103336098F80030A7
:10F3E8006B763046F5F72EFF3046F5F72BFF3046A3
:10F3F800F5F728FF3046F5F725FF3046F5F722FFE9
:10F40800D6F800807368A3EB0803002B7EF749AD9C
:10F41800DEE43046F5F716FF3046F5F7EFFE3046E6
:10F42800F5F710FFD6E90083A3EB0802002ACEDD2A
:10F43800C5E73046F5F7FAFEE8833046F5F7F6FEFD
:10F44800D6E90083A3EB0802032A2884B0DD4346EB
:10F4580008F10102326013F8022B2A76336098F81B
:10F468000130AB763046F5F7E1FE0A22A0F57A7353
:10F4780093FBF2F32B77736898E708F10103336085
:10F48800624A98F800101170FB1A002B7EF709AD3C
:10F4980008F10203336098F80130003318BF0123E4
:10F4A800012553702B46FEF7E2BC3046F5F7BEFE49
:10F4B800574F38603046F5F7B9FE78603046F5F7B3
:10F4C800B5FE0125B8602B46FEF7D1BC3046F5F7EE
:10F4D80095FE504B93F8F821C3F8FC01002A7EF4FE
:10F4E800E0AC012283F8F82115461346FEF7BFBCAD
:10F4F80008F10103336098F80050132D3FF69AA8DD
:10F5080008F10203336098F8010013F02FFD00287A
:10F518003FF490A8062303FB05F33F4D0278EA5415
:10F5280008F1030232601D4498F802306B7008F14C
:10F538000403336098F80330AB7008F105033360B7
:10F5480098F80420EA70BB420ED008F10603336035
:10F5580098F805302B7108F10703336098F8060016
:10F5680013F004FD03786B7101251AF061FB2B463B
:10F57800FEF77DBC294A0023C2E90033C2E9023301
:10F58800B9F1100F28BF4FF0100913744B45BEF4A2
:10F5980088AC3168481C30600978D1540133F5E7EC
:10F5A80008F101033360BB4218BF08F1020398F861
:10F5B80000201ABF336098F80130002382B14FF45D
:10F5C8000040FDF73FF9164B1B78DB0701D50EF01D
:10F5D80073F9144B002201251A702B46FEF747BC1D
:10F5E800114910480A68003318BF012322F4004269
:10F5F800012503700A602B46FEF739BC38610020EC
:10F60800A8080020181F00208C140020706C00200F
:10F618008C5800201C0F0020486E00200821002074
:10F6280099490020F6600020A81B00207E4B1B781B
:10F6380013F001017EF4FEAF08F10103336098F87E
:10F64800000001250FF062FA2B46FEF710BC434676
:10F6580008F101023260754A13F8021B9170336099
:10F66800734A98F80130537108F103033360714B02
:10F6780098F80220DA7001252B46FEF7F8BB3046D1
:10F68800F5F7D4FD3046F5F7D1FD3046F5F7CEFD58
:10F698003046F5F7D7FD3368674D1A46581C296878
:10F6A800306012F8020B81F8460032605B7881F80E
:10F6B80047303046F5F7C6FD3046F5F7C3FD30460E
:10F6C800F5F7C0FD3046F5F7BDFD30462F68F5F774
:10F6D800ADFD388730462F68F5F7A8FDD6E90083D9
:10F6E800A3EB0802012AF8860CDD08F101022B6859
:10F6F800326098F8002083F82D203046F5F7A2FDF7
:10F70800D6E90083A3EB0802032A0CDD30462F68F4
:10F71800F5F78CFD788630462F68F5F787FDD6F823
:10F7280000807368B886A3EB0802012A04DD30461E
:10F73800F5F77CFDD6E90083A3EB08010D292A68BB
:10F7480036DD08F10103336098F8003082F8513053
:10F758003046F5F777FD3046F5F774FD3046F5F796
:10F7680071FD3046F5F76EFD33682F681A46591C4F
:10F77800316012F8021B87F84F1032605B7887F807
:10F7880056303046F5F752FDB88130462F68F5F708
:10F798004DFD788230462F68F5F748FD33682A68B2
:10F7A8003883591C31601B7882F83030D6E90083E1
:10F7B800A3EB0803062B28682FDD434608F1010256
:10F7C800326013F8022B80F86E20336098F801300D
:10F7D80080F86F3008F10303336098F8023080F83E
:10F7E800703008F10403336098F8033080F8713002
:10F7F80008F10503336098F8043080F8723008F196
:10F808000603336098F8053080F86B3008F1070379
:10F81800336098F8063080F86C30012516F0A0FCAB
:10F828002B46FEF724BB00BF99490020641C00202A
:10F83800482400208C6A00200015002008F10103EC
:10F848003360CD4DCD4F98F80030FB803046D5F869
:10F858000080F5F7EBFCA8F802003046D5F80090D8
:10F86800F5F7E4FCD6E90083A3EB0802072AA9F818
:10F87800000018DD3046F5F7D9FC78813046F5F7F9
:10F88800D5FCB8813046D5F80080F5F7CFFCA8F84C
:10F8980004003046D5F80080F5F7C8FC7368A8F86E
:10F8A8000600D6F80080A3EB0802032A09DD3046DB
:10F8B800F5F7BCFCF8813046F5F7B8FCD6E90083CB
:10F8C8003882A3EB0802002A09DD08F101012A6841
:10F8D800316098F8001082F82610D6F80080A3EB63
:10F8E8000803092B23DD08F10103336098F8003081
:10F8F800BB703046F5F7A6FC3046F5F797FCF88064
:10F908003046F5F793FC336838811A46591C316044
:10F9180012F8021B797532605B78D5F80090BB75D8
:10F928003046F5F783FCD6F80080A9F84C007368D8
:10F93800A3EB0803082B1BDD08F101022B683260DA
:10F9480098F8002083F860203046F5F76FFCB883FC
:10F958003046F5F76BFCF88330462F68F5F766FC00
:10F96800A7F8620030462E68F5F760FCA6F8640038
:10F97800F5F754F809F0FCF9814B28681B68002B4F
:10F988006BD0012514F04CFC2B46FEF770BA4346A9
:10F9980008F101023260794F13F8022B7A70336054
:10F9A800784A98F80130137008F103033360764DF4
:10F9B80098F802302B7108F10403336098F803308B
:10F9C800092BA8BF09233046AB70F5F72FFCD6E901
:10F9D8000083A3EB0802012A288005DD3046F5F7ED
:10F9E80025FCD6E9008328824345424627D1A2EB6D
:10F9F8000802072A1DDD434608F10102326013F8A8
:10FA0800022B3A71336098F80130FB7008F1030358
:10FA1800336098F802303B703046F5F707FC78837E
:10FA28003046F5F703FC336878825A1C32601B783D
:10FA38003B750125F4F7F2FF2B46FEF718BA30465E
:10FA4800F5F700FCD6E900329342F2D0591C316038
:10FA58001B78EB70D6F80080C9E74C484C494D4AF2
:10FA68004D4B036001250B6013602B46FEF7FFB971
:10FA78004A4B1D68002D53D02B6828465B68984771
:10FA880007463046F5F7D2FB3F2835D941F26F7368
:10FA9800984203D8424B002298801A70D6E9003267
:10FAA800D21A012A7EF7FDA95A1C3260DFF8F080CD
:10FAB8001A7888F80220FF2F3EF4F3A99A1C0CA9A3
:10FAC800326000225F7801F8202D284606F0F8F809
:10FAD8009DF81030BB4203D03946284606F0F3F8AB
:10FAE800D6E900329A423EF4DCA95A1C32601B78EF
:10FAF80088F80830FEF7D5B9C208DFF8A4800132CB
:10FB080000F007030133D0B2014688F800001A4616
:10FB1800284688F8013005F01DFFA8F80400BDE765
:10FB2800FF27AEE71F4B1B78012B3EF6BAA908F159
:10FB3800010342463360DFF8709012F8023B89F8FF
:10FB48000230326008F1030398F801003360FB1AB1
:10FB5800012B98F8021040F3FF803046F5F766FB5A
:10FB68000125A9F800002B46FEF781B9024B186859
:10FB7800034600F11E011BE000150020F8310020AB
:10FB8800646A00207C6A0020503B0020205B002033
:10FB9800945B00207C5C00205D0500089C490020E7
:10FBA800A04900206417002068170020D6F80080BC
:10FBB800424608F10105356012F8025B1D72326099
:10FBC80098F801205A7208F10302326098F802206E
:10FBD8009A7206339942E9D11FE69E4B1B78D807E3
:10FBE8003EF55FA99C4B4FF4C87201251A802B463D
:10FBF800FEF73DB9B9F1090F7EF71CAD974F08F133
:10FC080001033D6833602979EA7898F80030EB7091
:10FC1800914208F1020208BF2B713260E979AA7992
:10FC280098F80130AB71914208BFEB7105F10902F8
:10FC380005F10C013368581C3060187802F8010B84
:10FC48009142F7D19A1C32605A78642AA8BF64227C
:10FC5800D91C2A7331609A782A701A1D3260DB78B1
:10FC68006B703046F5F7E2FAD6E90083A3EB080299
:10FC7800002AE8812EDCA3EB0803012B0BDD4346A9
:10FC880008F101013A68316013F8021B11743360FE
:10FC980098F80130537401251AF058F82B46FEF7EE
:10FCA800E6B86C4B1B78D9073EF5FBA86C4A13786D
:10FCB800012543F0040313702B46FEF7D8B800F073
:10FCC8007F00062828BF002001250EF0DBFF2B4609
:10FCD800FEF7CDB808F10102396832609A1A98F82F
:10FCE80000000872002A7DDCD6F80080C3E73046A1
:10FCF800F5F784FAD6E900835A4FA3EB0802002AE5
:10FD0800386007DD08F10102326098F800203A7186
:10FD1800D6F80080A3EB0803032B7EF7C2A8304671
:10FD2800F5F76CFA0125B8602B46FEF7A0B808F184
:10FD380001034D4933600A7898F80030C2B90422AB
:10FD48000A704A4A9B001380F2F7D8FC484B0125F9
:10FD580018602B46FEF78BB8464B1A88012512FB14
:10FD680000F22B4692FBF1F2A9F80020FEF77FB8CB
:10FD7800042A7EF496A8E4E7434608F101023260BB
:10FD880013F8025B336008F1030298F8013032601F
:10FD980098F80210002D48D0012D7EF482A8052B7A
:10FDA8003EF67FA805293EF67CA899423EF479A83C
:10FDB800314E1A2001FB006213FB00F311685068F2
:10FDC800D2F808C0D768995133445860C3F808C0BE
:10FDD800DF601169506958611961128B1A832B46CB
:10FDE800FEF745B808F10202326098F801204A711E
:10FDF800D6F80080A3EB0802002A7FF73CAF08F191
:10FE080001013A68316098F800101171D6F8008045
:10FE1800A3EB0802002A7FF72EAF08F101013A6828
:10FE2800316098F80010D1715EE7022B3EF639A8D0
:10FE380002293EF636A899423EF433A80F487622A6
:10FE480001FB0201012503FB020023F096FB2B4670
:10FE5800FEF70DB899490020266100208C1E00206D
:10FE680053140020106100205E6600208466002084
:10FE7800F0600020686A0020B016002010150020ED
:10FE88002DE9F04FA14BA24D1B7895F80090DB07A8
:10FE980085B080463FD59F4C9F4EB9F1010F66D083
:10FEA800C0F08280B9F1020F2AD0E37B83B1A38925
:10FEB80073B19A4B1B785BB10EF0FAFE002800F084
:10FEC800EE80237C83422CBF01220022327000E0A6
:10FED8003278217A632907D89148B9F1020F03785B
:10FEE80070D0002B40F085808E49A37B914538BFA8
:10FEF800914681F80090002B4AD105B0BDE8F08FFB
:10FF0800894A8A4B12881B889A42CED94FF0010938
:10FF180085F80090C9E7844F7E4C3A88A9F103031D
:10FF2800012B40F282807B88D31A002BB8BF5B423A
:10FF3800142B05DCE388934265D82188914262D36B
:10FF4800754E7B4B1B78022BA7D17A883B88734967
:10FF58009B1A002BB8BF5B42142B764A0978918014
:10FF6800CCBF00230123B9F1010FD38098D16F4B87
:10FF78006D4A1B88617C12885B1A9A4234DD6E4B8D
:10FF88001B88934291D24FF0000985F800908CE7C6
:10FF9800B9F1010F7DD0B9F1020FAED1072005B03C
:10FFA800BDE8F04FFCF716BB634B5F4A1B88617CCA
:10FFB80012885B1A9A423FF778AF4FF0010985F82B
:10FFC800009072E7ABB90125C0F804800570C1F153
:10FFD80064015A4D03FB01F385FB0351DB17A3EBC7
:10FFE800A153643343707FE74FF0020985F800900E
:08FFF8005BE74368524DA8EBE2
:020000040801F1
:100000000303AB42C8BF41703FF772AFE3E7B2EB07
:10001000430F434E99DC43484949464A00234FF079
:10002000030986F8009085F8009003700B80138018
:100030008BE7E388934228D82188914225D37B8897
:10004000D31A002BB8BF5B42142B3FF77DAF344E61
:10005000237D4FF0000E86F800E085F800E02BB31A
:10006000304AF1461370A188354AB4F802C03148CD
:100070009BB211FB03F111801CFB03F32A4A03809E
:1000800064210023517053605FE7B2EB430FD6DC6D
:10009000B9F1030F3FF458AF49E7082005B0BDE8B8
:1000A000F04FFCF79BBA0222327016E727492388EB
:1000B0000968B2FBF3F20132082A91F97410DFF8F3
:1000C0006490A8BF0822D3B2914289F800306ED064
:1000D00000296CD01E49DFF880C091F800B00BF108
:1000E0000101ACFB01A0400800EB4000081A584594
:1000F00002905CD017494FF0760A0AFB001E9EF969
:1001000074E096454BD0CDE900CA03934FF0FF3A17
:10011000014627E099490020884B002070130020F9
:10012000B04B00200E180020904B00201318002028
:10013000081800208C4B00201C4A0020204A002078
:100140008A4B00206BCA5F6B7F96980000150020D9
:10015000E414002010150020ABAAAAAA9CF974E0B0
:10016000964527D001F1010C0099A1FB0C314908FB
:10017000019B01EB4101ACEB01019C460E4BBAF136
:10018000000F0CFB013C03DABEF1000F08BF8246F2
:1001900059450846E2D1039B5046002807DBC0B210
:1001A000FDF7AEFD99F8003095F800905BE74FF051
:1001B000000958E7039BF0E7101500202DE9F04FE8
:1001C000B64B1D788DB0002D57D1B54BB54C93F87B
:1001D00000B0DFF80093DFF800A30BF0010B04F58B
:1001E000257854F80B0C40B1F2F776FD064600284E
:1001F00040F00D8114F8033C3BB9DC34444505F173
:100200000105EED10DB0BDE8F08FDAF8002054F80A
:10021000071C521A632AF0D9012B00F03183022BFC
:10022000EBD1A14BA149DA7889F819030032A04833
:10023000C9F8000218BF0122984854F80B3C0A7014
:1002400001219C4A0170C9F80432C9F80C33C9F87D
:1002500014339948C9F81023402389F81833F4F768
:10026000D3FB4FF48050FCF7F1FA9448F4F762FBAB
:1002700089F85C6389F85D63BFE7DFF85892D9F8C5
:1002800000020028BED0F4F709FBDFF830A209F520
:100290000378D9F80402F2F71FFD0028B2D0D9F88C
:1002A0000402F2F711FD09280346D9F808621DD0AF
:1002B0003F281BD0002E6FD1042800F0DB820C28D1
:1002C00000F09E807F28E4D0A0F12002D2B25E2A06
:1002D000DFD8202BDDD009EB06021846013682F864
:1002E0000C32C9F80862F4F71DFBD2E7002E65D185
:1002F000734B354603F5A477002D46D00833BB4237
:10030000FAD1DFF8D8B12868DBF80020845D935D6E
:100310009C42304402EB060140F0B082741E44441B
:10032000324613B9FD2A40F2F58004F8013F01324C
:10033000C9F8082210F8013F11F8017F9F42F0D060
:100340000AB1AB4513D05F48F4F7F4FAAB4508D3D4
:1003500055F8080BF4F7EEFA0920F4F7E3FA5D45D7
:10036000F6D95046F4F7E6FAD9F808220026964264
:100370008FD2741E444414F8010FF4F7D3FAD9F85D
:10038000083201369E42F6D383E703F10802BA42EF
:100390001D46B6D01346AFE70C2831D00A2B64D0E7
:1003A0000D2B62D07F2B00F0EF81FF2E3FF671AF57
:1003B000A3F12002D2B25E2A8DD96AE7404C4FF0F9
:1003C000000B04F5A4775D4602E00834BC420DD072
:1003D000324621684046F5F79FF90028F5D1A3463B
:1003E000002DF2D125460834BC42F1D1002D8AD12E
:1003F000BBF1000F3FF44DAF3248F4F79BFAA7E78B
:100400003148F4F797FA5046F4F794FA41E72F4B46
:10041000DAF8002044F8072CDC27002607FB053714
:10042000A4F10B0304F8036C009354F80B0CF2F7DF
:1004300053FC00283FF4E1AE54F80B0CF2F744FCF7
:1004400014F8021C4B1E02460B2B00F28A81DFE8D7
:1004500013F073016B015F01380126010C01E0000C
:100460009C008F00BA0076006E00F4F7B9FA2321E1
:10047000174823F0C1F8002800F07081A0EB0802B3
:10048000C9F80822BAB3531E09EB030191F80C1204
:10049000202940F02A82023A424427E0711B0020C2
:1004A00099490020E3180020E4140020C8510020DE
:1004B0002C120020DD020008F0A20308BCA20308F1
:1004C00074510308B4A20308C4A20308D81800207A
:1004D000281100201C0F0020C42D0020B452030856
:1004E00012F80119202940F05F810346581E002BA5
:1004F000F6D1C9F808324FF480720021404623F04B
:1005000064F8D74B1B78002B3FF47CAE5046F4F7D1
:1005100011FABEE6511C09EB01004A44202482F87E
:100520000C42C9F808120A4680F80C3209E794F820
:10053000CE30934200F09E8004F8026C75E71146BD
:1005400094F8CE000192F5F7BDFAD4F8C530019ABF
:1005500084F8CE00F9180133C4F8C530CA72D4F853
:10056000C92093427FF461AF0C2304F8023C5CE79E
:1005700094F8CD3094F8CE105340914284F8CD30A9
:10058000DAD1062304F8023C4FE7114694F8CE0076
:100590000192F5F797FAD4F8C53094F8CD10019A86
:1005A00084F8CE00F81851400133C4F8C53084F8FF
:1005B000CD10C272D4F8C92093427FF436AF09231C
:1005C00004F8023C31E7D4F8C530F9180133C4F817
:1005D000C530CA7294F8CE0001931146F5F772FA4D
:1005E000019B84F8CE00052B7FF41FAFB4F80330D5
:1005F000B4F801102278C4F8C560C4F8C930A4F872
:10060000C11084F8C320002BAED00B2304F8023CA9
:100610000BE7D4F8C530F9180133C4F8C530CA72F5
:1006200094F8CDC094F8CE00019382EA0C0C1146E8
:1006300084F8CDC0F5F746FA019B84F8CE00072B6D
:100640007FF4F3AEB4F80530B4F80310A278C4F820
:10065000C560C4F8C930A4F8C11084F8C320002BC9
:10066000ADD0082304F8023CDFE694F8CD30934285
:100670007FF462AF0D2304F8023C14F8017C002FD4
:1006800000F0B380012F00F00D81002304F8023C3C
:10069000DC34444505F101057FF4A3ADB2E5D4F89F
:1006A000C530F9180133C4F8C530CA7294F8CD00CA
:1006B000D4F8C91042408B4284F8CD207FF4B5AE07
:1006C0005FE7D4F8C530F9180133C4F8C530CA72F1
:1006D00094F8CD10022B82EA010284F8CD207FF439
:1006E000A4AE2378C02B3FF627AF6278FF2A00F034
:1006F000FE80C4F8C930A4F8C12084F8C360C4F8EF
:10070000C560002B3FF43DAF052304F8023C8CE6A6
:100710000A233C2A04F8023C0BD03E2A7FF40CAF9B
:10072000012304F8013C80E604233C2A04F8023C3F
:10073000F3D104F8016C78E64D2AC4F8C56084F85A
:10074000CD6084F8CE604AD0582A7FF4F5AE0322FB
:10075000022304F8022C84F8C43066E6D9F8082293
:1007600090E6242A77D0BBF1000F02D00D2984D067
:100770005BE6232A14D03B4B93F82A30934204BF04
:10078000012304F8033CF1E7013E09EB06030022D4
:100790003548C9F8086283F80C22F4F7CBF878E5FD
:1007A000022304F8033CE1E7C9F808324B442F4C1C
:1007B000002283F80C2204F5A47703E00834BC423D
:1007C00000F09F8021684046F4F7FCFF0028F5D038
:1007D000BC4280F0968063689847002389E6022334
:1007E00084F8C46004F8023C1FE6214BB4F8C1E071
:1007F000ADF82C700FCB0DF1300C04AE86E80F0075
:10080000D4F8C9104CF8247D601894F8C3300990CE
:1008100001276246314608A80894ADF828E08DF813
:100820002A308DF82E70FDF78BFA80BB039E0023D3
:1008300004F8023C002E3FF4E0AC54F80B0CFBF73C
:1008400021FDDC3454F8E70CB047444505F10105BF
:100850007FF4C7ACD6E4012304F8023CE5E500BF11
:10086000711B0020BC3B0020ECA20308745103085C
:10087000BC5203082548F4F795F8C3E432465FE517
:10088000234A244B24491160244ADA60B5E4049ACF
:10089000234B05923146009894F8C42004930EF03F
:1008A0003DFCC3E7D4F8C930B4F8C1200894234410
:1008B00009936E2A4FF00003ADF82E30CDF82A30A0
:1008C000ADF828207FF4E1AE08A8F4F7BFFC08A833
:1008D000F4F7B0FC064608A8F4F7ACFC08A8F4F757
:1008E000A9FC104BC3E90060CFE613465EE7052B79
:1008F0007FF622AE0122072384F8C42004F8023CCC
:1009000093E50948F5F7ACFA67E700BF2811002026
:10091000FC9F002000ED00E0EFBEADDE0400FA0514
:100920004C700020D84B0020D0A20308054A137851
:1009300051780133DBB29942137004BF0023137066
:10094000704700BF7C120020F8B56B4C636833B36E
:100950006A4B1B781BB36A4A237AA2FB0020012B47
:100960004FEA901023D01BD3022B18D1E3686433D5
:1009700083423ED8237804EB031393F82020FF2A08
:1009800005D060490132012083F820200870FFF76C
:10099000CDFF5D4B1B780122092B227220D0F8BDC0
:1009A00041F287339842FAD901232372F8BD564A9F
:1009B000564D2178E0601078642202FB0152002538
:1009C000A5770A25E577092804F1140513764FF079
:1009D000020325612372E2D14D4B01311980F8BD2C
:1009E000B4F8A2304A4A01339BB2A4F8A230538033
:1009F000F8BDA27FE37F9A42D1D104F1130104F143
:100A00001C00002311F8012F5340082213F0800F1F
:100A10004FEA430318BF83F00703013ADBB2F5D175
:100A20008842EFD1617F2078994231D194F81BC080
:100A3000354DB4F81710B4F81970237F94F815E009
:100A400004EB001649BA7FBA43EA0C2395F800C0BC
:100A5000A57D86F820208AB2B9B22A4F726245EA93
:100A60000E251BB294F91420B162BCF10C0F4FF0AB
:100A700001017584B38586F82120397026D0BCF138
:100A80000D0F02D1224B23F81020FFF74FFF8BE709
:100A900004EB001393F82020FF2A05D019490132F6
:100AA000012083F820200870FFF740FF164B1B78C9
:100AB0000122092B22727FF472AFB4F8A030144ADD
:100AC00001339BB2A4F8A0309380F8BD114A104EB8
:100AD000157E03EB830303EB830301F166319A0078
:100AE0006B0892FBF3F281FB0213D217C2EBA30255
:100AF00026F81020C9E700BF7C120020984900208A
:100B0000D34D62106C0100201C4A0020D43C002010
:100B1000204A0020503B0020084B997FDA7F914209
:100B20000BD010B49A7F1C69D2B2511CC0B2C9B2AA
:100B30009977A0545DF8044B704770477C120020F1
:100B40000C4AD2F8B83030B41C68D2F8B0501981D1
:100B500000219981611CC3E900152070D2F8B830DA
:100B6000D2F8B0101A685A604FF6F67219609A817E
:100B700030BC70477C12002010B50C4C5E28D4F8B5
:100B8000BC2007D15D209047D4F8BC303E20BDE8A2
:100B9000104018475D2802D0BDE81040104790472C
:100BA000D4F8BC303D20BDE8104018477C1200202E
:100BB0000348D0F8D0300BB1C0301847704700BFA1
:100BC0007C12002030B44FF4167340F2D935012462
:100BD0004FF48071002203811523458104804180F8
:100BE0008280837130BC7047094BB3F8F620B3F8AC
:100BF000F430801A9B1AC00090FBF3F00628A8BFBF
:100C0000062020EAE070C0F19600C0B2704700BF35
:100C10007C120020074B03EB4002B2F80C211205B6
:100C200007D5D3F89821511CC3F89811134483F8C1
:100C30009C0170477C120020436826221A7043688A
:100C40007E225A70436827229A7043680022DA7025
:100C500070472F490A23B1F9D02192FBF3F383EABD
:100C6000E372A2EBE3725A2A30B505DD002BB4BF64
:100C70006FF0B302B422D31A91F8D64142683CB95E
:100C8000244C2478E4073FD491F8D74125073BD47E
:100C900091F8DC41B32C03D891F8D741240733D421
:100CA000B1F9D2110A2491FBF4F103B961B381EADD
:100CB000E17583EAE374A5EBE175A4EBE374B5EBAE
:100CC000440F13DAB4EB450F10DA002908DD002BCE
:100CD000CCBF6E2362231370436800225A7030BD6C
:100CE000002BCCBF6A2366231370F5E7A54205DD10
:100CF0000029CCBF602368231370EDE7002BCCBF25
:100D00006C2364231370E7E720231370E4E700BF2C
:100D10007C12002099490020054B93F879312BB9BA
:100D20004FF4A4735843642390FBF3F0704700BF63
:100D30007C12002090F8603043B9426901210720FD
:100D400082F84430A2F8460082F84810704700BF8D
:100D50000120704700207047027A407A02FB00F0C1
:100D6000704703681B6A184730B405798D4206D373
:100D70004579954203D3036830BCDB68184730BC23
:100D80007047037913F0020308D00369D0E9092002
:100D9000013B101A1840C0B2181A70471846704725
:100DA00001717047704703799B070AD5436A8269CE
:100DB000D154436A01690133B3FBF1F201FB1233F1
:100DC00043627047037913F0010306D0D0E907327C
:100DD000C0689B1A0138184070471846704710B514
:100DE000037913F0010301460ED0FFF7EBFF50B17A
:100DF0000B6A4A69CC68D05C0133B3FBF4F204FBA4
:100E00001233C0B20B6210BD1846FCE790F84B38A5
:100E100030B53BB990F8491890F84A380124DAB255
:100E2000914200D830BDB0F8525804FA03F22A4378
:100E3000A0F852280133F2E7D0E90920131A5842EA
:100E400058417047014B5868704700BF6C01002043
:100E50007047F0B5664C94F8DE31002B46D094F81C
:100E6000DF31002B42D194F8E61194F8E751C1F13B
:100E7000FF0189B200293AD184F8E05184F8E151A8
:100E800084F8E25194F8E03194F8E12194F8E21109
:100E9000B4F8E851B4F8EA6101280BBF12021B0252
:100EA00042EA034343EA02430B4352491722012714
:100EB00007FA02F0184214BF3046284612F1FF32FA
:100EC00001F8010FF4D2012384F8DF31D4F80432A1
:100ED00018225A60D4F8082200215162118841F08A
:100EE000010111801A6842F001021A60F0BDC1F1DF
:100EF000FF036B433C21B4F8E421B2FBF1F61B1273
:100F00000F46052EBED8DFE806F0031125384D5FE9
:100F1000D9B2EB1A5A433C23B2FBF3F20A4484F8E9
:100F2000E05184F8E12184F8E211ABE7B2FBF7F17C
:100F300007FB112291B2DEB2C1F13C02E91A514322
:100F4000B1FBF7F1314484F8E01184F8E15184F801
:100F5000E26197E73C27B2FBF7F107FB1122DEB213
:100F600092B2EB1A5343B3FBF7F3334484F8E061D6
:100F700084F8E15184F8E23184E7B2FBF7F607FB2D
:100F8000162292B25FFA83FCC2F13C02E91A514385
:100F9000B1FBF7F1614484F8E0C184F8E11184F811
:100FA000E2516FE7B2FBF7F107FB1121DEB289B224
:100FB000EB1A5943B1FBF7F1314484F8E01184F89E
:100FC000E16184F8E2515DE73C27B2FBF7F107FBF2
:100FD000112292B2DEB2BA1AEB1A5343B3FBF7F303
:100FE000334484F8E05184F8E16184F8E23149E760
:100FF0007C12002067140020064A074B1068074A3D
:10100000C3F8E401002193F8120283F80C12FF23C5
:1010100013721EE7CC5203087C1200206C010020E2
:10102000034B5A7A0AB901225A720020704700BF56
:101030006C010020174B184A93F81C1231B3174962
:10104000097801BB16495161164A17491268C3F85D
:101050002012117983F82412D168C3F82812134999
:10106000C3F82C12517983F830121169C3F8341285
:101070000F49C3F838129179D26983F83C12C3F84A
:101080004022002070470B495161DDE70A49516158
:10109000DAE700BF7C1200206C0100203A4A0020F1
:1010A000045303089C490020324A0020334A0020A0
:1010B000364A00209053030800540308034BB3F84A
:1010C0004422034B4FF0FF301A8070477C120020FF
:1010D000384A0020034B1A88034B0020A3F844220F
:1010E000704700BF384A00207C120020074B93F95C
:1010F0000030012B06D0064BB3F84822A3F8462255
:10110000002070474FF0FF30704700BF14070020E9
:101110007C12002008B5064B1A782AB1054A1278CD
:10112000012A1CBF00221A70FFF784FF002008BDAF
:101130003A4A0020304A0020064B93F90020064B23
:1011400012B91A70002070471A78002AFAD10122C9
:10115000F7E700BF14070020364A0020114B93F830
:101160004A2283F8FD2093F84B2283F8FE20B3F83F
:101170004C22A3F8F42093F8532283F85022B3F8BA
:101180005822A3F85422B3F85A22A3F85622B3F8EF
:101190006022A3F85C22B3F86222A3F85E2200204A
:1011A000704700BF7C120020114B93F8FD2083F89C
:1011B0004A2293F8FE2083F84B22B3F8F420A3F8D8
:1011C0004C2293F8502283F85322B3F85422A3F808
:1011D0005822B3F85622A3F85A22B3F85C22A3F897
:1011E0006022B3F85E22A3F862220020704700BF9D
:1011F0007C1200200020704700207047084A0949EF
:10120000B2F864324B8292F8663203EB83035B00E0
:101210000B8292F8783282F86A320020704700BF61
:101220007C120020503B0020084A094B518AA3F849
:101230006412128A0A21B2FBF1F283F8662293F853
:101240006A2283F878220020704700BF503B0020BC
:101250007C12002030B1007910F1FF3018BF4FF040
:10126000FF3070474FF0FF307047144A144B5288DC
:1012700002F0010283F8792293F8132283F87A228C
:1012800093F8142283F87B2293F8152283F87C22AA
:10129000B3F81622A3F87E2293F8182283F880224E
:1012A00093F8192283F8812293F8102283F882227E
:1012B00093F81A2283F8832200207047C038002058
:1012C0007C1200200A4BD3F88422B3F88812518094
:1012D000B3F88A12A2F84C10B3F88C129180B3F8CC
:1012E0008E12B3F89032D18013800020704700BF77
:1012F0007C1200200D4B93F89222762101FB0232E2
:101300000020B2F89612A3F88812B2F8E012A3F8FF
:101310008A12B2F89812A3F88C12B2F89A12B2F8A4
:101320009422A3F88E12A3F8902270477C1200201A
:101330000A4A0B4BB2F8F613D980B2F8F8131981A8
:10134000B2F8FA135981B2F8FC139981B2F8FE137E
:10135000B2F80024D9811A82002070477C12002044
:10136000F83100200A4A0B4BD188A3F8F6131189F3
:10137000A3F8F8135189A3F8FA139189A3F8FC1381
:10138000D189128AA3F8FE13A3F800240020704725
:10139000F83100207C1200201E4B1F4993F80224D4
:1013A00030324A7693F89222762101FB02320020F5
:1013B00092F8DB1283F8031492F8AE1283F8041447
:1013C00092F8AF1283F8051492F8B01283F806145D
:1013D000B2F8C812A3F80814B2F8C612A3F80A1497
:1013E00092F8E31283F80C1492F8071383F80D14A3
:1013F00092F8081383F80E1492F8021383F80F146E
:1014000092F8031392F8042383F8101483F811243C
:10141000704700BF7C1200206C0100200D4A92F83A
:101420009232762101FB032392F8121483F8FA1208
:1014300092F8131483F8FE1292F8141483F8FB1236
:1014400092F8151492F8162483F8FC1283F8FD2202
:10145000002070477C1200200D4B93F892227621D9
:1014600001FB0232002092F8FA1283F8121492F86B
:10147000FE1283F8131492F8FB1283F8141492F8F6
:10148000FC1292F8FD2283F8151483F81624704795
:101490007C1200200F4B104993F8022430320A7757
:1014A00093F8172430328A7793F8D0241A2101FB5D
:1014B000023202F2344103F5836302F24C4251F8E6
:1014C000040B43F8040B9142F9D10A881A800020DA
:1014D000704700BF7C1200206C0100200A4A92F87D
:1014E000D0341A2101FB032303F2344302F5836154
:1014F00002F5866251F8040B43F8040B9142F9D1CE
:101500000A881A80002070477C12002010B5124A09
:10151000124992F8023492F8920230334B7602F577
:101520002571762300FB031302F2D141002002F261
:10153000DA421C7A0C705C7A4C709C7A8C709C89B4
:1015400022F810400130032803F1060301F10301E2
:10155000EFD1002010BD00BF7C1200206C010020E4
:10156000084B93F8682283F89222013283F8022410
:1015700093F8692283F8D024013283F817240020DD
:10158000704700BF7C1200200A4930B50A4C002287
:1015900001F59C60135DA3F16105052D9CBF203B07
:1015A000DBB283540132072AF4D1002081F8E7042A
:1015B00030BD00BF7C1200203B770308094B93F835
:1015C000E824012A08D893F8E924012A02D0032A42
:1015D00018BF032283F8EE24B3F8F224A3F8EC2416
:1015E000002070477C12002010B5044623790E2B92
:1015F00000D110BD032B04D1D4F809309868FFF74F
:10160000F3FF0E34F2E70B49D1F8F4349A6813462D
:1016100018790E280CD19B1A5A10074B5343013BE3
:1016200091F8FD2493FBF2F3013381F8FC34704709
:101630000E33EDE77C120020B76DDBB62DE9F047E5
:10164000184B04461E2093F8009093F801A09D7853
:10165000B3F80480DF881E7A18F050F920B11FB16A
:10166000B84601254FF000090F4B1B78DA070BD461
:101670000E4A92F803253AB9012E11D0022E03D159
:1016800013F0020F08BF012584F8009084F801A030
:10169000A570A4F80480E78026722046BDE8F08794
:1016A0003546F1E7A0490020994900207C1200202E
:1016B00010B582B002AB322203F8082D064A046846
:1016C0008188CDF801401846ADF80510D2F82435D0
:1016D000984702B010BD00BF7C1200200E4B41683D
:1016E000B3F9D4310A2293FBF2F31B0103F5B9538A
:1016F0004FF4B4721433B3FBF2F3084A03F00F0350
:1017000013441A680A605A684A601B7A0B7243686D
:1017100000225A72704700BF7C1200203854030820
:10172000084B93F8793107EE900A4BB9F8EEE77A57
:101730009FED057A9FED050AA7EE870A21F0C6BE48
:10174000704700BF7C1200206766E63F0000004241
:10175000012806D003D3022807D000207047F0F7F5
:10176000D1BF044BD3F828057047024BD3F82C05A2
:10177000704700BF7C120020024B0146D3F8500591
:10178000F1F7AEBA7C1200202DE9F041294D2A4A2A
:10179000D5F85435B5F86075B5F85C6582FB034241
:1017A000DB17C3EBA2031FFA83F8474503D1B5F853
:1017B0006235B34236D002680F463423511C0160B3
:1017C000137002680023511C0446016013704146E7
:1017D000F3F772FD31462046F3F76EFD47F6FF71D1
:1017E0002046F3F769FD47F6FF712046F3F764FDE5
:1017F00047F6FF712046F3F75FFD204647F6FF717D
:10180000F3F75AFD2368A5F860854FF6FF721A803A
:101810002368A5F862650233C5F86475236001206A
:10182000BDE8F081D5F86435044ACB1A9342C2D89A
:101830000020F5E77C1200206766666680841E0043
:1018400003687F22591C01601A7003680022591C2A
:1018500001601A7003684FF0FF321A605A609A6094
:101860009A8103680E3303600120704703687E226B
:10187000591C10B501601A7003680022591C0160E0
:101880001A704FF6FF710446F3F7F0FC0F4B93F814
:101890007325B3F88C158AB92046F3F7E7FC204688
:1018A00047F6FF71F3F7E2FC23684FF0FF321A604E
:1018B0005A60236808332360012010BD93F89235E5
:1018C00091FBF3F12046F3F7D1FCE8E77C1200200E
:1018D00008B5A0F10103B3FA83F302284FEA5313CA
:1018E00001D0184608BD0F2017F0E2FF28B9054BBC
:1018F0001B7803F00103184608BD0F20BDE808401F
:1019000017F0FCBF9949002038B5224D4468B5F85E
:1019100094355A0505D520461F49BDE8384021F0C9
:1019200078BE180505D520461C49BDE8384021F091
:1019300070BE590605D520461949BDE8384021F04A
:1019400068BEDA0705D520461649BDE8384021F0C3
:1019500060BE9B0705D520461349BDE8384021F0FD
:1019600058BE252017F0CAFF28B120460F49BDE810
:10197000384021F04EBE95F896352BB120460C49E3
:10198000BDE8384021F045BE20460A49BDE8384050
:1019900021F03FBE7C12002030A4030835A40308C8
:1019A0003AA403083FA4030844A4030849A4030875
:1019B0004EA4030853A40308074B93ED087AD3ED14
:1019C000097AB4EEE77AF1EE10FA03DD03494068D4
:1019D00021F01FBE704700BF6C01002058A403080F
:1019E0007FB5124B1249064618680B78D0B1426990
:1019F000D45C4A78036953F822508B788DF80F3005
:101A000028B10B7A1BB10DF10F01FFF7AAF99DF870
:101A10000F30009322462B4606497068F6F780FF88
:101A200004B070BD3F24044DE7E700BF9C4900208F
:101A3000A04900205DA403085BA4030837B5044651
:101A40001C4800EB4303B3F87A5105F00F0039B19D
:101A5000611CD8B102288CBF20239C2323700C4624
:101A6000B2B1C5F30315FFF773FE3C23012D1249F4
:101A7000B0FBF1F191FBF3F203FB12130AD00F4913
:101A8000204603B0BDE83040F6F74ABF9B23E5E7A8
:101A90001546E8E7642542F21071B0FBF1F0B0FBA7
:101AA000F5F105FB1100009005492046F6F738FFD7
:101AB00003B030BD7C12002040420F0067A4030831
:101AC00071A40308037840680122053B1146B5E77D
:101AD00006494068B1F88C25D1F854350449534380
:101AE00042F2107293FBF2F2F6F71ABF7C1200205A
:101AF00080A4030807B5084BD3F88422917A137A9F
:101B00000191527A00920549054A4068F6F708FFAC
:101B100003B05DF804FB00BF7C12002089A4030819
:101B200085A4030807B5084BD3F88422917D137D63
:101B30000191527D00920549054A4068F6F7F0FE92
:101B400003B05DF804FB00BF7C12002089A40308E9
:101B500098A4030807B5084BD3F88422117C937B23
:101B60000191D27B00920549054A4068F6F7D8FEFC
:101B700003B05DF804FB00BF7C12002089A40308B9
:101B80009CA40308054A064992F8693292F8682233
:101B9000406801330132F6F7C3BE00BF7C1200205B
:101BA000A0A403080B4B4068B3F9D4310A2293FB7D
:101BB000F2F31A0102F5B9524FF4B4711432B2FBC8
:101BC000F1F2C2F1080202F00F0260320249F6F7A8
:101BD000A7BE00BF7C120020A6A4030837B5114998
:101BE000456891F89735022B044619D0B1F88C0559
:101BF00091F8923590FBF3F0FEF7F6FF2870B1F8FC
